:020000040800F2
:1000000000800020F5C800084FD70008D19C0008E8
:1000100000000000000000000000000000000000E0
:1000200000000000000000000000000051D70008A0
:10003000000000000000000053D70008E19C000809
:1000400029C900082BC900082DC900082FC90008BC
:1000500031C9000833C9000835C9000833E2000877
:1000600039C90008319D00083DC900083FC9000892
:1000700041C9000843C9000845C9000847C900082C
:1000800049C900084BC900084DC900084FC90008FC
:1000900051C90008519D000855C9000857C90008FA
:1000A00059C900085BC900085DC90008419D0008E6
:1000B00061C9000863C9000865C9000867C900086C
:1000C000EDAF16204A62304029BD56B31544E9BF52
:1000D00077900D9CFE0B88C07E2615FA83807340B6
:0800E0000FCE674B80D541C033
:1000E800000000000000244000000000000059400B
:1000F800000000000088C3400000000084D797413A
:100108000080E03779C34143176E05B5B5B893460B
:10011800F5F93FE9034F384D321D30F94877825AD7
:080128003CBF737FDD4F15752C
:1001300001000000000000000A00000000000000B4
:100140006400000000000000E80300000000000060
:100150001027000000000000A08601000000000041
:1001600040420F0000000000809698000000000050
:1001700000E1F5050000000000CA9A3B0000000005
:1001800000E40B540200000000E87648170000006D
:100190000010A5D4E800000000A0724E180900006D
:1001A00000407A10F35A00000080C6A47E8D030040
:1001B0000000C16FF286230000008A5D784563016C
:1001C000000064A7B3B6E00D0000E8890423C78AE5
:1001D00000B581B06946002008700A4A1168012004
:1001E00003021943116000F00FF8002803D069469C
:1001F0000120087001E009F051FD6846007801B067
:0802000000BDC04600200240D1
:1002080000B583B0029001A9002008701748007853
:10021800002824D0164800680090144801787D20F2
:10022800C0000BF041FA014600980BF03DFA0DF0C2
:100238004EFD00280FD10298032808D80299002201
:10024800D0430DF036FD02980A49086002E001A982
:100258000120087002E001A90120087002E001A94C
:100268000120087001A8007803B000BD9C000020A0
:0802780098000020880000201E
:100280000348027803490868801808607047C04630
:080290009C000020B00F0020CB
:0C029800014800687047C046B00F00200D
:1002A40000B583B00290FFF7F5FF0190029800902B
:1002B4000098401C002804D0074801780098401892
:1002C4000090FFF7E7FF0199401A0099884200D295
:0C02D400F7E703B000BDC0469C0000200E
:1002E00000B589B0079006A9002008700590049019
:1002F00002900798002803D108A90120087066E140
:1003000007983C21405C0128FFD10798006900282C
:1003100005D007980069012149058842FFD1079857
:10032000806D002808D1079805F040FB0799002050
:10033000C865079954228854079800680DF0BBFBE4
:10034000002812D10798006800F052F9A24800680E
:10035000A2490BF0ADF94000801C029002980028E1
:1003600003D00298401E0290F8E7079800680DF04D
:10037000A2FB00280BD10799886D102210438865D5
:10038000079AD16D01200143D16506A9087007982D
:1003900000680CF074FB03900798806DC00600287D
:1003A00000D509E10398002800D005E10798806D89
:1003B00002210843012109028843079988650798AB
:1003C00000680DF082FB002800D0A1E0079881684A
:1003D000027E92031143427ED2031143827E520376
:1003E0001143026B531E9A4112031143C268114319
:1003F0000191C07C0006002806D5079800690121FC
:10040000C9078843009002E001204005009001994F
:100410000098014307982C22805C40000143059816
:100420000843059007982021405C012813D10798C4
:10043000807E002805D10598012109040843059014
:1004400009E00799886D2022104388650799C86DD7
:1004500001221043C8650798406A002809D0079810
:10046000416A072292011140806A014305980843BE
:10047000059007980068C0685949084005990843E5
:1004800007990968C86007984168032292071140DC
:10049000C06C014304980843049007983C21405CD9
:1004A00001280FD1079948680322920710400A6C6F
:1004B00010434A6C1043896C084304990843012196
:1004C0000843049007980068006946490840049969
:1004D000084307990968086107984068032189075C
:1004E000884215D0079840680121890788420FD0BB
:1004F000079840680121C907884209D03A4908682D
:100500000F2293049843079A52681A408018086093
:10051000079908684A6B00210CF0F9FA07990868F6
:100520008A6B32490CF0F3FA07980069002807D16A
:1005300007980168886A0F22D2431043886216E048
:100540000798006901214905884210D10798006881
:10055000806A0799C8698000021F1C2002400F2092
:10056000C04390400A6E104309688862FFE707980D
:10057000006800210DF0B1FA0799496B88420BD150
:1005800007990020C8650798806D01210843022162
:100590008843079988650EE00798806D102108430D
:1005A0000221884307998865079AD16D012001438C
:1005B000D16506A9087007E00799886D10221043DD
:1005C000886506A901200870069808A9087008A87F
:1005D000007809B000BDC04698000020400D03001F
:1005E0000102DEFF02FCFF1F0827014004FFFF0796
:1005F00081B00090009880680121090708430349F1
:1006000008400099886001B07047C046E8FFFF7F4E
:1006100081B000900098806803490840801C0099D0
:0C062000886001B07047C046E8FFFF7F13
:10062C0000B585B0039000200190039800680DF090
:10063C0046FA00285BD10398006880682F4908426D
:10064C000CD00399886D102210438865039AD16DE4
:10065C0001200143D16504A908704BE003980068A0
:10066C0000F062F826480CF068FA000200280DD55C
:10067C002448006824490BF015F8401C019001989F
:10068C00002803D00198401E0190F8E70398407EA3
:10069C0001282CD0FFF7FAFD02900398006800683F
:1006AC00C007002823D1039800680DF008FA002831
:1006BC0003D10398006800F037F8FFF7E7FD0299C3
:1006CC00401A032812D3039800680068C00700285A
:1006DC000CD10399886D102210438865039AD16D53
:1006EC0001200143D16504A9087003E0D5E704A9F2
:1006FC000020087004A8007805B000BD1700008029
:0C070C000827014098000020400D030069
:1007180081B000900098806803490840001D009946
:0C072800886001B07047C046E8FFFF7F0A
:1007340081B000900098806803490840401C0099EB
:0C074400886001B07047C046E8FFFF7FEE
:1007500000B585B0039002910192039800680CF0F7
:100760008EF9002860D103985421405C012803D100
:1007700004A9022008705DE00399542201208854E6
:1007800003980068C068C00700280FD1039800686C
:100790000DF09BF9002803D003980068FFF738FF9D
:1007A00003980168C86801221043C8600398FFF7E6
:1007B0003DFF0146684601700078002833D1039858
:1007C000806D0121090208431C490840039988658E
:1007D00003990020C8650398016D1948C862039801
:1007E000016D184808630398016D17484863039822
:1007F00001681C2008600399542200208854039843
:10080000016848681022104348600399086D096820
:100810004031029A019B0CF091FA694608700398E6
:100820000068FFF779FF02E069460220087000982F
:1008300004A9087004A8007805B000BDFEF1FFFF10
:0C084000A7DB00086FCB000885CB000888
:10084C0000B59DB01B901A9119A900200870179043
:10085C001B9800690121C907884204D01B980069C4
:10086C00E649884200D1FFE71B985421405C0128DF
:10087C0003D11CA902200870BCE11B995422012051
:10088C0088541B9800680CF0F4F8002800D0A2E102
:10089C001A984068022800D15BE11B98006901217D
:1008AC00C907884204D01B980069D449884206D1F4
:1008BC001B9800681A99096800F0AEF9F1E01B98D2
:1008CC00016E1A9843681F2213400F229A409143DD
:1008DC00169100684003002807D11A9800681F2160
:1008EC0089060840800E1590C2E01A980078C0075F
:1008FC00002802D000201490B8E01A9800788007E5
:10090C00002802D501201390AEE01A980078400719
:10091C00002802D502201290A4E01A980078000753
:10092C00002802D5032011909AE01A980078C0068E
:10093C00002802D50420109090E01A9800788006C8
:10094C00002802D505200F9086E01A980078400602
:10095C00002802D506200E907CE01A98007800063C
:10096C00002802D507200D9072E01A984078C00735
:10097C00002802D008200C9068E01A984078800774
:10098C00002802D509200B905EE01A9840784007A9
:10099C00002802D50A200A9054E01A9840780007E3
:1009AC00002802D50B2009904AE01A984078C0061E
:1009BC00002802D50C20089040E01A984078800658
:1009CC00002802D50D20079036E01A984078400692
:1009DC00002802D50E2006902CE01A9840780006CC
:1009EC00002802D50F20059022E01A988078C007C5
:1009FC00002802D01020049018E01A988078800704
:100A0C00002802D5112003900EE01A9801680120ED
:100A1C00820411401220002301939142029001D0D4
:100A2C000198029002980390039804900498059002
:100A3C0005980690069807900798089008980990D2
:100A4C0009980A900A980B900B980C900C980D90A2
:100A5C000D980E900E980F900F9810901098119072
:100A6C001198129012981390139814901498159042
:100A7C00169815991A9A52681F231A4091400843E8
:100A8C001B9908661A9840688008401C1B99C96914
:100A9C00884206D81B9800681A9A516812680CF0A4
:100AAC0080F81B9800681A9A1168926800F0C2F8D6
:100ABC001A98C078000600284AD551480CF03DF829
:100ACC0018901A9800684F4988421DD118A8807850
:100ADC000006002818D418990120C0050143484885
:100AEC000DF0B7F84A4800684A490AF0DBFD0146A8
:100AFC000C2048430C3017901798002803D01798F7
:100B0C00401E1790F8E723E01A9800683E49884287
:100B1C000CD118A8C078C007002807D1189901205B
:100B2C000006014336480DF094F811E01A9800685D
:100B3C00364988420CD118A880784006002807D482
:100B4C0018990120800501432D480DF082F8FFE72C
:100B5C0040E01B9800690121C907884204D01B980A
:100B6C0000692649884205D11B9800681A990968C2
:100B7C0000F074F81A98C078000600282AD520488E
:100B8C000BF0DBFF18901A9800681E49884207D1B9
:100B9C0018990120C005814319480DF05AF819E045
:100BAC001A9800681849884207D118990120000644
:100BBC00814313480DF04DF80CE01A980068134966
:100BCC00884207D118990120800581430C480DF00B
:100BDC0040F8FFE707E01B99886D202210438865D9
:100BEC0019A9012008701B995422002088541998C7
:100BFC001CA908701CA800781DB000BD0400008062
:100C0C0008270140001000B0004000B8002000B4DC
:080C1C0098000020400D0300C8
:100C240082B001900091009A034802400199886AB9
:0C0C34001043886202B07047FFFF070009
:100C400083B00290019100920298406901990A02D2
:100C5000904300991140034A1140084302994861AA
:080C600003B0704700FFFF071D
:100C680082B0019000910098C24304480243019960
:100C7800886A1040886202B07047C0460000F8FFDA
:100C880000B58BB009900020079004900998542172
:100C9800405C012803D10AA902200870C5E009991F
:100CA80054220120885409980CF021FF08A90870E3
:100CB800099800680CF0DDFF002800D0A9E0099829
:100CC800806D02210843012109028843099988653A
:100CD80009980068C0685749084006900998016853
:100CE800C868554A1040C860002005900598072834
:100CF8002DD8099800680BF06DFF099800680CF072
:100D0800C0FF002817D00798401C079007984C4947
:100D180088420FD30998806D102108430221884327
:100D28000999886509995422002088540AA9012044
:100D380008707AE0E1E7099800680BF058FF01466F
:100D48000498401804900598401C0590CEE7059932
:100D580004980AF0A9FC04900998006800F072F859
:100D6800099800680BF04CFF002817D133480BF0A6
:100D780050FF02900298800C07280FD30298800C2D
:100D8800C11E0120884001900198400801900198F7
:100D9800002803D00198401E0190F8E709980068E0
:100DA80004990CF078FF0998006800F059F8FFF7EB
:100DB8006FFA0390099800680CF05BFF002819D0BF
:100DC800FFF766FA0399401A032812D309980068B6
:100DD8000CF04FFF00280CD00999886D10221043A1
:100DE8008865099AD16D01200143D1650AA9087067
:100DF8001BE0DFE7069A09980168C8681043C860D5
:100E08000998806D01210843022188430999886562
:100E180004E00999886D10221043886509995422C5
:100E28000020885408980AA908700AA800780BB00E
:100E380000BDC04603800000FC7FFFFF082701407B
:040E480000F20200B2
:100E4C0081B000900098806803490840401C0099CC
:0C0E5C00886001B07047C046E8FFFF7FCF
:100E680081B000900098806803490840801C009970
:0C0E7800886001B07047C046E8FFFF7FB3
:100E840070B582B0024601A802700091002140565C
:100E9400002815D4002401A908570322D34318407D
:100EA400164A805809578C07E50EFF24AC40A0432E
:100EB400009CA401E4B2AC4020431940885019E0DE
:100EC40001A908780F24204008380322D34318408E
:100ED400094A8058002549578D07EE0EFF25B54075
:100EE400A843009DAD01EDB2B54028432140083927
:100EF4001940885002B070BD1CED00E000E400E031
:100F040081B001466846017000214056002807D48C
:100F1400684601781F20014001208840014908608B
:080F240001B0704700E100E09C
:100F2C0081B00146684601700021405600280BD460
:100F3C00684601781F200140012088400349086061
:100F4C00BFF34F8FBFF36F8F01B0704780E100E0AC
:100F5C0000B583B001900198401E000E002802D00D
:100F6C000120029010E00198401E09490860002001
:100F7C000090C0430321FFF77FFF009805490860EC
:100F8C00054A072111600290029803B000BDC046CB
:0C0F9C0014E000E018E000E010E000E0CD
:100FA80000B583B001900198002803D102A901205F
:100FB800087050E00198407F002805D10199002071
:100FC800087701980CF08BFE019902204877019868
:100FD800007900280CD101980168214848610198DE
:100FE80000688068182188430199096888600AE0C8
:100FF80001988168C2680BF0B5FC002803D002A9EB
:101008000120087027E001984079002805D101984F
:1010180001680020C043086103E001990869096874
:1010280008610198006880686021884301994A69CD
:1010380010430968886001980068806880218843A7
:1010480001998A69104309688860019901204877E5
:1010580002A90020087002A8007803B000BDC046AD
:04106800B71DC104EB
:10106C0000B585B003900398002803D104A9012092
:10107C00087066E003980190006834494018142108
:10108C000AF010FB019980000864039925220220C4
:10109C0088540398016808682D4A1040086003982A
:1010AC0002908268C1680A4301690A4341690A4394
:1010BC0081690A43C1690A43016A0A4301680868E5
:1010CC0010430860039800F045F8039880680121EC
:1010DC008903884202D1039900204860039948682B
:1010EC003F221040496C08600399C86C896C4860B9
:1010FC000398406800280FD00398406804280BD848
:10110C00039800F049F80398016D002008600399DA
:10111C00886D496D486006E00399002008650399C5
:10112C0048650399886503990020C86303992522B3
:10113C0001208854039924220020885404A90020FB
:10114C00087004A8007805B000BDC046F8FFFDBFCC
:04115C000F80FFFF02
:1011600000B583B002900299086C032290430B4AA9
:101170008018486402980078083814210AF098FA18
:10118000019002990648886401991F2001400120BE
:1011900088400299C86403B000BDC0460008024000
:0411A0008008024081
:1011A40082B00190019840683F2108400090009867
:1011B4008000084940180199086501990648486566
:1011C4000098411E03200140012088400199886550
:0C11D40002B07047FC08024040090240D5
:1011E00084B003900291019200930399C86C896CBA
:1011F00048600398006D002803D00399886D496DFD
:1012000048600398006C1C210840012282400F496D
:1012100008681043086000980399096848600398BB
:101220008068102808D1019803990968886002989D
:1012300003990968C86007E0029803990968886003
:10124000019803990968C86004B07047040002401F
:1012500000B583B002904C48006801900298006885
:101260000068009001980299096C1C221140C84046
:101270004007002822D568460078400700281DD581
:101280000298006800688006002805D4029801686A
:1012900008680422904308600298006C1C210840F2
:1012A0000422824039490868104308600298006BA4
:1012B000002802D00298016B884763E001980299E8
:1012C000096C1C221140C840800700282AD56846B6
:1012D00000788007002825D50298006800688006FD
:1012E000002809D40298016808680A22904308601F
:1012F00002992522012088540298006C1C21084084
:101300000222824021490868104308600299242281
:10131000002088540298C06A002802D00298C16A4E
:1013200088472FE001980299096C1C221140C8409F
:101330000007002826D5684600780007002821D538
:101340000298016808680E22904308600298016CB8
:101350001C200140012003468B400C4A11681943B0
:1013600011600299C86302992522885402992422A7
:10137000002088540298406B002802D00298416BEC
:101380008847FFE703B000BD0000024004000240B0
:1013900010B588B006900591039302921C4800781E
:1013A000012803D107A9022008702DE01849012067
:1013B00008701749002048607D20C00000F034F814
:1013C000014601A801700078002817D1069801286D
:1013D00005D10598039B029A00F07AF803E005987E
:1013E000029900F019F87D20C00000F01DF801A955
:1013F0000870069A0749086890430860044900206D
:101400000870019807A9087007A8007808B010BDF7
:10141000840F00201420024008B4024B9C4608BCF4
:081420006047C04601000020F6
:1014280000B585B00390FEF733FF0190012000045A
:10143800029021480068029908420FD00398401C86
:1014480000280AD0FEF724FF0199401A0399884220
:1014580003D304A90320087029E0EAE716490868BD
:10146800164A10400290164808600298002806D0D4
:1014780002981449486004A90120087017E00E4832
:101488000068400300280FD50398401C00280AD0A4
:10149800FEF7FEFE0199401A0399884203D304A976
:1014A8000320087003E0EAE704A90020087004A8F4
:1014B800007805B000BDC04610200240FA83000045
:0814C800FB830000840F0020EB
:1014D00084B00390019300920749086801221043E9
:1014E0000860009803990860BFF36F8F0198039913
:0C14F000486004B07047C0461420024061
:1014FC0081B06946002008700A480068C00F0028B7
:10150C000CD009490948086009480860054800687A
:10151C00C00F002802D06946012008706846007888
:10152C0001B0704714200240082002402301674597
:04153C00AB89EFCDBB
:1015400000B583B002A90120019008707D20C00081
:10155000FFF76AFF019A08480168D207114301604A
:101560000068C00F002802D002A90020087002A85D
:0C157000007803B000BDC046142002400B
:10157C0081B06946012008700A48006840000028C4
:10158C000CD50949094808600948086005480068F5
:10159C004000002802D46946002008706846007894
:1015AC0001B07047142002400C2002403B2A19085D
:0415BC007F6E5D4C95
:1015C00000B583B002A90120019008707D20C00001
:1015D000FFF72AFF019A084801689207114301604A
:1015E00000684000002802D502A90020087002A867
:0C15F000007803B000BDC046142002408B
:1015FC0000B585B0039002912E480078012803D1E4
:10160C0004A90220087051E02A49012008702949D8
:10161C00002048607D20C000FFF700FF014601A8B4
:10162C000170007800283BD103990420486003988E
:10163C00006804280AD10398406800F03FF87D2028
:10164C00C000FFF7EBFE01A9087029E00299002009
:10165C00C04308600398806800900098039A9168D2
:10166C00D2688918884216D203984068009900F015
:10167C0033F87D20C000FFF7D1FE014601A80170B0
:10168C000078002803D000980299086003E00098C5
:10169C00401C0090E1E7084908680222904308606A
:1016AC00044900200870019804A9087004A8007867
:0C16BC0005B000BD840F00201420024087
:1016C80081B00090009804490A681043012212046E
:0C16D8001043086001B07047142002406D
:1016E40083B00290019107490868074A10400090AE
:1016F400009A0198C0001043044A1043086003B0E4
:101704007047C0461420024007E0FFFF02000100BA
:1017140000B587B0059035480078012803D106A9A3
:10172400022008705EE03149012008702F49002032
:10173400486005980078C007002805D0059A5068CD
:101744009168D26800F056F80598006806210840B0
:10175400062806D1059A50699169126900F064F867
:101764001DE0059800788007002809D500F074F87A
:101774000490049905980269084600F055F80EE0B3
:10178400059800784007002809D500F073F8049004
:10179400059948698969049A00F046F8FFE77D20B5
:1017A400C000FFF73FFE014603A80170007800283F
:1017B40012D10F4902910868012252040192104388
:1017C40008607D20C000FFF72DFE019A029903AB4B
:1017D4001870086890430860044900200870039852
:1017E40006A9087006A8007807B000BD840F002081
:0417F400142002407B
:1017F80083B00290019100920298012806D10098C6
:101808000004019908430649086005E000980004AF
:10181800019908430149086003B07047302002402D
:041828002C2002402E
:10182C0084B0039002910192084908680090039AD1
:10183C0000989043FF22904300900098029A104326
:10184C00019A1043086004B07047C0462020024043
:10185C0081B004480068044908400090009801B029
:0C186C007047C0462020024000604F077B
:1018780082B009480068C0B200900098AA2805D034
:101888000098CC2802D0BB20019001E0009801907C
:0C189800019802B07047C04620200240BA
:1018A40000B581B00090009907200860009A506844
:1018B400114608310C3200F00FF8FFF7DBFF0099F6
:1018C4000861FFF7C9FF00998861009901484861E0
:0818D40001B000BD00604F07E8
:1018DC0083B0029001910092029801280CD10E481D
:1018EC0002683F210A40019B1A6000680904084005
:1018FC00000C009908600BE0064802683F210A4082
:10190C00019B1A60006809040840000C00990860EB
:0C191C0003B07047302002402C20024035
:101928008AB00990089100200790089800680799E4
:10193800C840002800D130E108980068079A0121C2
:101948009140084006900698002800D121E10898A7
:10195800406803210840012805D008984068032101
:10196800084002282AD10998806805900798400005
:10197800032181400598884305900898C168079815
:1019880040008140059808430590059809998860AA
:101998000998406805900798012181400598884377
:1019A800059008984068102108400109079881406F
:1019B8000598084305900598099948600898406873
:1019C80003210840032814D00998C0680590079897
:1019D8004000032181400598884305900898816854
:1019E8000798400081400598084305900598099993
:1019F800C860089840680321084002281ED1099849
:101A08000799C90889004018006A05900798400797
:101A1800C00E0F21814005988843059008980169F8
:101A280007984007C00E814005980843059005981F
:101A38000999079AD20892008918086209980068DB
:101A4800059007984100032002468A400599914372
:101A58000591089949680140079840008140059818
:101A680008430590059809990860089880798007C7
:101A7800002800D18DE00798032188434849405841
:101A8800059007988007C00E0F218140059888436C
:101A98000590099805210907884202D10020049081
:101AA8001DE009983F49884202D10120039014E0C3
:101AB80009983D49884202D1022002900BE0099919
:101AC8003A4A0320052300939142019001D00098DF
:101AD8000190019802900298039003980490049949
:101AE80007988007C00E814005980843059005981F
:101AF8000799032291432A4A88502D480068059087
:101B0800069905988843059008988079C0060028AA
:101B180003D5069905980843059005982449086057
:101B28002448006805900699059888430590089808
:101B380080798006002803D5069905980843059002
:101B480005981C4908601C48006805900699059886
:101B580088430590089880798007002803D506995E
:101B680005980843059005981349086013480068CC
:101B78000590069905988843059008988079C007CC
:101B8800002803D0069905980843059005980B4945
:101B980008600798401C0790C7E60AB07047C0461F
:101BA800601802400004005000080050000C00506B
:101BB80000180240041802408418024080180240AD
:101BC80000B581B0694608800D4800680988084258
:101BD80006D0684601880A4A116000880BF036F979
:101BE8000848006869460988084206D0684601889E
:101BF800044A1160008806F033FF01B000BDC046FA
:081C08000C1802401018024004
:101C10000349086801221202104308607047C04659
:041C20000070004010
:101C24000349086801221202904308607047C046C5
:041C340000700040FC
:101C380000B583B001901749086803225202904307
:101C4800019A10430860019801214902884219D17C
:101C58001148016806204843104909F025FD401C39
:101C680000900F480068400500280BD50098002810
:101C780003D00098401E009003E002A903200870DA
:101C880003E0EEE702A90020087002A8007803B07C
:101C980000BDC046007000409800002040420F0080
:041CA8001470004074
:101CAC0010B588B006900698002803D107A901202A
:101CBC000870C0E206980078C007002873D0FA4874
:101CCC000068382108400490F84800680321084057
:101CDC0003900498102802D10398032802D004988A
:101CEC0008280DD1F24800688003002807D5069813
:101CFC004068002803D107A9012008709BE252E03C
:101D0C000698406801210904884206D1E849086810
:101D1C0001221204104308601AE00698406805215D
:101D2C00090488420AD1E249086801229304184345
:101D3C000860086812041043086009E0DC49086870
:101D4C0001221304984308600868920490430860C9
:101D5C0006984068002813D0FEF798FA0590D448EE
:101D6C000068800300280AD4FEF790FA0599401AFF
:101D7C00652803D307A9032008705CE2EFE712E0A3
:101D8C00FEF784FA0590CA480068800300280AD53B
:101D9C00FEF77CFA0599401A652803D307A903209E
:101DAC00087048E2EFE7069800788007002800D416
:101DBC0090E0BD480068382108400490BB4800689A
:101DCC000321084003900498102802D1039802289C
:101DDC0002D00498002834D1B5480068400500288A
:101DEC0007D50698C068002803D107A90120087000
:101DFC0021E2B04908687F2212029043069A526988
:101E0C00120210430860049800280FD1A8480268F9
:101E1C000721C9028A43069B1B691A4302600068AA
:101E2C000840C10AA448C840A4490860A4480068F6
:101E3C00FEF7E4F9002803D007A901200870FAE1A5
:101E4C0048E00698C06800282BD0994908680722FA
:101E5C00D2029043069A1269104308600868012266
:101E6C00120210430860FEF711FA0590F64800685C
:101E7C00400500280AD4FEF709FA0599401A0328F0
:101E8C0003D307A903200870D5E1EFE7EF490868F1
:101E9C007F2212029043069A526912021043086084
:101EAC0018E0E94908680122120290430860FEF725
:101EBC00EDF90590E4480068400500280AD5FEF7C6
:101ECC00E5F90599401A032803D307A903200870E4
:101EDC00B1E1EFE7069800780007002848D5D8480C
:101EEC0000683821084018280DD1D94800688007AF
:101EFC00002807D506988069002803D107A901207E
:101F0C00087098E134E006988069002818D0D04910
:101F1C000868012210430860FEF7B8F90590CC4818
:101F2C000068800700280AD4FEF7B0F90599401A1A
:101F3C00032803D307A9032008707CE1EFE717E01F
:101F4C00C3490868012290430860FEF79FF9059089
:101F5C00BF480068800700280AD5FEF797F9059955
:101F6C00401A032803D307A90320087063E1EFE7A5
:101F7C00069800784007002800D4ADE002A90020A4
:101F8C000870AF4800683821084020280DD1B348AC
:101F9C0000688007002807D506988068002803D1C0
:101FAC0007A90120087046E196E0AA480068C00025
:101FBC0000280CD4A7480268012109070A430260D3
:101FCC00006808400190019802A901200870A248FD
:101FDC000068C005002818D49F4908680122120225
:101FEC0010430860FEF752F905909B480068C00545
:101FFC0000280AD4FEF74AF90599401A032803D39E
:10200C0007A90320087016E1EFE7069880680128FD
:10201C0005D19249086801221043086016E0069821
:10202C008068052809D18D4908680422104308608E
:10203C00086801221043086008E0884908680122FA
:10204C0090430860086804229043086006988068F2
:10205C00002814D0FEF71AF9059080480068800714
:10206C0000280BD4FEF712F90599401A7C498842D6
:10207C0003D307A903200870DDE0EEE722E0FEF7AA
:10208C0005F9059075480068800700281AD5FEF7F9
:10209C00FDF80599401A7249884203D307A9032019
:1020AC000870C8E0EEE7C046081002400C10024071
:1020BC0000100240041002400024F400980000209C
:1020CC008800002002A80078012805D16149086821
:1020DC0001221207904308600698C069002800D1BD
:1020EC00A6E0574800683821084010286AD00698A6
:1020FC00C069022847D1544908680122120690434E
:10210C000860FEF7C3F805904F480068800100286E
:10211C000AD5FEF7BBF80599401A032803D307A983
:10212C000320087087E0EFE7464908684E4A1040E4
:10213C00069B1A6A5C6A22439C6A24022243DC6A6C
:10214C0022431B6B1A43104308603F4B1868012253
:10215C001406204318600868120710430860FEF745
:10216C0095F8059038480068800100280AD4FEF7DD
:10217C008DF80599401A032803D307A9032008708A
:10218C0059E0EFE71DE03049086801221206904340
:10219C000860FEF77BF805902B480068800100284A
:1021AC000AD5FEF773F80599401A032803D307A93B
:1021BC00032008703FE0EFE722490868294A1040E5
:1021CC00086035E00698C069012803D107A90120F1
:1021DC00087030E01B480068039003980321084006
:1021EC000699096A88421FD1039870210840069904
:1021FC00496A884218D103987F2109020840069940
:10220C00896A090288420FD103981F2149040840AA
:10221C000699C96A884207D10398072149070840E3
:10222C000699096B884203D007A90120087002E0C7
:10223C0007A90020087007A8007808B010BDC04698
:10224C00081002400C100240001002400410024022
:10225C00601002403C100240007000405C100240D4
:0C226C0089130000FCFFFEEF8C80C11FF6
:1022780000B585B0039002910398002803D104A902
:1022880001200870E9E002987649096807221140A0
:1022980088421CD97349086807229043029A104360
:1022A8000860FDF7F5FF01906E48006807210840B7
:1022B800029988420BD0FDF7EBFF0199401A71494A
:1022C800884203D304A903200870C6E0ECE703980A
:1022D80000788007002813D5039800784007002865
:1022E80005D56149086807221203104308605E4952
:1022F80008680F2212029043039A926810430860FC
:1023080003980078C007002860D003984068012827
:1023180009D1584800688003002803D404A9012083
:1023280008709AE032E003984068022809D15148C1
:1023380000688001002803D404A9012008708CE0FB
:1023480024E003984068002809D14A4800684005FD
:10235800002803D404A9012008707EE016E0039841
:102368004068032809D1424800688007002803D440
:1023780004A90120087070E008E03C480068800764
:10238800002803D404A90120087066E036490868CB
:1023980007229043039A526810430860FDF778FFBC
:1023A8000190314800683821084003994968C900FC
:1023B80088420BD0FDF76CFF0199401A31498842D9
:1023C80003D304A90320087047E0EAE702982549E7
:1023D80009680722114088421CD22249086807224E
:1023E8009043029A10430860FDF752FF01901D4880
:1023F800006807210840029988420BD0FDF748FF82
:102408000199401A1F49884203D304A90320087080
:1024180023E0ECE7039800784007002808D5124924
:102428000868072212039043039AD2681043086091
:1024380000F02AF80C4909680F22120211408A0993
:102448000D4989581F221140C8400C4908600C48A2
:102458000068FDF7D5FE04A9087004A8007805B047
:1024680000BDC04600200240081002405C10024037
:102478006010024000100240FCC7000898000020CD
:08248800880000208913000008
:1024900000B587B03A4800688006400F00280ED18A
:1024A0003B4800680721C9020840C10A0120884052
:1024B00002900299354809F0FBF801905CE0304841
:1024C000006838210840082802D12F48019053E0C5
:1024D0002B48006838210840102837D12948016866
:1024E0000322114005910068702108400009401C3A
:1024F000039005980090022810D0009803280DD171
:102500000399214809F0D4F801461E4800687F224B
:1025100012021040000A484306900CE003991B4841
:1025200009F0C6F80146174800687F2212021040E1
:10253000000A4843069013480068400F401C04906E
:102540000698049909F0B4F8019015E00C48006869
:1025500038210840202803D10120C00301900BE05E
:102560000748006838210840182803D17D20000260
:10257000019001E000200190019807B000BDC04625
:10258000081002400C10024000127A000024F400EF
:0425900000100240F5
:0C259400014800687047C0469800002015
:1025A00000B581B0FFF7F6FF009000F00DF801468E
:1025B0000098090B8A00034989581F221140C8401E
:0825C00001B000BD3CC8000899
:1025C80002480068072109030840704708100240C4
:1025D80000B587B0069003A90020087002A908700A
:1025E800069880788007002800D487E001A9002099
:1025F800087072480068C00000280CD46F48026850
:10260800012109070A430260006808400090009809
:1026180001A9012008706A490868012212021043C2
:102628000860FDF735FE049065480068C00500287D
:102638000AD4FDF72DFE0499401A032803D303A9F1
:102648000320087000E0EFE703A80078002848D1CD
:102658005C48006803210902084005900598002895
:1026680014D005980699896988420FD05549086899
:1026780003221202904305900868012212041043B5
:1026880008600868904308600598086005A8007805
:10269800C007002813D0FDF7FBFD049049480068E7
:1026A800800700280BD4FDF7F3FD0499401A46492A
:1026B800884203D303A90320087000E0EEE703A8CB
:1026C8000078002809D13F49086803221202904384
:1026D800069A92691043086002E0039802A90870FC
:1026E80002E0039802A9087001A80078012805D122
:1026F800324908680122120790430860069800785A
:10270800C007002807D03149086803229043069A79
:10271800526810430860069800788007002807D59B
:102728002A4908680C229043069A92681043086068
:10273800069800788006002808D5244908680322EE
:1027480012039043069AD2681043086006984078AE
:102758004006002814D51D490868032292079043B3
:10276800069A526910430860069840690121890752
:10277800884205D1164908680122120410430860EE
:10278800069840780007002814D5104908680322E5
:1027980092039043069A12691043086006980069EC
:1027A80001218903884205D10949086801221204D8
:1027B8001043086002A8007807B000BD3C10024032
:1027C800007000405C100240891300005410024061
:0427D8000C1002409F
:1027DC0000B583B0029001A901200870029800286E
:1027EC0065D002982921405C00280AD10299282240
:1027FC000020885402991120C0024860029807F00A
:10280C0079F8029929220220885402980168CA207A
:10281C0048620298016853204862029800F04EF812
:10282C00014601A801700078002834D10298016893
:10283C008869214A104088610298826841690A437C
:10284C00C1690A4301688869104388610299086963
:10285C00096808610298C1680A0401680869104394
:10286C000861029800F066F8014601A80170007832
:10287C00002810D1029801688869072252079043FA
:10288C0088610298426A016A0A4381690A430168B5
:10289C0088691043886102980168FF20486201A88A
:1028AC000078002803D1029929220120885401A81C
:0C28BC00007803B000BDC046BFFF8FFBDA
:1028C80000B585B0049002A900200870049800683B
:1028D800C0684006002828D404980168C868802287
:1028E8001043C860FDF7D4FC039004980068C168E1
:1028F800002049060029019005D402A80078C01ECE
:10290800411E884101900198C00700280DD0FDF7AD
:10291800BFFC0399401A0749884205D302A903203E
:102928000870049929228854DFE702A8007805B0C6
:0829380000BDC046E9030000E8
:1029400000B583B0029001A90020087017490868FB
:1029500080229043086016480068800600280BD447
:10296000029800F027F8002805D0029929220320B8
:10297000885401A9087014E00D490868202290438A
:102980000860029800F016F8002805D00299292264
:102990000320885401A908700549086820221043C3
:1029A000086001A8007803B000BDC0460C280040B4
:0429B00018280040A3
:1029B40000B583B0019001980168C868A0229043D3
:1029C400C860FDF767FC009001980068C068800645
:1029D40000280BD4FDF75EFC0099401A0749884291
:1029E40003D302A90320087003E0EDE702A9002045
:1029F400087002A8007803B000BDC046E9030000D7
:102A040000B589B007900691059207982821405C8B
:102A1400012803D108A90220087085E0079928221B
:102A240001208854079929220220885407980168B4
:102A3400CA20486207980168532048620798FFF744
:102A440041FF014603A801700078002859D1059878
:102A5400002825D10798006880694006002800D521
:102A640002E006990020C870069800780BF0CBF9B4
:102A740000040190069840780BF0C5F901460198CE
:102A8400090240180290069880780BF0BCF90146C0
:102A9400029840180699C97889050843049015E0FE
:102AA4000798006880694006002800D502E006996E
:102AB4000020C8700699087800044A781202801829
:102AC4008A788018C97889050843049004981849BD
:102AD4000840079909680860079801688869012215
:102AE4009204904388610698C2680069024307987B
:102AF40001688869104388610798FFF71FFF03A9DD
:102B0400087007980168FF20486203A8007800282D
:102B140003D10799292201208854079928220020EB
:102B24008854039808A9087008A8007809B000BD63
:042B34007F7F7F0020
:102B380000B589B007900691059207982821405C56
:102B4800012803D108A9022008706FE007992822FC
:102B580001208854079929220220885405980028C2
:102B68000AD106984078C006002805D50699487805
:102B7800EF2210400A304870059800281BD10698AB
:102B8800C0780BF03EF900040190069840780BF0ED
:102B980038F9014601980902401802900698807891
:102BA8000BF02FF901460298401806990978490355
:102BB800084304900BE00699C87800044A7812028A
:102BC80080188A7880180978490308430490079880
:102BD8000168CA204862079801685320486207982C
:102BE800FFF76EFE014603A80170007800280AD19D
:102BF8000498104908400799096848600798FFF742
:102C08009BFE03A9087007980168FF20486203A883
:102C18000078002803D107992922012088540799B0
:102C2800282200208854039808A9087008A800786A
:082C380009B000BD3FFFFF00E1
:102C400010B584B002900298002803D103A9012096
:102C5000087090E00298406A00280AD10298406803
:102C600041218900884200D102E002990020C86118
:102C700004E002990020086102994861029900204D
:102C8000886202985D21405C002806D102995C228E
:102C900000208854029806F0B3FF02995D220220BA
:102CA000885402980168086840229043086002989E
:102CB000C0683349884202D30020019002E001201D
:102CC000000301900298C0680F210902884208D0D1
:102CD0000298C06807210902884202D002990020A8
:102CE0008862029A009250684121890008409168E8
:102CF00021239B02194040181169022319404018F2
:102D0000536901210B40C01893694C022340C0183D
:102D1000D36938242340C018136A80242340C01884
:102D2000936A4C032340184312681060029A508B38
:102D300004231840536A10242340C018536B0824FE
:102D40002340C018D3680F2424022340C018019BDD
:102D50000C032340C0181268506002980268D069C2
:102D6000CB029843D061029A00201066029A5D233C
:102D7000D15403A9087003A8007804B010BDC04660
:042D80000107000047
:102D840010B58CB00E9C0A9009910892079302A981
:102D94000020087007980190FDF77CFA024601981C
:102DA4000E99891A40180590FDF774FA04900A9850
:102DB40000680C30039005993A4802682320504378
:102DC400000D484306900A980068806809990840F5
:102DD400089988425FD0099803214902884207D1A3
:102DE4000898002804D10398007802A90870029872
:102DF4000798401C00284DD0FDF74CFA0499401A5E
:102E04000599884202D2059800283BD10A980168A6
:102E14004868E022904348600A984068412189004C
:102E2400884211D10A9880680121C903884205D0DB
:102E34000A98806801218902884205D10A980168AC
:102E440008684022904308600A98806A0121490377
:102E540088420BD10A980168086801225203904302
:102E640008600A9801680868104308600A995D229E
:102E7400012088540A995C22002088540BA903205D
:102E840008700BE00698002801D1002005900698F0
:102E9400401E069097E70BA9002008700BA8007845
:082EA4000CB010BD98000020E5
:102EAC0010B58AB00C9C0890079106A80270059387
:102EBC0005980190FDF7EAF9024601980C99891AD8
:102ECC0040180390FDF7E2F9029003993548006829
:102EDC004001000D484304900898006880680799E9
:102EEC000840401A4142484106A90978884252D00C
:102EFC000598401C00284DD0FDF7C8F90299401ADE
:102F0C000399884202D2039800283BD108980168A3
:102F1C004868E02290434860089840684121890045
:102F2C00884211D1089880680121C903884205D0D4
:102F3C000898806801218902884205D108980168A7
:102F4C0008684022904308600898806A0121490370
:102F5C0088420BD1089801680868012252039043FB
:102F6C0008600898016808681043086008995D2299
:102F7C000120885408995C220020885409A9032058
:102F8C0008700BE00498002801D1002003900498ED
:102F9C00401E0490A0E709A90020087009A8007839
:082FAC000AB010BD98000020DE
:102FB40010B58EB0109C0C900B910A9209A8038056
:102FC4000120049003A9002008700C985C21405C47
:102FD400012803D10DA90220087083E10C995C2219
:102FE40001208854FDF756F905900C985D21415C49
:102FF40006A801700C9949680791099908AA1180DB
:103004000078012810D0079841218900884207D10F
:103014000C988068002803D106A80078042803D0FF
:1030240003A90220087056E10B98002806D00A98DC
:10303400002803D009A80088002803D103A901208F
:10304400087048E10C985D21405C042803D00C9979
:103054005D22052088540C99002008660A990C9A70
:10306400116409990C9A4623D15209990C9A442364
:10307400D1520B990C9A916309990C9AD1870999A9
:103084000C9A91870C99C8640C9908650C98C068CF
:103094009649884207D30C980168486801221203B4
:1030A4009043486006E00C980168486801221203C6
:1030B400104348600C98006800684021084040288C
:1030C40005D00C98016808684022104308600C98E9
:1030D400C0688649884271D30C984068002803D0A0
:1030E40008A8008801280CD10C99886B008809680D
:1030F400C8600C99886B801C88630C99C88F401E2B
:10310400C8870C98C18F01200029029005D10C9822
:103114004621405A411E884102900298C007002867
:103124004BD00C98006880688007002815D50C984F
:10313400C08F002811D0049801280ED10C99886BF7
:1031440000880968C8600C99886B801C88630C9996
:10315400C88F401EC887002004900C9800688068BF
:10316400C007002815D00C984621405A002810D0DA
:103174000C980068C0680C99096C08800C99086C5C
:10318400801C08640C994622885A401E88520120EB
:103194000490FDF77FF80599401A109988420BD3E3
:1031A4001098401C002807D003A9032008700C992C
:1031B4005D22012088548EE0A3E773E00C984068F8
:1031C400002803D008A8008801280CD10C99886B2A
:1031D4000078096808730C99886B401C88630C9903
:1031E400C88F401EC8870C98C18F01200029019008
:1031F40005D10C984621405A411E884101900198FE
:10320400C00700284ED00C9800688068800700280A
:1032140015D50C98C08F002811D0049801280ED120
:103224000C99886B0078096808730C99886B401CAA
:1032340088630C99C88F401EC887002004900C989E
:1032440000688068C007002815D00C984621405AB1
:10325400002810D00C980068007B0C99096C087049
:103264000C99086C401C08640C994622885A401E2C
:10327400885201200490FDF70DF80599401A109921
:10328400884203D31098401C002802D110980028CB
:1032940007D103A9032008700C995D2201208854EA
:1032A40019E0A0E70C981099059A09F0D6FD0028BA
:1032B40005D003A9012008700C99202008660C98F9
:1032C400006E002803D003A90120087003E00C99C4
:1032D4005D22012088540C995C22002088540398B4
:1032E4000DA908700DA800780EB010BD01070000EC
:1032F40083B00290019102980068009002983349CB
:10330400884203D002983249884208D1009870213B
:1033140088430090019841680098084300900298FF
:103324002A49884213D00298294988420FD002982A
:10333400284988420BD002982749884207D002982E
:103344002649884203D002982549884209D1009829
:1033540003210902884300900198C168009808433A
:10336400009000988021884301994969084300909E
:10337400009802990860019880680299C8620198CF
:103384000068029988620298104988420BD002981A
:103394001149884207D002981049884203D0029804
:1033A4000F49884203D10198006902990863029980
:1033B4000120486102980069C007002804D00299DE
:1033C400086901229043086103B07047002C014052
:1033D400000400400020004000400140004401403F
:0433E400004801405C
:1033E80000B581B0009000993D22022088540098D1
:1033F8000068006A204908420BD100980068006AFA
:103408001E49084205D100980168086801229043C6
:10341800086000980AF01DFD009948220020885491
:1034280000993E220020885400993F228854009930
:103438004022885400994122885400994222885495
:103448000099432288540099442200208854009906
:103458004522885400994622885400994722885466
:1034680000993D220020885400993C22002088546D
:10347800002001B000BDC046111100004404000046
:1034880000B597B01590149113A9002008701498EE
:10349800002804D115983E21405C0F902BE0149829
:1034A800042804D115983F21405C0E9021E014981F
:1034B800082804D115984021405C0D9017E0149815
:1034C8000C2804D115984121405C0C900DE014980B
:1034D800102804D115984221405C0B9003E0159800
:1034E8004321405C0B900B980C900C980D900D9814
:1034F8000E900E980F900F9811A908701498002834
:1035080004D115984421405C0A9017E014980428C7
:1035180004D115984521405C09900DE014980828BD
:1035280004D115984621405C089003E0159847217E
:10353800405C08900898099009980A900A9810A980
:10354800087011A80078012803D110A80078012874
:1035580003D016A901200870D2E01498002804D1DD
:1035680015993E22022088542FE01498042805D18A
:1035780015993F2202208854079025E014980828BE
:1035880005D1159940220220885406901AE0149813
:103598000C2805D1159941220220885405900FE086
:1035A8001498102805D115994222022088540490B5
:1035B80004E0159943220220885404900498059049
:1035C800059806900698079007981498002804D143
:1035D800159944220220885419E01498042805D12A
:1035E800159945220220885403900FE01498082862
:1035F80005D11599462202208854029004E01599B5
:103608004722022088540290029803900398149845
:1036180001900C283AD80198810001A040588746AB
:103628005D3600089536000895360008953600087E
:103638006B36000895360008953600089536000860
:103648007936000895360008953600089536000842
:103658008736000815980168C86802221043C860B8
:1036680017E015980168C86804221043C86010E084
:1036780015980168C86808221043C86009E01598C1
:103688000168C86810221043C86002E013A901202D
:10369800087013A8007800282FD11598006814998D
:1036A800012209F01FFC159800681749884209D0C3
:1036B800159800681549884204D01598006814497F
:1036C800884214D115980068806812490840129001
:1036D800129806280AD0129801210904884205D0B8
:1036E80015980168086801221043086005E01598DC
:1036F80001680868012210430860139816A9087029
:1037080016A8007817B000BD002C01400004004046
:08371800004001400700010020
:1037200000B58BB00A90099108A90020087009988B
:1037300007900C283AD80798810001A04058874686
:1037400075370008AD370008AD370008AD37000801
:1037500083370008AD370008AD370008AD370008E3
:1037600091370008AD370008AD370008AD370008C5
:103770009F3700080A980168C86802229043C86011
:1037800017E00A980168C86804229043C86010E0F6
:103790000A980168C86808229043C86009E00A983E
:1037A0000168C86810229043C86002E008A901209F
:1037B000087008A80078002871D10A980068099953
:1037C000002209F093FB0A980068006A3649084213
:1037D0000BD10A980068006A3449084205D10A985A
:1037E000016808680122904308600998002804D104
:1037F0000A993E22012088542FE00998042805D117
:103800000A993F2201208854069025E0099808284B
:1038100005D10A9940220120885405901AE00998A0
:103820000C2805D10A9941220120885404900FE008
:103830000998102805D10A99422201208854039042
:1038400004E00A99432201208854039003980490CD
:10385000049805900598069006980998002804D1C8
:103860000A9944220120885419E00998042805D1B6
:103870000A9945220120885402900FE009980828EF
:1038800005D10A99462201208854019004E00A9942
:10389000472201208854019001980290029808A8BC
:1038A00000780BB000BDC0461111000044040000B8
:1038B00000B583B0029002980068C0680190029839
:1038C00000680069009068460078800700281FD5CE
:1038D00001A80078800700281AD502980168022004
:1038E000C043086102990120087702980068806946
:1038F0008007002803D0029801F002FB05E002983F
:103900000AF0AFFA02980AF0A0FA029900200877AC
:10391000684600784007002820D501A800784007B5
:1039200000281BD5029801680420C0430861029951
:10393000022008770298006880698005800F0028BF
:1039400003D0029801F0DCFA05E002980AF089FA47
:1039500002980AF07AFA02990020087768460078FF
:10396000000700281FD501A80078000700281AD5F5
:10397000029801680820C043086102990420087772
:1039800002980068C0698007002803D0029801F0FF
:10399000B7FA05E002980AF064FA02980AF055FABC
:1039A00002990020087768460078C006002820D5D4
:1039B00001A80078C00600281BD5029801681020D5
:1039C000C043086102990820087702980068C0691E
:1039D0008005800F002803D0029801F091FA05E0DD
:1039E00002980AF03EFA02980AF02FFA0299002093
:1039F000087768460078C00700280CD001A8007836
:103A0000C007002807D0029801680120C043086160
:103A100002980AF016FA009880210840802804D005
:103A200068464078800600280BD501A8007800067B
:103A3000002806D5029801681D48086102980AF01E
:103A4000A2FA68464078C00700280BD001A8007889
:103A50000006002806D502980168164808610298F9
:103A60000AF095FA68460078400600280CD501A8AF
:103A700000784006002807D5029801684020C0431E
:103A8000086102980AF0F1F968460078800600287B
:103A90000CD501A800788006002807D50298016897
:103AA0002020C043086102980AF019FA03B000BD53
:083AB0007FDFFFFFFFFEFFFFB7
:103AB80087B006900591049203930698006A0190D6
:103AC800069A116A01208143116206998969029157
:103AD80006991E4A914200900BD0069901201C4A73
:103AE8009142009005D006981A4940184142484131
:103AF80000900098C007002808D002980321884346
:103B08000290049902980843029003E00298012168
:103B1800084302900298F02188430290039800011C
:103B2800C1B202980843029001990A208143019189
:103B38000599014001980843019002980699886107
:103B480001980699086207B07047C046002C0140EA
:083B58000004004000C0FEBFA4
:103B600000B5F7B076900020729071A9087070903F
:103B7000769988680A6910434A691043C9690843FD
:103B800075907698416E75980843759076980068A0
:103B900000686A4908407599084376990968086081
:103BA0007698006840680321090388437699CA68BB
:103BB0001043096848607698806975907698016A24
:103BC0007598084375907698006880685C4908404D
:103BD0007599084376990968886076980068C06A84
:103BE0000F21884376994A6A10430968C86276981B
:103BF00000685449884227D153480068032108408F
:103C00006F9003281CD86F98810001A04058874608
:103C1000213C0008313C0008293C0008393C0008E0
:103C200073A9002008700EE073A9022008700AE052
:103C300073A90420087006E073A90820087002E048
:103C400073A91020087054E0769800683F498842B4
:103C50003AD13D4800680C2108406E900C282FD8BE
:103C60006E98810001A040588746C046A13C0008DC
:103C7000C13C0008C13C0008C13C0008B13C000840
:103C8000C13C0008C13C0008C13C0008A93C000838
:103C9000C13C0008C13C0008C13C0008B93C000818
:103CA00073A9002008700EE073A9022008700AE0D2
:103CB00073A90420087006E073A90820087002E0C8
:103CC00073A91020087014E0769800682049884293
:103CD00003D173A9002008700BE0769800681D4995
:103CE000884203D173A90020087002E073A9102054
:103CF00008707698C0690121C903884200D03DE26E
:103D000073A800786D90082800D918E26D9881009A
:103D100001A040588746C046593D00083F41000871
:103D2000553E00083F4100084B3F00083F41000856
:103D30003F4100083F41000847400008F369FFCFBA
:103D4000FFF4FF11003801405410024000440040CD
:103D500000480040004C0040FEF722FC6C90769832
:103D6000406A002802D101206B9065E07698406A95
:103D7000012802D102206A905CE07698406A02280D
:103D800002D10420699053E07698406A032802D15A
:103D9000062068904AE07698406A042802D10820FC
:103DA000679041E07698406A052802D10A20669023
:103DB00038E07698406A062802D10C2065902FE002
:103DC0007698406A072802D11020649026E0769801
:103DD000406A082802D1202063901DE07698406A4E
:103DE000092802D14020629014E07698406A0A289F
:103DF00002D1802061900BE07698416A01205F90AB
:103E000000020B29609001D05F98609060986190EB
:103E100061986290629863906398649064986590EA
:103E200065986690669867906798689068986990BA
:103E300069986A906A986B906C986B9907F038FC57
:103E40004000769949684A08801807F031FC80B232
:103E5000729077E17698406A002802D101205E9046
:103E600065E07698406A012802D102205D905CE00E
:103E70007698406A022802D104205C9053E076983C
:103E8000406A032802D106205B904AE07698406A97
:103E9000042802D108205A9041E07698406A05280B
:103EA00002D10A20599038E07698406A062802D15B
:103EB0000C2058902FE07698406A072802D11020F5
:103EC000579026E07698406A082802D12020569024
:103ED0001DE07698406A092802D14020559014E0F0
:103EE0007698406A0A2802D1802054900BE0769898
:103EF000416A0120529000020B29539001D0529840
:103F0000539053985490549855905598569056986D
:103F10005790579858905898599059985A905A983D
:103F20005B905B985C905C985D905D985E905E990C
:103F3000A14807F0BDFB4000769949684A088018FF
:103F400007F0B6FB80B27290FCE0FEF7A1FA519048
:103F50007698406A002802D10120509065E076985A
:103F6000406A012802D102204F905CE07698406AB6
:103F7000022802D104204E9053E07698406A03282C
:103F800002D106204D904AE07698406A042802D17A
:103F900008204C9041E07698406A052802D10A201A
:103FA0004B9038E07698406A062802D10C204A905F
:103FB0002FE07698406A072802D11020499026E029
:103FC0007698406A082802D1202048901DE0769813
:103FD000406A092802D14020479014E07698406A50
:103FE0000A2802D1802046900BE07698416A012091
:103FF000449000020B29459001D044984590459883
:1040000046904698479047984890489849904998D4
:104010004A904A984B904B984C904C984D904D98A4
:104020004E904E984F904F9850905198509907F05D
:104030003FFB4000769949684A08801807F038FB32
:1040400080B272907EE07698406A002802D101200A
:10405000439065E07698406A012802D102204290A0
:104060005CE07698406A022802D10420419053E037
:104070007698406A032802D1062040904AE076985C
:10408000406A042802D108203F9041E07698406AB7
:10409000052802D10A203E9038E07698406A06282A
:1040A00002D10C203D902FE07698406A072802D17B
:1040B00010203C9026E07698406A082802D1202003
:1040C0003B901DE07698406A092802D140203A9042
:1040D00014E07698406A0A2802D1802039900BE0DB
:1040E0007698416A0120379000020B29389001D060
:1040F000379838903898399039983A903A983B9058
:104100003B983C903C983D903D983E903E983F9027
:104110003F984090409841904198429042984390F7
:1041200043990120C00307F0C3FA4000769949681B
:104130004A08801807F0BCFA80B2729002E071A9B8
:10414000012008707298102814D372A840880028A3
:1041500010D172990F20814374A8018072990E22A8
:1041600011404A08749911430180008876990968C2
:10417000C86002E071A90120087020E273A80078ED
:104180003690082800D908E23698810001A04058EE
:104190008746C046BD4100089B450008B74200085D
:1041A0009B450008AB4300089B4500089B45000861
:1041B0009B450008A54400080024F400FEF7F0F930
:1041C00035907698406A002802D10120349065E04D
:1041D0007698406A012802D1022033905CE07698FC
:1041E000406A022802D10420329053E07698406A57
:1041F000032802D1062031904AE07698406A0428CC
:1042000002D10820309041E07698406A052802D11A
:104210000A202F9038E07698406A062802D10C20B8
:104220002E902FE07698406A072802D110202D901A
:1042300026E07698406A082802D120202C901DE0C4
:104240007698406A092802D140202B9014E0769895
:10425000406A0A2802D180202A900BE07698416AB1
:104260000120289000020B29299001D0289829903C
:1042700029982A902A982B902B982C902C982D9046
:104280002D982E902E982F902F9830903098319016
:1042900031983290329833903398349035983499DD
:1042A00007F006FA769949684A08801807F000FA7C
:1042B00080B2729074E17698406A002802D10120A1
:1042C000279065E07698406A012802D10220269066
:1042D0005CE07698406A022802D10420259053E0E1
:1042E0007698406A032802D1062024904AE0769806
:1042F000406A042802D10820239041E07698406A61
:10430000052802D10A20229038E07698406A0628D3
:1043100002D10C2021902FE07698406A072802D124
:104320001020209026E07698406A082802D12020AC
:104330001F901DE07698406A092802D140201E9007
:1043400014E07698406A0A2802D180201D900BE084
:104350007698416A01201B9000020B291C9001D025
:104360001B981C901C981D901D981E901E981F90C5
:104370001F98209020982190219822902298239095
:104380002398249024982590259826902698279065
:104390002799934807F08CF9769949684A0880185C
:1043A00007F086F980B27290FAE0FEF771F81A9081
:1043B0007698406A002802D10120199065E076982D
:1043C000406A012802D1022018905CE07698406A89
:1043D000022802D10420179053E07698406A0328FF
:1043E00002D1062016904AE07698406A042802D14D
:1043F0000820159041E07698406A052802D10A20ED
:10440000149038E07698406A062802D10C20139068
:104410002FE07698406A072802D11020129026E0FB
:104420007698406A082802D1202011901DE07698E5
:10443000406A092802D14020109014E07698406A22
:104440000A2802D180200F900BE07698416A012063
:104450000D9000020B290E9001D00D980E900E9831
:104460000F900F9810901098119011981290129828
:1044700013901398149014981590159816901698F8
:10448000179017981890189819901A98199907F07A
:104490000FF9769949684A08801807F009F980B23F
:1044A00072907DE07698406A002802D101200C903D
:1044B00065E07698406A012802D102200B905CE00A
:1044C0007698406A022802D104200A9053E0769838
:1044D000406A032802D1062009904AE07698406A93
:1044E000042802D10820089041E07698406A052807
:1044F00002D10A20079038E07698406A062802D157
:104500000C2006902FE07698406A072802D11020F0
:10451000059026E07698406A082802D12020049071
:104520001DE07698406A092802D14020039014E0EB
:104530007698406A0A2802D1802002900BE0769893
:10454000416A0120009000020B29019001D00098DF
:1045500001900198029002980390039804900498A7
:104560000590059806900698079007980890089877
:10457000099009980A900A980B900B980C900C9946
:104580000120C00307F094F8769949684A0880181A
:1045900007F08EF880B2729002E071A901200870D5
:1045A0007298102808D372A84088002804D1729805
:1045B00076990968C86002E071A9012008707699AF
:1045C0006A220120885276996822885276990020C2
:1045D000C8667699086771A8007877B000BDC046B4
:0445E0000024F400BF
:1045E40000B585B003900399882200208850FBF71A
:1045F40051FE0290039800680068000700280ED559
:104604000398029B1949009101214905002209F0F0
:10461400C0FC002803D004A90320087022E00398FA
:1046240000680068400700280ED50398029B0F49D4
:10463400009101218905002209F0ABFC002803D078
:1046440004A9032008700DE00399802220208850DB
:1046540003998422885003997C220020885404A959
:104664000020087004A8007805B000BDFFFFFF011A
:1046740084B00290019168460280029880214058DB
:10468400202800D081E00198002803D068460088E3
:10469400002803D103A90120087079E002988068FA
:1046A4000121090388420CD102980069002808D12D
:1046B40001A80078C007002803D003A901200870CE
:1046C40066E002987C21405C012803D103A9022002
:1046D40008705DE002997C220120885401980299B7
:1046E400086500980299542288520098029956222B
:1046F40088520299002008670299882288500299FA
:104704008022212088500298406E01214907884266
:104714001CD10298806801210903884207D10298BC
:104724000069002803D102991E48086702E0029933
:104734001B48086702997C2200208854029801686B
:1047440088680122D205104388601AE002988068C4
:1047540001210903884207D102980069002803D186
:1047640002990E48086702E002990B48086702990B
:104774007C22002088540298016808688022104333
:10478400086003A90020087002E003A90220087051
:1047940003A8007804B0704763D3000839480008C0
:0847A400E5D20008AD47000852
:1047AC0083B0029002988021405821283AD1029877
:1047BC006A21405A6946088068460088002831D032
:1047CC0002985621405A00280DD102980168886839
:1047DC000122D20590438860029801680868402243
:1047EC00104308601EE002980068C06900060028AB
:1047FC0013D50298006D0190019800880A49084071
:10480C000299096888620299086D801C08650299F2
:10481C005622885A401E8852FFE70098401E69466F
:0C482C000880C9E703B07047FF010000DE
:1048380082B00190019880214058212824D1019804
:104848005621405A00280CD1019801680868802236
:104858009043086001980168086840221043086086
:1048680012E00198006D0090009800880749084000
:104878000199096888620199086D801C0865019989
:104888005622885A401E885202B07047FF01000025
:1048980084B00290019168460280029884214058B1
:1048A800202800D0D3E00198002803D0684600886B
:1048B800002803D103A901200870CBE00298806882
:1048C8000121090388420CD102980069002808D107
:1048D80001A80078C007002803D003A901200870A8
:1048E800B8E002987C21405C012803D103A902208A
:1048F8000870AFE002997C2201208854019802993F
:104908008865009802995C228852009802995E2274
:10491800885202990020C86602988068012109031C
:1049280088420DD102980069002804D102996022BA
:104938004A48885203E002996022FF20885229E001
:104948000298806800280DD102980069002804D1D7
:1049580002996022FF20885203E0029960227F209A
:10496800885217E0029880680121090788420DD112
:1049780002980069002804D1029960227F20885299
:1049880003E0029960223F20885203E002996022E6
:104998000020885202998822002088500299842297
:1049A800222088500298026890680121084390608C
:1049B8000298406E4907884229D1684600880299C2
:1049C8006822895A884222DB0298806801210903FB
:1049D800884207D102980069002803D10299234828
:1049E800C86602E002992048C86602997C22002025
:1049F8008854029801680868012213021843086065
:104A08000298016888681207104388601BE00298C2
:104A1800806801210903884207D1029800690028AB
:104A280003D102990F48C86602E002990C48C8668B
:104A380002997C220020885402980168086809229B
:104A480052011043086003A90020087002E003A97E
:104A58000220087003A8007804B07047FF01000026
:104A680043D40008B5D30008694B0008794A000808
:104A780000B587B0069006986021405A04A90880BE
:104A880006988421405822285ED106986821405A09
:104A980002A9088002A80088002835D00698006876
:104AA800406A03A908800698806D059003980499C8
:104AB8000840059908800699886D801C8865069AC3
:104AC8005E21505A401E50520698405A002816D16E
:104AD8000698016808680122120290430860069847
:104AE800016888681D4A1040886006998422202041
:104AF800885006990020C866069809F08EFA029830
:104B0800401E02A90880C5E706985E21415A01A8FF
:104B180001800088002816D001A80088069968221C
:104B2800895A88420FDA06980168886801221207B4
:104B38009043886006990848C8660698016808681E
:104B480020221043086005E0069801688869082259
:104B58001043886107B000BDB5D30008FEFFFFEF22
:104B680000B585B0049004986021405A03A90880D4
:104B780004988421405822285CD104986821405A1E
:104B880001A9088001A80088002833D0049800688B
:104B9800406A02A908800298039908400499896D1F
:104BA80008700499886D401C8865049A5E21505AE3
:104BB800401E50520498405A002816D104980168A3
:104BC8000868012212029043086004980168886806
:104BD8001D4A104088600499842220208850049936
:104BE8000020C866049809F018FA0198401E01A927
:104BF8000880C7E704985E21415A6846018000880A
:104C0800002816D06846008804996822895A884284
:104C18000FDA0498016888680122120790438860B7
:104C280004990848C8660498016808682022104357
:104C3800086005E0049801688869082210438861C3
:0C4C480005B000BD43D40008FEFFFFEFE4
:104C540000B585B000200190049004987F282DD8D9
:104C6400049881002348405800900020029003904B
:104C740003987F280DD8009803998A001D49895804
:104C8400884202DD0298401C02900398401C039065
:104C9400EEE70499029A164881540299405C002870
:104CA40008D10198012803D1134806F0CBFDFEE793
:104CB400012001900498401C0490CEE70B49402049
:104CC40008700020049004987F280DD807480078C5
:104CD400049A0749895C884202D104980349087000
:104CE4000498401C0490EEE705B000BD9D00002030
:0C4CF400421400206C08002076E3000849
:104D000080B500F06FF802490420086080BDC046FD
:044D1000241000204B
:104D140000B585B02D48006804280CD12B4901202A
:104D240008602B480021FEF7ADFB152007F07CFF3F
:104D34000220049046E025480068032802D002209F
:104D440004903FE021480068032839D1152007F07A
:104D540076FF1F480021FEF7E1FC1C49042008608F
:104D64001C480068002806D01B48006802031B4941
:104D740008688018086017480068092806D815498B
:104D84000868401C0860022004901BE00020029088
:104D94000390104908600E480068806A401C009027
:104DA4000E48019000680A2106F080FC009B0199DE
:104DB400024602985A43039208600398049001E063
:104DC40000200490049805B000BDC04624100020C3
:104DD400C40E0020C00F002028100020D40F002093
:104DE40000B587B01E480268012149040A430260E5
:104DF40000680840029002981A4801901A4901601C
:104E0400FEF7F0FA01981949C1600021416001617F
:104E1400816008F082F8002800D0FEE700220392A7
:104E2400012004900C20059006920E4803A908F076
:104E3400C1F8002800D0FEE70A480221002209F048
:104E440050F8002800D0FEE71520009000221146FB
:104E540008F031FF009807F0F2FE07B000BDC0462D
:104E640040100240C40E002000440140FFFF000037
:104E740000B587B0002000900490FFF73FFF009832
:104E8400802102911B4909687F2212021140090AFC
:104E94000391049004980299884220D21549086825
:104EA4007F2212029043049A1202104308600220E7
:104EB40006900698022803D1FFF72AFF0690F8E728
:104EC40000200590069905984018059005980499C6
:104ED4008A00094988500498401C0490DAE705497F
:104EE40008687F2212029043039A1202104308605A
:0C4EF40007B000BD041002406C08002054
:104F000000B583B002900298007F012863D1334836
:104F10000068012809D10298002107F0B9FD324943
:104F200008602E490220086055E02C4800680228DD
:104F300051D102980021009107F0AAFD2849019162
:104F40000860152007F07DFE00992648FEF7E8FB73
:104F5000019802990A680221C94311610068224937
:104F60000968884215D91E4800681F490968411A16
:104F70001F480160006800031E49884208D81E4887
:104F800006F062FC1A48006801031C4806F05CFC4D
:104F90001EE01348006814490968884217D2124875
:104FA00001680F480068401A104941181048016014
:104FB000006800030F49884208D80F4806F044FCF7
:104FC0000B48006801030D4806F03EFC00E0FEE7D8
:104FD00002490320086003B000BDC0462410002031
:104FE0000C100020C40E002010100020FFFF000055
:104FF000281000203F5DC60009E800081AE80008F4
:1050000010B588B00B9C0A9C0790069105920493FA
:10501000069807990860079801684548086007984E
:1050200001684B20000248600798026801210803CC
:105030009060079802680020D060079A1268890281
:10504000116107990A680C21516107990968886103
:1050500007990968C861079909680862079909688A
:105060004862079909688862059807990968486045
:105070000498002809D10798026801208102116173
:10508000079909680003886014E0049801280AD190
:105090000798016803204002086107980168012011
:1050A0000003886006E007980168002008610799FE
:1050B000096888600A98012804D1079801680020CF
:1050C000C86004E00798016801204003C8600798A1
:1050D000006803900B9806F061FA00220292154BCB
:1050E00008F055FB06F0D2F9029B014603980091A7
:1050F00019461A4600F022F8002801D008F026FBD5
:105100000798006808F095FF002801D008F01EFB02
:1051100007990868273101221202FFF7BDFB00281A
:1051200003D0054806F090FBFEE708B010BDC0466E
:0C5130000038014000000C4079E5000848
:10513C0010B588B00A9C06900591049203930698CA
:10514C00002803D107A90120087063E0069880218C
:10515C004058002806D106997C22002088540698D5
:10516C0004F0EEFE069980222420885006980168EF
:10517C0008680122904308600698FEF7EBFC0128B2
:10518C0003D107A90120087044E00698806A002822
:10519C0002D0069808F005F80698016848680122C4
:1051AC00D3051843486006980168086892061043B6
:1051BC000860069840684B21090288420BD8069873
:1051CC0000684069FF21090608400A9908430699BE
:1051DC000968486113E00698416810484843104933
:1051EC0006F060FA401C0190069800684069FF21A7
:1051FC000906084001990843069909684861069810
:10520C00016808680122104308600698FFF7E4F96A
:10521C0007A9087007A8007808B010BDD6060000D2
:04522C0040420F00ED
:1052300010B58AB0099009980068C069089009986B
:10524000006800680790099800684068069009980F
:1052500000688068059008980F2108400490049821
:1052600000285BD005988F49084205D107A800881F
:1052700009214901084251D008A80078C007002838
:105280000DD007A84078C007002808D0099800680A
:10529000012303620999882288581843885008A876
:1052A0000078800700280ED505A80078C0070028E0
:1052B00009D0099801680220086209998822885853
:1052C00004231843885008A80078400700280ED50A
:1052D00005A80078C007002809D0099801680420B3
:1052E000086209998822885802231843885008A820
:1052F00000780007002811D507A80078800600284C
:1053000003D405986749084208D009980068082323
:1053100003620999882288581843885008A8407861
:105320000007002819D507A8C0784007002804D432
:1053300005A88078000600280FD50998026801208A
:10534000C1021162099A84232021D150099A802335
:10535000D15055490875554A885408A800788006E8
:1053600000282BD507A800788006002804D405A8BB
:10537000C078C006002821D50998842140582228E9
:1053800016D149484521C9004058FF2810D809982E
:105390000068406A44494522D2008B58CB18272424
:1053A00018558858401C8850404A0120885405E010
:1053B00009980168886908221043886108A8007864
:1053C0000006002813D507A800780006002804D49A
:1053D00005A880780006002809D5334802900068A7
:1053E00008F05DFE0299232002010120885408A8DC
:1053F0000078400600280FD507A80078400600284E
:105400000AD52949262200208854099808F09BF8DB
:105410000999842222208850099888214058002820
:105420003DD0099984222220885008A8007880065F
:10543000002814D507A800788006002804D405A801
:10544000C078C00600280AD5099801688869082232
:105450001043886109998822002088501FE008A81D
:105460000078000600281AD507A800780006002852
:1054700004D405A880780006002810D50A490191B7
:10548000262200208854099808F05DF80199099AAD
:1054900084232220D05023200201012088540AB006
:1054A00010BDC04601000010380600203102000087
:1054B00085B00490039102A918480880002001904B
:1054C00001980399884225D204980199415C029879
:1054D000484002A90880082000900098002815D0B4
:1054E00002A80088C007002808D002A90888400840
:1054F000088002980A4A5040088003E002A9088800
:10550000400808800098401E0090E6E70198401C83
:105510000190D5E702A8008805B07047FFFF0000A2
:0455200001A00000E6
:1055240000B585B003900398273001900398452176
:10553400C90040580290019800780090029804280D
:1055440005D8039808F02EF8002004901FE0019875
:10555400029908F0D8FD401C002805D1039808F0F2
:1055640021F80020049012E00098002802D10220C3
:1055740004900CE000980749098B884202D102206C
:10558400049004E0039808F00DF8002004900498B7
:0855940005B000BDA0000020DD
:10559C0010B588B006900591049203A803700078AA
:1055AC003649098B88420BD003A80078002807D015
:1055BC000698049B06210B2208F02CF8079059E062
:1055CC00059988780002C9784018029005990879E5
:1055DC0000024979401800900098002802D00098E9
:1055EC007E2807D30698049B0322114608F012F874
:1055FC0007903FE0029800994018401E80087728D9
:10560C0007D30698049B0321022208F003F80790A5
:10561C0030E00699049A032088540498401C0490A6
:10562C00009840000699049A88540498401C0490F1
:10563C000298019001980299009A8918884217D211
:10564C00019841000D4841184978069A049BD154A1
:10565C000499491C049101994900405C0699049AEB
:10566C0088540498401C04900198401C0190E1E778
:10567C0004980790079808B010BDC046A000002001
:10568C0000B587B0059004910392029302982C49BF
:10569C00098B88420AD00298002807D00598039BF2
:1056AC0006210B2207F0B6FF069045E00499887896
:1056BC000002C9784018019001988008772807D318
:1056CC000598039B0621022207F0A4FF069033E005
:1056DC000498007901994A0019498A185070049865
:1056EC004079019A520088540599039A06208854EF
:1056FC000398401C03900198000A0599039A88545A
:10570C000398401C039001980599039A88540398B8
:10571C00401C0390049800790599039A88540398C7
:10572C00401C0390049840790599039A8854039877
:10573C00401C039003980690069807B000BDC04625
:04574C00A000002099
:1057500000B589B0079006910592049304984149D9
:10576000098B88420AD00498002807D00798059B27
:1057700006210B2207F054FF08906FE00699887805
:105780000002C97840180390069908790002497907
:1057900040180290072000900298002802D002983A
:1057A0007C2807D30798059B1021032207F038FFB8
:1057B000089053E0039802994018401E800877280B
:1057C00007D30798059B1021022207F029FF0890B4
:1057D00044E00398019001980399029A891888423D
:1057E00015D206980099405C01994A001D498A1813
:1057F0005070069A009880184078019A5200885498
:105800000098801C00900198401C0190E3E70799E4
:10581000059A102088540598401C05900398000AAA
:105820000799059A88540598401C05900398079994
:10583000059A88540598401C05900298000A07991B
:10584000059A88540598401C059002980799059A76
:1058500088540598401C059005980890089809B050
:0858600000BDC046A0000020BD
:1058680010B586B000210191059104910391434838
:105878000290434A02600122D4074460031D8160FC
:10588800C160046108244461017641768276C26170
:105898001977416281622C23C25401630723436351
:1058A80083633C23C2541022026420224264816430
:1058B800C164FAF711FD002801D007F043FF012069
:1058C80003900490002005902C4803A9FAF7BAFF2A
:1058D800002801D007F036FF2A480390274803A97B
:1058E800FAF7B0FF002801D007F02CFF26480390F4
:1058F800224803A9FAF7A6FF002801D007F022FFE3
:10590800224803901D4803A9FAF79CFF002801D0FC
:1059180007F018FF1E480390184803A9FAF792FFEA
:10592800002801D007F00EFF1A480390134803A976
:10593800FAF788FF002801D007F004FF1648039003
:105948000E4803A9FAF77EFF002801D007F0FAFEF7
:1059580012480390094803A9FAF774FF002801D0F8
:1059680007F0F0FE0E480390044803A9FAF76AFF0F
:10597800002801D007F0E6FE06B010BD040E002096
:105988000024014002000004040000080800000C84
:1059980010000010001000B00001002000020024D8
:0459A80000040028CF
:1059AC0030B593B012900020119010900F900E9083
:1059BC000D90129800684F49884200D098E04E48EC
:1059CC000268012109050A430260006808400C9036
:1059DC000C984A48026801210A430260006808409A
:1059EC000B900B984548026802210A43026000683C
:1059FC0008400A900A98012007900D90032003900C
:105A0C000E90002008900F9005200690000704903F
:105A1C000DA90591FBF782FF039B04980599089A41
:105A2C0002250D950E930F92FBF778FF039B0498BC
:105A3C000599089A04240D940E930F92FBF76EFFB0
:105A4C00039A0599079B08980D930E920F902C487A
:105A5C000290FBF763FF0298039B0599089A0D953A
:105A6C000E930F92FBF75AFF0298039B0599089A25
:105A7C000D940E930F92FBF751FF039B049805991D
:105A8C00089A08240D940E930F92FBF747FF039B83
:105A9C0004980599089A10240D940E930F92FBF715
:105AAC003DFF069B079A089916480990164C04600E
:105ABC0043608160C1608023036113024361D202A1
:105ACC0082612022C2610162FBF7CAFA002801D070
:105ADC0007F036FE12980B490165129888620C206B
:105AEC0001900022114608F0E2F8019807F098F8AE
:105AFC0013B030BD0024014040100240341002406D
:0C5B0C0000040050680E00200800024059
:105B180030B58DB00C900BA8099001700AAC0894B0
:105B2800222001902070052000070790012106918E
:105B3800C90305910022029208F03DF90C980A2148
:105B4800039100910323049321462246FDF72EFA80
:105B58000599069A079808F02EF9029A0798059968
:105B6800A37807252B400B9D2B436370422323709A
:105B780008F021F903990C98009102232146224646
:105B8800FDF714FA0599069A079808F014F9019B8D
:105B9800029A07980599237008F00DF90399049B58
:105BA800089A0C9800911146FDF700FA0599069A93
:105BB800079808F000F9089909988A780178084642
:105BC8001040884203D0034805F03AFEFEE70DB0C6
:085BD80030BDC0460BEA0008D5
:105BE00000B581B0009000983121C900405800995B
:105BF00088670098CE21405A00997C2288520098EC
:105C0000CC21405A00997E2288520098D4214058D5
:105C10000099802288500348002102F0C3F901B0A6
:085C200000BDC046A0000020F9
:105C280000B585B004900498D4214058049A842182
:105C3800505004984058049980228958401A03907B
:105C48000A480068029002997D20C00048430399E1
:105C580005F002FD019001980499882288500448B3
:105C6800002102F09BF905B000BDC046E40F0020FA
:045C7800A000002068
:105C7C0000B585B00F490191CC200A5A8C200A52EC
:105C8C00085E7E22895E401A04900B4800680390DF
:105C9C0003997D20C0004843049905F0DBFC0146C4
:105CAC0001980291029990228150002102F074F91E
:0C5CBC0005B000BDA0000020EC0F00208F
:105CC80000B58DB00C90424805F0BAFD0C989C21A7
:105CD8004058002803D14A4805F0B2FD75E00C98F9
:105CE8009C210291405805F009FC00220992394B89
:105CF800039305F063FA384B01931A685B6805F063
:105D08005DFA099A0B910A900A980B99334B0893FC
:105D180007F039FD05F050FB014601980C9A9423D1
:105D28000793D1500C99CE22895A0C9A9823049340
:105D3800D1520C99CC22895A0C9A9A230593D152A4
:105D480043680268264805F07BFD02990C98405884
:105D580005F0D4FB039B099A05F030FA02460B467E
:105D6800204805F06DFD04990C98405E05F0C6FBCF
:105D7800099A1D4B069305F021FA02460B461B486B
:105D880005F05EFD05990C98405E05F0B7FB069B93
:105D9800099A05F013FA02460B46154805F050FD1E
:105DA80007990C98405805F0A9FB089B099A07F039
:105DB800EAFC02460B460F4805F042FD0E4805F086
:105DC8003FFD09990D4802F0E9F80DB000BDC04645
:105DD80087E5000800408F401006002080842E418F
:105DE80033E800088DE30008000059409CE30008F0
:105DF800F3E5000827EA0008FDE50008A0000020F8
:045E080099E5000810
:105E0C0000B58FB04A4805F019FD4A480A90CE21DA
:105E1C000191425AA0214252405E05F06DFB0022D6
:105E2C000992454B079305F0C7F902460B464348C8
:105E3C0005F004FD0A990198085E9822895E401AC3
:105E4C000B900B9805F058FB079B099A05F0B4F9D9
:105E5C0002460B463A4805F0F1FC3A4801684268A4
:105E6C000D920C9143680268374805F0E7FC0A98DC
:105E7C009C210291405805F03FFB099A334B039348
:105E8C0005F09AF902460B46314805F0D7FC029909
:105E9C000A98405805F030FB039B099A05F08CF9E1
:105EAC000C9A0D9B05F088F9099A0D910C900C98A1
:105EBC000D99284B089305F0D1F80D910C900C9886
:105ECC0004900D9805900B9805F016FB024604986B
:105EDC000B46059905F070F9099A0D910C900C98E8
:105EEC000D991D4B069307F04CFC05F063FA024626
:105EFC000A98A4214250405805F0FEFA069B099AD4
:105F0C0005F05AF9079B099A07F03BFC089B099A84
:105F1C0004F0C0FF02460B46104805F08FFC1048F9
:105F2C0005F08CFC09990A9802F036F80FB000BD08
:105F3C00A7E30008A000002000005940BEE30008C1
:105F4C0013E6000800060020CDE3000800408F4057
:105F5C0021E600080000F03F65CDCD4100E40008CB
:045F6C003BEA000804
:105F700000B58DB00AA90020059008810B9047213B
:105F80000A912A4909910870052000070290012210
:105F900001921103039107F012FF96200890FAF77F
:105FA00081F9059A224800902021069107F007FF09
:105FB0000898FAF777F90098019A069907F0FFFE1A
:105FC0000898FAF76FF902980399059A07F0F7FE17
:105FD000059A07200490022107F06FFE049806F04E
:105FE00025FE1448079000F027F80898FAF75AF9A8
:105FF00006990798FFF790FD0599079800F060F85B
:106000000699079800F0C0F80798342100F020F9AD
:1060100000F066F900F072FA0898FAF743F9099966
:106020000320087008F0F9F80DB000BDD21400206C
:0860300000040050A00D002047
:1060380010B58AB0099008AC079400220292A270A9
:106048001B48208005200007069001210591C903FF
:10605800049107F0B0FE09980A21039100910223E8
:1060680021462246FCF7A2FF0499059A069807F0F4
:10607800A2FE029A069804992623237007F09BFE35
:106088000399079A0998009103231146FCF78EFF9C
:106098000499059A069807F08EFE079880780A28D2
:1060A80003D0044805F0CCFBFEE70AB010BDC0469B
:0860B800460A000050E8000850
:1060C00030B58DB00C900BA8099001700AAC089403
:1060D00023200190207005200007079001210691E0
:1060E000C90305910022029207F069FE0C980A216B
:1060F000039100910323049321462246FCF75AFFA3
:106100000599069A079807F05AFE029A079805998A
:10611000A378EF252B400B9D2B4363704323237003
:1061200007F04DFE03990C98009102232146224668
:10613000FCF740FF0599069A079807F040FE019B7F
:10614000029A07980599237007F039FE0399049B7A
:10615000089A0C9800911146FCF72CFF0599069AB5
:10616000079807F02CFE089909988A780178084664
:106170001040884203D0034805F066FBFEE70DB0EF
:0861800030BDC0462BE600080B
:1061880030B58DB00C900BA8099001700AAC08943A
:106198002320019020700520000707900121069117
:1061A800C90305910022029207F005FE0C980A2106
:1061B800039100910323049321462246FCF7F6FE3F
:1061C8000599069A079807F0F6FD029A0798059927
:1061D800A3789F252B400B9D2B436370432323708B
:1061E80007F0E9FD03990C98009102232146224605
:1061F800FCF7DCFE0599069A079807F0DCFD019B81
:10620800029A07980599237007F0D5FD0399049B16
:10621800089A0C9800911146FCF7C8FE0599069A51
:10622800079807F0C8FD089909988A780178084600
:106238001040884203D0034805F002FBFEE70DB08A
:0862480030BDC04657EA000812
:1062500010B58CB00B900AA80890017009AC079497
:10626000512020700A98607000220292A2700520CE
:106270000007069001210591C903049107F09FFDD5
:106280000B980A2103910091022321462246FCF734
:1062900091FE0499059A069807F091FD029A0698D6
:1062A00004993123237007F08AFD0399079A0B980C
:1062B000009103231146FCF77DFE0499059A069888
:1062C00007F07DFD0798089980780978884202D008
:1062D000024805F0B9FA0CB010BDC04623E400082E
:1062E00000B5A3B005202290002021901F901F9898
:1062F000042834DC1EA90E9100228A707C48088094
:106300001DA81290827002800520000711900121C3
:106310001091C9030F9107F052FD0E99129A0A20AD
:10632000009074480323FCF745FE0F99109A1198CA
:1063300007F045FD12980078FF280CD11DA8407881
:106340001EA90978884206D11DA8807820A9087066
:106350000120219003E01F98401C1F90C7E721985F
:10636000002809D1052000070121C90207F03BFDE3
:10637000C820F9F797FFF5E720986021084320A986
:10638000087000201C901B901B98042830DC1AA970
:106390000991452008702098487019A80D90002296
:1063A0000280052000070C9001210B91C9030A917E
:1063B00007F005FD09990D9A0A2000904D48022327
:1063C000FCF7F8FD0A990B9A0C9807F0F8FC0D9869
:1063D0000078FF2808D119A840781AA909788842BE
:1063E00002D101201C9003E01B98401C1B90CBE7BE
:1063F0001C98002809D1052000070121C90207F0D7
:10640000F2FCFA20F9F74EFFF5E7002018901790FC
:10641000179804285CDC15A904910020039088805B
:10642000334815903448022206F043FC039A04993D
:10643000887013A8089082801392052000070790A7
:1064400001210691C903059107F0B9FC0499089A46
:106450000A20009027480623FCF7ACFD0599069A10
:10646000079807F0ACFC08980078FF282BD113A8F8
:10647000407815A90978884225D113A8807815A9F4
:10648000497888421FD113A8C07815A98978884215
:1064900019D113A841790291011D1748012206F074
:1064A00008FC0146029888420DD113A800794006E5
:1064B000002807D513A800798006002802D50120FE
:1064C000189005E000E0FFE71798401C17909FE741
:1064D000189800280AD1052000070121C90207F0F9
:1064E00082FC4B208000F9F7DDFEF4E723B000BD0D
:0C64F00025EC0000A00D00203C0F002057
:1064FC0000B599B0052018900020179016901698AA
:10650C0004283FDC5E4815905E4815A908910222CC
:10651C0006F0C9FB08998870002214920520000728
:10652C000B9001210A91C903099107F042FC0899CB
:10653C000A200090544814AA0C920423FCF734FD52
:10654C0009990A9A0B9807F034FC0C980078FF28EC
:10655C0014D114A8407815A9097888420ED114A832
:10656C00807815A94978884208D114A8C07815A953
:10657C008978884202D10120179003E01698401CBC
:10658C001690BCE7179800280AD1052000070121B6
:10659C00C90207F022FCAF204000F9F77DFEF4E7BA
:1065AC000020139012901298042859DC10A9039122
:1065BC00002002908880354810903248022206F064
:1065CC0072FB029A039988700EA8079082800E9233
:1065DC0005200007069001210591C903049107F0DD
:1065EC00E8FB0399079A0A20009027480623FCF73A
:1065FC00DBFC0499059A069807F0DBFB07980078FA
:10660C00FF2828D10EA8407810A90978884222D1F9
:10661C000EA8807810A9497888421CD10EA8C078A1
:10662C0010A98978884216D10EA841790191011DD3
:10663C001448012206F037FB0146019888420AD122
:10664C000F990DA8017000780006002802D50120D2
:10665C00139005E000E0FFE71298401C1290A2E7AF
:10666C00139800280AD1052000070121C90207F060
:10667C00B4FB19200001F9F70FFEF4E719B000BDC7
:10668C00F2EC00003C0F0020A00D002021EC0000DB
:10669C0000B591B00DA903910020029008720E90E4
:1066AC0047480D904748022206F0FDFA029A0399DA
:1066BC0088700AA8079002720B920A920992052020
:1066CC000007069001210591C903049107F071FBA5
:1066DC000399079A0A2000903B480923FCF764FCB5
:1066EC000499059A069807F064FB07980078FF2830
:1066FC0058D10AA840780DA90978884252D10AA825
:10670C0080780DA9497888424CD10AA8C0780DA987
:10671C008978884246D10AA8017A0191011D29483D
:10672C00042206F0C0FA0146019888423AD10B992E
:10673C0008A801700078000600282AD508A800785F
:10674C004007002825D508A800784006002820D44A
:10675C0008A80078000700281BD410A90020C870D6
:10676C000AA842798A7082794A70C07908701098A8
:10677C00C00D002806D0109815494018109010989C
:10678C00099005E01098C00D002801D110980990CF
:10679C0007E00E49C1204200885A401C8852FFF77E
:1067AC00E1FB07E00949C1204200885A401C88528D
:1067BC00FFF7D8FB099800F00DF811B000BDC046EA
:1067CC0012EC00003C0F0020A00D0020A0000020C7
:0467DC00010000FFB9
:1067E00010B59CB01B908A4800688A49884203D043
:1067F00087490868401C086087480168CA0F8A18E2
:106800005210891A01601B9A01688918016000689A
:10681000C10F401840101A901A9980480A903122EE
:10682000D20081500146C83109911A9A836FD21A59
:106830007B4B01931A60C96880228258891A19918A
:10684000199988228058484304F05CFE00220D927A
:10685000744B059304F0B6FC04F0B2FD019A0A995A
:10686000034609981893189B6324A4000B511268DF
:10687000189BD21A6C4B06931A600422805E7E220B
:10688000895E401A04F03EFE02460A9802920A46C9
:1068900002991792169117990491169903919021D4
:1068A000405804F02FFE024603980B46049906F068
:1068B0006EFF059B0D9A04F085FC04F081FD0146F6
:1068C0000698159100681599411A584801600068AA
:1068D00004F018FE0D9A564B06F059FF0D9A554BD1
:1068E00006F055FF0D9A544B04F06CFC02460A98D2
:1068F0000B4652494B600A604A6808920968079142
:106900009421405804F0FEFD0D9A4D4B04F05AFCC2
:10691000024607980B46089906F039FF0246099887
:106920000C460A99474B0C935C601A600622805E05
:106930009822895E401A04F0E5FD02460A980B92FF
:106940000A460B9913921291A421405804F0DAFDE3
:106950000D9A3D4B04F036FC11911090129813994A
:10696000109A119B06F013FF0D9A384B04F098FA19
:106970000A460C990F920E90086849680E9A0F9B70
:1069800006F005FF0D9A0B4631494B600860086818
:106990004968304B04F0D4FC002808D12C49086821
:1069A000496800222C4B04F0EBFC002806D01B4960
:1069B000192000010858E42288500BE02449086897
:1069C00049680022174B06F0E2FE04F0F9FC134977
:1069D000E42288500E480068152813DB0F49C8319F
:1069E000C869096A884203DD0C49C831C869086270
:1069F0000A49C831C869496A884203DA0749C83177
:106A0000C869486215490120086000201CB010BD0B
:106A100034100020FFFFFF7F38100020A00000206E
:106A2000E40F002000408F40EC0F0020E80F002012
:106A300000000840000049400000604110060020AE
:106A400080842E410006002065CDCD410000F03F3E
:106A50000806002000206140002061C0B80F00201F
:106A60000649C86D4042E12213014343D81705226D
:106A700092018B50891848607047C046A0000020E2
:106A800000B585B00D480190C06DE1210A010023D9
:106A90000093194604F0CCFD009B0A46019903922D
:106AA0000290F8200858F8314968054A04F0C0FD02
:106AB000029A039B04F020FE05B000BDA000002058
:046AC000A0860100AB
:106AC40000B58DB000200B9031480A9031482D213B
:106AD400C9004058002806D52E482D21C900405829
:106AE4004042059001E0002005900599C8170891DF
:106AF40009900020079006902648432189004058B9
:106B0400002815DC08980999214A0492002303936C
:106B140004F08CFD039B1F4AD26D04F0EBFD034689
:106B240003980A460499C91A90410691079016E001
:106B340008980999164A02920023019304F076FDFD
:106B4400144A43239B00D258D31704F0D3FD0346C1
:106B540001980A460299C91A90410691079007982C
:106B6400069A00210C4BD21A884104DB00200790BE
:106B74000748069008E00799069A00205242884187
:106B840002DB00200790069006980DB000BDC046B9
:0C6B9400A0860100A0000020A1860100E6
:106BA00010B5A8B00023169327932693259324931A
:106BB00023932293219320931F931E931D931C9341
:106BC0001B931A93EE48C06DE1210A01194604F0A7
:106BD0002FFD19911890EB48416800680843002880
:106BE00009D1FE484B2189004158FE484843FC49E1
:106BF00000224A600860FC48416800680843002899
:106C000009D1F648132109014158F6484843F6498D
:106C100000224A600860F148E421405800281ED450
:106C2000EE4813905221405A04F06CFC0022EF4BC6
:106C300004F0C8FA0246139814920A4614991F9257
:106C40001E91C8301590C06904F05CFC1E9A1F9B11
:106C500006F09DFD04F0B4FB1599886259E0DF4908
:106C60001291C86D6822895A04F022FD01461298DB
:106C70001791E421405817994942884245DAD7488C
:106C80000E90C8301190C06904F03CFC259124900E
:106C900024980C9025980D90179804F033FC024628
:106CA0000C980B460D9904F08DFA02460E980F923F
:106CB0000A460F992792269127990122D20751401F
:106CC00027915021405A04F01DFC00221092C74B1E
:106CD00004F078FA109A2391229022982399C44BB9
:106CE00004F0DEF802460B462799269803F07AFF57
:106CF0002191209024982599209A219B06F047FD08
:106D000004F05EFB1199886203E0B449C831C86998
:106D10008862B2487021425EC830816A891A8162F5
:106D2000C069002823D5AD480B90C8300A90C069CF
:106D30004442E317AA4948680A68121958410A6090
:106D4000486008684968A74A002304F0EDFC0B99E5
:106D500002460A984266426E7D20C0005043C96DCB
:106D600004F0A6FC0B994F229200885213E09B4836
:106D7000C8300990C469E3179B4948680A6812192A
:106D800058410A60486008684968964A002304F040
:106D9000CBFC0999886691490791C83108918C6AA2
:106DA000E317486B0A6B121958410A6348638C6AEF
:106DB000E317C86F8A6F121958418A67C867886FCE
:106DC000C96FE1221201002304F096FC079A0146E4
:106DD00008982D23DB00D150416B036B1998189A4A
:106DE000D21A884106DA1998189A7C49F823CA50B1
:106DF000F8314860794905208201881840688A582E
:106E00000021521E884106DB7449052082010020C2
:106E100088508918486071480690C16D5422805A84
:106E2000484304F0BBFB0022704B04F0CBF904F0A4
:106E3000E1FA0A4606991B921A90D820085858225F
:106E4000895A88420DDD6548E4214258D0171B99C4
:106E50001A9BD21A884104DA66490888401C0880C7
:106E600002E064490020088000216248405E5B49DE
:106E70005622895A88420DDD1898199A5749C83107
:106E80004A6308630020C867886703F053FB5A49C8
:106E90000120086051490491C8310591086B496B84
:106EA000E1221201002304F027FC04990246059810
:106EB000C26200690322D201895A884247DA4748F0
:106EC000D82140584D49884241DB4D480188491C32
:106ED000018000880A2839DB47480068012835D13D
:106EE00047490A2008803D480921490140580009C6
:106EF000E12826D3394809214901405841498842AF
:106F00001FD836482D21C9004058002805D43348E1
:106F10002D21C9004058039005E030482D21C900BB
:106F200040584042039003982C490291432292001A
:106F3000885003F075F902982F4A0021116001F082
:106F400031F82649492082000020885002E02C496F
:106F50000020088021486421405A0190042836D836
:106F60000198810001A040588746C046896F0008FB
:106F7000976F0008A56F0008B36F0008C16F000885
:106F8000A000002028060020FFF77AFD1349012207
:106F90001202885020E0FFF795FD104901221202ED
:106FA000885019E003F0A2F90C490122120288501E
:106FB00012E003F0D3F909490122120288500BE0D4
:106FC00003F03AFA054901221202885004E003490D
:106FD000012002020020885028B010BDA00000202F
:106FE0002806002080EE36003006002000005940C0
:106FF0000000F0BF40100020B40F0020E9030000A3
:087000003E10002080FC0A0094
:1070080000B587B006902D4800682D49884203D006
:107018002A490868401C08602A4801680A0A891A2F
:107028000160069A0168891801600068000A0590E5
:1070380005982549C83104914A88002303931946C5
:1070480004F0F2FA039B062204F0EEFA0A460499C9
:107058001204000C80180861184800681B4988420F
:1070680013DB1949C83108694969884203DD1649A3
:10707800C831086948611449C83108698969884272
:1070880003DA1149C8310869886106980E490291E6
:10709800CA228A5A00230193194604F0C5FA019BB3
:1070A800062204F0C1FA0A4602991204000C80185C
:1070B80065229200885007B000BDC0462C10002001
:1070C800FFFFFF7F30100020A0000020010A000011
:1070D80000B587B01A4806900698008804F04AFA66
:1070E800059005988B21C905019104F01DF80590BC
:1070F80005981449029103F0BBFF04F0B1F9124955
:1071080003910860114806900698008804F032FA46
:1071180001990490049804F007F8029904900498DF
:1071280003F0A6FF04F09CF90399024608480260A0
:1071380000680968401A0749086007B000BDC046E2
:10714800A875FF1F00803B45DC0F0020CA75FF1F94
:08715800E00F0020D80F002019
:1071600000B583B00290029910484843000C01908A
:1071700001980F490968401A019001990D48484348
:10718000019001980C49096804F06AFA019001988D
:107190000A494018019001980A2104F061FA08494F
:1071A000CC22885200F00EF803B000BDE40C0000C1
:1071B000DC0F0020A0860100D80F002030750000F1
:0471C000A00000200B
:1071C40030B583B018495A20085A0322D201885294
:1071D400CC20085E6A22895E884222DA1249CC20D9
:1071E4000A5A02AB1A80085E6C22895E884204DC6B
:1071F4000D486C21405A02A908800B4B01936C2066
:10720400185E6E21595E6A229A5E5A241B5F00251D
:1072140002AC645F009406F01AFA01990322D201C9
:0C722400885203B030BDC046A00000201E
:1072300000B583B00948026801210A430260006872
:10724000084002900298092001900121002206F0D6
:1072500034FD019805F0EAFC03B000BD381002408F
:1072600000B583B001901E48007880021D49401887
:107270006946012200F03EF8002803D002A903204D
:10728000087029E00198002802D000980199087040
:1072900068460078FF2806D1154804F0D5FA02A9FF
:1072A0000020087018E068460078392806D10F4899
:1072B00004F0CAFA02A9012008700DE068460078BF
:1072C000382806D1084804F0BFFA02A90220087045
:1072D00002E002A90320087002A8007803B000BDF4
:1072E000E075FF1F00F8FF0773EA00084DE600088D
:0472F00042E400086C
:1072F40086B00490039102920498029940181149AF
:10730400097889020122D2068918884203D905A97D
:107314000120087011E00020009000980299884232
:1073240008D20498009A805C039988540098401C01
:107334000090F2E705A90020087005A8007806B0BF
:087344007047C046E075FF1F11
:10734C00F0B587B006908C4804F078FA8B4805901D
:10735C0005994B20000288610599002000908883D4
:10736C0005990124CC8305990C84059948850599C8
:10737C0088850599C88505990886059948860599D3
:10738C0088860599C886059988630599C863059907
:10739C00086405994864059A794991640599C8640B
:1073AC000599086505994865059A76499165059A88
:1073BC0080236321D152059A82236921D152059AE7
:1073CC0084237149D150059A88237049D150059A6C
:1073DC008C230A21D152059A8E230221D152059B6E
:1073EC0090256B4A5A53059D92266A4BAB53059DCB
:1073FC009426AC55059C96256153059D9826664CA4
:10740C00AC53059C9A256353059C9C25634B635395
:10741C00059B9E241A53059BA024614A1A53059B75
:10742C00A2247D2201921A53059AA4235D4DD552B4
:10743C00059AA6235C4CD452059AA8265B4B935311
:10744C00059EAA275A4AF253059EAC27F553059D73
:10745C00AE26AC53059CB0256353059BB2241A533E
:10746C00059BB42432221A53059BB624514A1A5355
:10747C00059BB824504A1A53059BBA2407221A5369
:10748C00059ABC23D050059AC023D050059AC4232A
:10749C00D050059AC823D050059BCC245A221A539D
:1074AC00059AD023D050059A50661066059BC243AE
:1074BC009A66059BDA66059B5A67404A1A67059AD5
:1074CC00C943D1673E499167059A9168491C9160FF
:1074DC00059AD82191800599C880059939200870A2
:1074EC00FAF706F80198C000F9F798FF35480068DC
:1074FC00C007002804D03349086801229043086073
:10750C00314802210160314909784908491E8160DE
:10751C000121C16004A9FAF76BF8002800D0FEE73E
:10752C002A48007880022A494018039000200290D3
:10753C000398264909788902264A8918884214D268
:10754C0003990298C3000D4AD018D2584368012001
:10755C00F9F718FF002806D1039808300390029819
:10756C00401C029000E0FEE7E2E7F9F7E3FF069823
:10757C0000F032F807B0F0BD7BE60008580400209C
:10758C0090D0030040420F00A086010080482800E4
:10759C00B0360000D4300000E02E0000983A000015
:1075AC0083FF00004C1D0000581B000054F200002B
:1075BC0048F4000038FF00001027000000D68AEACB
:1075CC00007884C914200240A00F0020E075FF1F32
:0875DC0000F8FF07D4F8FF07D7
:1075E400F0B58BB00990CB4800788002CA494018A6
:1075F400CA49D822FFF77CFE002803D00AA901203B
:10760400087082E1C5480890089880690999086162
:107614000898808B099988820898C08B0999C88238
:107624000898008C099908830898408C09998883E4
:107634000898808C0999C8830898C08C0999088493
:107644000898008D099948840898408D09997C22EE
:1076540088520898808D09997E2288520898C08D96
:1076640009999827C8530898008E09999A2688532F
:107674000898408E09998C22039288520898808E2B
:107684000999A02408530898C08E0999A822069243
:1076940088520898806B0999802200928850089833
:1076A400C06B09998422029288500898006C099949
:1076B4008822019288500898406C0999902204927B
:1076C40088500898806C09999C2548510898C06C8A
:1076D4000999A423C8500898006D0999AC2207920F
:1076E40088500898406D099988670898806D099AB0
:1076F40094210591505000990898405A09995222B2
:10770400885208988221405A099950228852019A35
:107714000299089840580999C865039908988058AF
:10772400099A10660898405A099954228852089870
:107734008E21405A099A5621505204990898405A69
:1077440009995822885208989221405A099A5A2134
:10775400505205990898405C099964228852089807
:107764009621405A099968228852069A07990898DE
:10777400C05B099FB8860898805B099EF0860898CC
:10778400405B099D288708989E25405B099D688772
:107794000898005B099CA0870898A224005B099CB8
:1077A400E0870898C05A099B402418530898A623D8
:1077B400C05A099B422418530898805A099A4423B2
:1077C400D0520898AA22805A099A4623D05208987F
:1077D400405A0999482288520898AE21405A09997A
:1077E4004A2288520898B021405A09994C2288525A
:1077F4000898B221405A09994E2288520898B42117
:10780400405A09996A2288520898B621405A09991F
:107814006C2288520898B821405A09996E228852DD
:107824000898BA21405A0999702288520898BC21B4
:10783400405809994B22920088500898C02140581A
:1078440009991322120188500898C42140580999B3
:107854004D22920088500898C8214058099927223F
:10786400D20088500898CC21405A09997222885233
:107874000898D021405809992522D20088500899A7
:10788400486E0A6E099B1946F831F8241A5148606B
:107894000898806E09994322920088500898C06E17
:1078A40009991122120188500899486F0A6F099B9F
:1078B40005218C0119191A5148600899C86F8A6FFB
:1078C400099B2921CC0019191A5148600898C068ED
:1078D4000999486008988088D82803D00AA901200B
:1078E400087012E00898C088002803D00AA9012073
:1078F40008700AE008980078392803D00AA9012002
:10790400087002E00AA9002008700AA800780BB0E9
:10791400F0BDC046E075FF1F00F8FF0758040020C3
:1079240000B5B3B031903091F84803F08BFFF848BC
:1079340000788002F7494018F749D022FFF7D8FCB5
:10794400002803D032A90120087003E3F2482F90E5
:10795400F2482E902F98406D2E9948652F98408DAF
:107964002E9948852F98808D2E9988852F98806B25
:107974002E9988632F98C06B2E99C8632F98006C3A
:107984002E9908642F98408E2E9948862F98406C23
:107994002E9948642F98806D2E9988652F98C08DF4
:1079A4002E99C8852F98008E2E9908862F98806C62
:1079B4002E9988642F98808E2E9988862F98C06C73
:1079C4002E99C8642F98C08E2E99C8862F98006D62
:1079D4002E9908653098012803D14B2000022A9083
:1079E40002E02F9880692A902A982E99886130980D
:1079F400012802D10020299002E02F98808B299041
:107A040029982E9988833098012802D10120289042
:107A140002E02F98C08B289028982E99C88330981C
:107A2400012802D10120279002E02F98008C279092
:107A340027982E9908843098012802D10020269096
:107A440002E02F98408C269026982E9948843098EE
:107A5400012802D10020259002E02F98808C2590E7
:107A640025982E9988843098012802D100202490EA
:107A740002E02F98C08C249024982E99C8843098C2
:107A8400012802D10020239002E02F98008D23903A
:107A940023982E9908853098012802D163202290DA
:107AA40003E02F987821405A229022982E99802220
:107AB40088523098012802D19948219002E02F98E9
:107AC400C06F219021982E998422885030980128E3
:107AD40002D19448209003E02F98802140582090B0
:107AE40020982E99882288503098012802D10A20A3
:107AF4001F9003E02F988421405A1F901F982E99BD
:107B04008C2288523098012802D169201E9003E00B
:107B14002F987A21405A1E901E982E9982228852BC
:107B24003098012802D102201D9003E02F9886216D
:107B3400405A1D901D982E998E2288523098012803
:107B440002D179481C9003E02F988821405A1C9058
:107B54001C982E99902288523098012802D173489B
:107B64001B9003E02F988A21405A1B901B982E9952
:107B7400922288523098012802D101201A9003E001
:107B84002F988C21405C1A901A982E99942288542C
:107B94003098012802D10220199003E02F988E21F9
:107BA400405A199019982E99962288523098012893
:107BB40002D1EF48189003E02F989021405A189072
:107BC40018982E99982288523098012802D1E748B3
:107BD400179003E02F989221405A179017982E99E6
:107BE4009A2288523098012802D1E248169003E084
:107BF4002F989421405A169016982E999C228852B8
:107C04003098012802D1D848159003E02F98962186
:107C1400405A159015982E999E2288523098012822
:107C240003D17C20C043149003E02F989821405E38
:107C3400149014982E99A02288523098012802D1C9
:107C44007D20139003E02F989A21405E139013989F
:107C54002E99A22288523098012802D1C648129047
:107C640003E02F989C21405E129012982E99A42232
:107C740088523098012802D1C048119003E02F980F
:107C84009E21405E119011982E99A6228852309818
:107C9400012802D1BA48109003E02F989E21405E3B
:107CA400109010982E99A82288523098012802D159
:107CB400B4480F9003E02F98A221405E0F900F98D4
:107CC4002E99AA2288523098012802D1AA480E90EF
:107CD40003E02F98A421405E0E900E982E99AC22BA
:107CE40088523098012802D1A4480D9003E02F98BF
:107CF400A621405E0D900D982E99AE2288523098A0
:107D0400012815D19E480C9016E0C046BBEA000835
:107D1400E075FF1F00F8FF0730050020580400201D
:107D2400A086010080482800B0360000D43000004E
:107D34002F98A821405E0C900C982E99B02288525E
:107D44003098012802D18F480B9003E02F98AA2184
:107D5400405E0B900B982E99B222885230980128DD
:107D640002D132200A9003E02F98AC21405E0A90A1
:107D74000A982E99B42288523098012803D1C7203A
:107D8400C043099003E02F98AE21405E0990099802
:107D94002E99B62288523098012802D17A48089048
:107DA40003E02F98B021405A089008982E99B822E1
:107DB40088523098012802D10720079003E02F98B9
:107DC400B221405E079007982E99BA2288523098C3
:107DD400012802D10020069003E02F98B4214058D6
:107DE400069006982E99BC2288503098012802D11A
:107DF4000020059003E02F98B8214058059005987D
:107E04002E99C02288503098012802D15A2004901B
:107E140003E02F98C421405A049004982E99CC2250
:107E240088523098012802D10020039003E02F9853
:107E3400C8214058039003982E99D02288502E9937
:107E44000020486608662E9AC14391662E9AD16630
:107E54002E9A51674D4911672E9A0221C943D16761
:107E64004B4991672E99C42288502E99C822885074
:107E74002F9A9168491C91602E9A91602E9AD8216C
:107E840091802E99C8802E99392008703098012845
:107E940002D10020029002E02F98007C0290029808
:107EA4002E9908743098012802D10020019002E034
:107EB4002F98C068019001982E99C860F9F71CFBAF
:107EC4007D20C000F9F7AEFA32480068C0070028E8
:107ED40004D0304908680122904308602E480221EA
:107EE40001601E4909784908491E81600121C16069
:107EF4002DA9F9F781FB002800D0FEE71748007888
:107F04008002174940182C9000202B902C9813497C
:107F140009788902214A8918884214D22C992B980D
:107F2400C300104AD018D25843680120F9F72EFA3A
:107F3400002806D12C9808302C902B98401C2B90AC
:107F440000E0FEE7E2E7F9F7F9FA3198FFF748FBBA
:107F540032A9087032A8007833B000BDE075FF1F65
:107F640000F8FF0758040020B0360000D4300000A9
:107F7400E02E0000983A00004C1D0000581B000041
:107F840054F2FFFF48F4FFFF1027000000D68AEAEE
:107F9400007884C914200240A00F0020D4F8FF0701
:107FA400F0B58FB00E900DA808900170E44803F06E
:107FB40049FCE4480C900E9800690C9988610E986D
:107FC400808A0C9988830E98C08A0C99C8830E986D
:107FD400008B0C9908840E98808B0C9948840E9819
:107FE400C08B0C9988840E98008C0C99C8840E98C8
:107FF400408C0C9908850E987E21405A0C998885EE
:108004000E987C21405A0C9948850E989821069127
:10801400405A0C99C8850E989A210791405A0C9998
:1080240008860E988C210391405A0C9948860E9824
:10803400A026805B0C9988860E98A824005B0C9976
:10804400C8860E98802280580C9988630E988421E3
:10805400019140580C99C8630E98882102914058A8
:108064000C9908640E989021049140580C99486426
:108074000E989C27C0590C9988640E98A4254059E1
:108084000C99C8640E98AC23C0580C9908650E98D6
:10809400806F0C9948650E989421059140580C996D
:1080A40088650E985221405A0C9988520E98502196
:1080B400405A0C9982228852019A0E98C06D0C99EC
:1080C4008850029A0E98006E0C998850039A0E9864
:1080D4005421405A0C9988520E985621405A0C99B2
:1080E4008E228852049A0E985821405A0C9988522C
:1080F4000E985A21405A0C9992228852059A0E9849
:108104006421405A0C9988540E986821415A0C9A5B
:108114009620115206980E99898E0C9A115207983E
:108124000E99C98E0C9A115208980E99098F0C9ABF
:10813400D1530E99498F0C9A9E27D1530E99898F4A
:108144000C9A91530E99C98F0C9AA22691530E99A9
:108154004022895A0C9A51530E994222895A0C9AF8
:10816400A62551530E994422895A0C9A11530E99FB
:108174004622895A0C9AAA2411530E994822895AE4
:108184000C9AD1520E994A22895A0C9AAE23D15292
:108194000E994C22895A0C9AB023D1520E994E2230
:1081A400895A0C9AB223D1520E996A22895A0C9A8E
:1081B400B423D1520E996C22895A0C9AB623D15207
:1081C4000E996E22895A0C9AB823D1520E997022B4
:1081D400895A0C9ABA23D1520E994B22920089588B
:1081E4000C9ABC23D1500E991322120189580C9A6F
:1081F400C023D1500E994D22920089580C9AC42361
:10820400D1500E992722D20089580C9AC823D150F4
:108214000E997222895A0C9ACC23D1520E99252296
:10822400D20089580C9AD023D1500E990A46F832BC
:10823400F823C95853680C9A536611660E99432261
:10824400920089580C9A91660E991122120189584C
:108254000C9AD1660E9905229301CA18C95853681D
:108264000C9A536711670E992922D300CA18C9586A
:1082740053680C9AD36791670C9A9168491C916072
:108284000C9AD82191800C9A0021D1800C9A392122
:1082940011700078002806D02B4803F0D3FA0E980A
:1082A40040680C99C860F9F727F97D20C000F9F7F8
:1082B400B9F826480068C007002804D02349086894
:1082C4000122904308602248022101602149097873
:1082D4004908491E81600121C1600BA9F9F78CF995
:1082E400002800D0FEE71B48007880021A49401895
:1082F4000A90002009900A98164909788902174AB9
:108304008918884214D20A990998C3000D4AD018D2
:10831400D25843680120F9F739F8002806D10A98A1
:1083240008300A900998401C099000E0FEE7E2E753
:10833400F9F704F90E98FFF753F90FB0F0BDC046F2
:1083440091E600085804002075E800081420024053
:10835400A00F0020E075FF1F00F8FF07D4F8FF0707
:1083640000B587B016484F218900405A002803DC25
:1083740006A9154808801EE01148C8300190C06E57
:1083840003F00AF90246019802920391006F03F088
:1083940003F9024602980B46039902F011FF059176
:1083A4000490049805990022064B05F0EEF903F0B9
:1083B40005F806A90880002106A8405E07B000BDA4
:0C83C400A000002000005940FFFF000056
:1083D00010B594B090492520C00008588F4A126803
:1083E000801ACD22520088521F2012901298012824
:1083F00011DB12988A4982008818001F0068885093
:108400001298884982008818001F006888501298C6
:10841000401E1290EAE78048C830C169804A116066
:1084200000698049086080491191002010900F91E7
:108430000E90C1430D910C910B910A9112901298DC
:108440001F2853DC1298810075484058C1174840D6
:10845000401A0F99884209DA1298810070484058F2
:10846000C1174840401A0F9012980D901298810041
:108470006B484058C1174840401A0E99884209DBA2
:108480001298810066484058C1174840401A0E9023
:1084900012980C901298810062484058C1174840C9
:1084A000401A1199884209DA129881005D484058B3
:1084B000C1174840401A119012980B9012988100F1
:1084C00058484058C1174840401A1099884209DD61
:1084D0001298810053484058C1174840401A1090E4
:1084E00012980A901298401C1290A8E70E980F99C3
:1084F000401AC1174840401A099010981199401A23
:10850000C1174840401A08904349C86D6822895AEB
:1085100003F0CEF807900798142103F0A1F8079014
:108520001920069009980799884203DA13A941484F
:1085300008806BE008980699884203DA13A93C4842
:10854000088063E00020C1430591049103911290DB
:1085500012981E2816DC129831498200881840684B
:108560008958401AC1174840401A04900498059948
:10857000884203DD04980590129803901298401CDD
:108580001290E5E7039810283DD1089802F0BAFF51
:1085900000900191099802F0B5FF024600980B4641
:1085A000019902F00FFE00220292204B05F0EFF835
:1085B00002F006FF02460298174947239B00CA5261
:1085C0002522D2008958154A1160129012981F284E
:1085D00019DC12998A00124880581F22511A8B0008
:1085E0000D49C831CB18F0241851129B9C000D483E
:1085F0000059D21A92008918172212018850129835
:10860000401C1290E2E713A900200880002113A863
:10861000405E14B010BDC046A00000202010002015
:10862000200D0020200C0020FFFFFF7F00408F4026
:08863000FEFF0000FFFF000047
:1086380010B594B091492520C0000858904A126896
:10864800801ACD22520088521F20129012980128B9
:1086580011DB12988B4982008818001F0068885027
:108668001298894982008818001F0068885012985B
:10867800401E1290EAE78148192109014158814AB0
:108688001160D42140588049086080491191002028
:1086980010900F910E90C1430D910C910B910A917E
:1086A800129012981F2853DC129881007548405880
:1086B800C1174840401A0F99884209DA1298810078
:1086C80070484058C1174840401A0F9012980D90B2
:1086D800129881006B484058C1174840401A0E99BB
:1086E800884209DB1298810066484058C117484003
:1086F800401A0E9012980C901298810062484058C7
:10870800C1174840401A1199884209DA1298810025
:108718005D484058C1174840401A119012980B9074
:108728001298810058484058C1174840401A10997B
:10873800884209DD1298810053484058C1174840C3
:10874800401A109012980A901298401C1290A8E7AC
:108758000E980F99401AC1174840401A099010986E
:108768001199401AC1174840401A08904349C86DEA
:108778006822895A02F098FF07900798C117890F55
:10878800401880100790642006900998079988423D
:1087980003DA13A9404808806BE0089806998842D4
:1087A80003DA13A93B48088063E00020C143059120
:1087B80004910391129012981E2816DC12983149E0
:1087C8008200881840688958401AC1174840401AE2
:1087D800049004980599884203DD0498059012983E
:1087E80003901298401C1290E5E7039810283DD199
:1087F800089802F083FE00900191099802F07EFE2D
:10880800024600980B46019902F0D8FC0022029219
:108818001F4B04F0B8FF02F0CFFD0246029817493B
:108828008F235B00CA522522D2008958144A11604E
:10883800129012981F2819DC12998A001148805842
:108848001F22511A8B000D49C831CB181401185139
:10885800129B9C000C480059D21A920089182722B2
:10886800120188501298401C1290E2E713A90020C8
:108878000880002113A8405E14B010BDA00000209D
:108888001C100020A00C0020A00B0020FFFFFF7F81
:0C88980000408F40FEFF0000FFFF0000CA
:1088A40000B58FB00E900D91284800682849884281
:1088B40003D026490868401C08600E980D99401A98
:1088C40002F01EFE0B910A900B9802900A980190F8
:1088D40020480790CA21405A02F012FE024601982D
:1088E4000B46029904F051FF002204921A4B02F045
:1088F40067FC049A0B910A900A980B99174B02F0A3
:108904005FFC174A174B02F05BFC02460798039280
:108914000A460399099208910999069108990591C3
:108924009421405802F0ECFD049A0F4B02F048FCED
:10893400024605980B46069904F027FF02F03EFD17
:1089440007991922120188500FB000BD1810002099
:10895400FFFFFF7FA00000200000F0400000444023
:0C896400FCA9F1D24D62403F80842E41FE
:1089700030B58FB000200E900D900C900B900A90A7
:108980003648026802210A430260006808400990E4
:1089900009983248026804210A43026000680840CE
:1089A000089008982D48026820210A430260006858
:1089B0000840079007982948026801210A4302608D
:1089C0000068084006900698052000070190F921EC
:1089D0004D0100220392294605F0F1F9039A012086
:1089E000029004021E480490214605F0E8F902991D
:1089F00004984A020A92212212040B920C910AA9AD
:108A00000591F8F791FF0198029B039A05990A9541
:108A10000B930C920D92F8F787FF0298039A059931
:108A200040230A930B920C900E48F8F77DFF029BAF
:108A3000039A049805990A940B930C920D92F8F7F7
:108A400073FF029B039A0498059920240A940B93C0
:108A50000C930D92F8F768FF0FB030BD3410024050
:088A6000000400500008005062
:108A680081B0014668460180008801214902884298
:108A780002D102490120086001B07047B80F0020F8
:108A880030B5A5B000201390249023902290209018
:108A98001F901E901B901A9019A9087018A90870A9
:108AA80000F058FA0028FFD125490868012212026F
:108AB80090430860F7F788FB00F084FA214802F039
:108AC800BFFEFCF719F9FCF7D1F9FCF7BFF8FFF77F
:108AD8004BFFFEF7A9FB01F067F8FCF7C1FE00F0B9
:108AE800C3FE00F0D1FA01F037F901F07DFAFDF785
:108AF800B3FF16A81190FEF7AFFB1199024615A80F
:108B080002700378104A53800978D1810078129056
:108B1800032823D81298810001A040588746C046F0
:108B2800398B0008418B0008558B00085F8B0008C3
:108B3800F648FEF707FC11E0F448FEF74FFD0DE09C
:108B48000020024059E40008A0000020EF4800215E
:108B5800FEF7E4FE02E0ED48FEF7F4FBEC4802F015
:108B68006FFEEA48FEF73AFDEA48402104F057F95B
:108B780000280FD13220F7F791FBE648402104F096
:108B88004EF9002806D1E44802F05AFEDF480121D8
:108B9800FEF7C4FEDD480169828AC38ADF48009077
:108BA800DF4804F08FFCFEF793FADE481090F8F7E0
:108BB80067F81098DC490922F7F7C6FD6420F7F733
:108BC8006DFBFDF7D1F9D94802F03AFE00F0CCFB75
:108BD800002014901498CD49098B884218DA052092
:108BE80000070D900122D1020E9105F0E4F8AF20A4
:108BF80040000F90F7F752FB0D980E99002205F0F0
:108C0800DAF80F98F7F74AFB1498401C1490E1E73C
:108C1800C7480068012827D1C54900200B90086083
:108C2800C1480A90806800F0F7FD0A98006800F0D3
:108C38009FFF0A984068FEF7E3F90A99C86809692E
:108C4800FFF72CFEB14AC8320C921069C117D269DD
:108C5800D31702F0E9FC0B9B7D22D20002F048FDFD
:108C68000C990864FFF7E4FCB2480068012806D1B3
:108C780005F0D7FAFFF7A8FBAE4900200860F7F720
:108C880007FB229022982399401A2190229823903A
:108C9800219920984018209021991F9840181F90DA
:108CA8001A98012805DB2198002802D01A98401E3E
:108CB8001A90A14801680A680F210A4019A90A7088
:108CC80000684068179018A80078097888426DD025
:108CD800199818A908708D492520C2008858401C89
:108CE80088501B9800280BD1052000070121099105
:108CF800890205F074F809980102904805F06FF8A8
:108D0800FDF74AFF01F080F900F038FB00F05CFC49
:108D180000F0E6F900F010FE7C4908916722920005
:108D28008852FFF71BFB08998B22520088527E4815
:108D38000490006AFEF710FA0498C06900F0DEFE9D
:108D4800049808994069CA2203928A5A0023069314
:108D5800194602F069FC069B0B22059202F064FC9E
:108D680002F026FC069A764B079302F027FA02F0E7
:108D780023FB039A069B08990446049815252D01A0
:108D88004C5380698A5A194602F04EFC059A069B94
:108D980002F04AFC02F00CFC069A079B02F00EFA5D
:108DA80002F00AFB0899A922520088525748408BC2
:108DB800002873D05A482621405C00286ED15348B9
:108DC800408B029001282CD0029802282ED00298BD
:108DD80003282FD00298042831D00298062837D0CB
:108DE8000298072836D00298082837D00298092810
:108DF80038D002980A2838D002980B2839D002981F
:108E08005049884238D002984F49884238D0029851
:108E1800FD218900884237D002984C49884212D0F7
:108E280035E03A480021FFF7B9F833E03748FEF754
:108E380089FA2FE035480121FEF770FD2AE0334812
:108E4800FEF7CCFB26E031480121FFF7A7F821E027
:108E580000F064F92D48FCF7BFFE1BE02B48FCF737
:108E6800DFFE17E0FCF706FF14E02848FCF728FFB0
:108E780010E0FCF7C7FF0DE0002000F05DF909E005
:108E8800012000F059F905E000F00AFA02E0304844
:108E980002F0D6FC1D4900204883FFE71D48402109
:108EA80003F0BDFF00281BD11A98002818D10A200A
:108EB800F7F7F4F91748402103F0B1FF00280FD164
:108EC8007D2080001A901B98002807D101221B9250
:108ED80005200007910204F06EFF01E000201B90BE
:108EE8000F4805F054F900280FD00D48FCF716FB81
:108EF800022806D11B98002802D1094804F05BFB20
:108F080003E0064984222220885081E6A000002040
:108F1800DBEA000800080050EBEA0008140B002008
:108F280038060020040E0020600F0020A7E6000885
:108F3800BC0F0020B80F0020100F002000040050C4
:108F480000002441F2030000F3030000D2040000F3
:048F580082E80008A3
:108F5C0000B589B00020009008900790069005900D
:108F6C0004900390029002A8F8F796FC009801A9CF
:108F7C0008700698AA2806D1104802F05FFC01A9D7
:108F8C000020087012E00698BB2806D10A4802F0AF
:108F9C0055FC01A90120087008E00698CC2805D1E1
:108FAC00044802F04BFC01A90220087001A80078CB
:108FBC0009B000BD4BEB00082FEB000813EB0008C9
:108FCC0000B59BB00EA80290342103F0E1FB002009
:108FDC0000900D900C900B900A90099008900790BF
:108FEC000690059004900390012001908002F8F700
:108FFC001DFEF8F707FE2149086818221043086087
:10900C00F8F70AFE009A0199029806230E93109124
:10901C000B02119312924023139302231593169370
:10902C001792082218924A04199249071A91F8F7D4
:10903C0037FE002801D004F083FB07200A900221A0
:10904C000B9100200C900D900AA8F9F70FF900284D
:10905C0001D004F075FB0A48039000200490012015
:10906C00810708910002099003A8F9F7AFFA0028CC
:10907C0001D004F065FB1BB000BDC0465C10024083
:04908C00014002009D
:1090900000B583B011480268012109030A43026048
:1090A00000680840029002980D4801900D49016047
:1090B000012101714171072282601022C260FF22EA
:1090C00002610022426182610162F7F76DFF0028B0
:1090D00001D004F03BFB03B000BDC0463810024095
:0890E0003C0F002000300240AB
:1090E80000B581B00A482521C9004058094902F055
:1090F800DBFA0090009808490968884206D0009871
:109108000549086002480021FEF748FF01B000BD8C
:0C911800A000002080510100F40F002096
:10912400BFF34F8F034904480860BFF34F8F00BF5C
:0C913400FDE7C0460CED00E00400FA0569
:1091400000B58BB009A90191087000200890079024
:109150000690059004900390029002A8F8F7A2FBF5
:1091600001980078C00700283AD04A4802F06CFB0A
:109170000698AA2830D102200290BB200690F8F76A
:10918000BDF9002802D0424802F05EFBF8F7F6F97C
:10919000002802D03D4802F057FB404802F054FB43
:1091A00002A8F8F7B7FA002808D03E4802F04CFBB6
:1091B000F8F706FA0AA90020087055E0F8F700FA57
:1091C0002E4802F041FBF8F7BBF92D4802F03CFBBA
:1091D000334802F039FB02E02F4802F035FB40E053
:1091E0000698BB283DD102200290AA200690F8F7ED
:1091F00085F9002806D0264802F026FB0AA900209F
:10920000087031E01A4802F01FFBF8F7B7F90028A0
:1092100006D01E4802F018FB0AA90020087023E0BF
:10922000144802F011FB02A8F8F774FA002808D0DD
:10923000F8F7C6F9144802F007FB0AA900200870E5
:1092400012E00D4802F000FBF8F7BAF90B4802F003
:10925000FBFAF8F775F90A4802F0F6FA094802F045
:10926000F3FA0AA9012008700AA800780BB000BD23
:109270008EE40008E9E60008FFE80008C5E80008F9
:109280007FE4000821E70008FFE6000868E4000822
:10929000FFEA000893E80008CBE60008B4E80008FD
:0892A000DEE80008B5E6000855
:1092A80000B589B0002007900690059004900390BF
:1092B8000290019001A8F8F7F1FA062001900190B8
:1092C800BB200590072000060690052000060790A1
:1092D800F8F710F9002802D0174802F0B1FAF8F7A9
:1092E80049F9002802D0154802F0AAFA144802F0F9
:1092F800A7FA01A8F8F70AFA002808D0144802F0DB
:109308009FFAF8F759F908A9002008700FE0F8F754
:1093180053F90C4802F094FAF8F70EF90A4802F0EB
:109328008FFA0A4802F08CFA08A90120087008A8E8
:10933800007809B000BDC046FFEA000868E40008EC
:10934800B4E80008C5E800087FE40008DEE8000883
:04935800B5E600086E
:10935C0081B0009002490120086001B07047C046FE
:04936C00BC0F002012
:109370000249C8310248C88788877047A00000208A
:04938000FFFF0000EB
:1093840080B589487421405A002800D0E6E0874817
:109394000088002804D084498320420084488852ED
:1093A400814883214900405E002807D07E488321FC
:1093B4004900405E401C002800D088E07A49D8204B
:1093C4000858898E88420EDA7E4802F03BFA7648C5
:1093D40083214A000121815205200007490200220D
:1093E40004F0EBFC73E07049E42008583C228A5EE8
:1093F4007D21C900514388420FDA714802F022FAF4
:109404006949832042000220885205200007012177
:109414004902002204F0D1FC59E06349CE20085EE1
:109424004822895E88420FDD644802F00BFA5E49E7
:1094340083204200032088520520000701214902AD
:10944400002204F0BAFC42E05749CC20085E4822CE
:10945400895E88420FDD574802F0F4F952498320AF
:1094640042000420885205200007012149020022FD
:1094740004F0A3FC2BE04C49CE20085E4C22895E0C
:1094840088420EDA4C4802F0DDF947498320420055
:1094940005208852000701214902002204F08DFCB6
:1094A40015E04149CC20085E4C22895E88420EDAE0
:1094B400404802F0C7F93C49832042000620885204
:1094C4000520000701214902002204F076FC3648F9
:1094D40083214900405E00283FD03349D8200858F2
:1094E400C98E884239DD3049E42008583C228A5E1E
:1094F4007D21C900514388422FDD2B49CE20085ECF
:109504004A22895E884228DA2749CC20085E4A220A
:10951400895E884221DA2449CE20085E4E22895E83
:1095240088421ADD2049CC20085E4E22895E88429A
:1095340013DD1D4883214900405E02280DD02248D6
:1095440002F080F918498320420000208852052047
:1095540000070122510204F030FC1FE0124874217C
:10956400405A012806D1052000070122510204F0C7
:1095740024FC13E00C487421405A022807D105202A
:10958400000701214902002204F017FC06E005202F
:10959400000701214902002204F00FFC0248742153
:1095A400405A0249088080BDA00000203C100020E1
:1095B400FFFF000065E7000867EB0008A1E400086E
:0C95C4001CE9000843E70008C4E40008AC
:1095D00080B589487621405A002800D0E6E08748C7
:1095E0000088002804D084494120820084488852A1
:1095F000814841218900405E002807D07E484121F2
:109600008900405E401C002800D088E07A49D820BC
:109610000858098F88420EDD7F4802F015F9764818
:1096200041218A0001218152052000070902002200
:1096300004F0C5FB73E07049E42008583E228A5EBE
:109640007D21C900514388420FDD724802F0FCF8C9
:10965000694941208200022088520520000701212B
:109660000902002204F0ABFB59E06349CE20085EFA
:109670004022895E88420FDD654802F0E5F85E49C8
:1096800041208200032088520520000701210902A1
:10969000002204F094FB42E05749CC20085E4022AF
:1096A000895E88420FDD594802F0CEF852494120C8
:1096B00082000420885205200007012109020022AF
:1096C00004F07DFB2BE04C49CE20085E4422895EED
:1096D00088420EDA4C4802F0B7F847494120820030
:1096E00005208852000701210902002204F067FBCF
:1096F00015E04149CC20085E4422895E88420EDA9A
:10970000404802F0A1F83C494120820006208852DE
:109710000520000701210902002204F050FB364811
:1097200041218900405E00283FD03349D8200858A5
:10973000498F884239DA3049E42008583E228A5E4F
:109740007D21C900514388422FDA2B49CE20085E83
:109750004222895E884228DA2749CC20085E4222CC
:10976000895E884221DA2449CE20085E4622895E3D
:1097700088421ADD2049CC20085E4622895E884254
:1097800013DD1D4841218900405E02280DD0234889
:1097900002F05AF818494120820000208852052022
:1097A00000070122110204F00AFB1FE01248762193
:1097B000405A012806D1052000070122110204F0B9
:1097C000FEFA13E00C487621405A022807D1052002
:1097D000000701210902002204F0F1FA06E0052049
:1097E000000701210902002204F0E9FA024876216B
:1097F000405A0249088080BDA00000209E00002041
:10980000FFFF0000A9E700088BEB000887E70008CE
:10981000D3E4000856E9000835E90008F6E400083A
:1098200000B583B002900E4801688A09891A016068
:10983000029A016889180160006880090190019905
:1098400008484843010C0848C8228152C83000909B
:109850000199064801F02CFF0099488003B000BD33
:1098600008100020E40C0000A00000200000B80B4D
:1098700000B589B0002101910891079106910591E9
:10988000049103911C4802901C4A026081607F226F
:10989000C260FF22026141618161C16101229207C0
:1098A00002624162F8F79AFF002801D003F04EFFF0
:1098B00004A9022008700020487088700590079065
:1098C00008900D480122F9F79DF8002801D003F017
:1098D0003DFF03A901220A700420487016208870F9
:1098E0001820C8700448F9F727F9002801D003F0C0
:1098F0002DFF09B000BDC046100F00200028004019
:1099000082B00190019800680A4988420FD10A4844
:109910000268012189020A43026000680840009041
:109920000098064908680122D2031043086002B07B
:109930007047C046002800403C1002405C100240C6
:1099400000B58DB05F480B905F480A900A200990DF
:109950005E48019058210091405A01F0D3FD5C4AC5
:109960005C4B03F014FF01F02BFD009902460198B7
:109970000892405A01F0C6FD574A584B03F007FFC2
:1099800001F01EFD01460198079155490968CF2253
:1099900052008152D8214058069006980899884272
:1099A00008DD5049002008604D4908600CA9544862
:1099B000088081E006980799884208DA4949002022
:1099C0000860474908600CA94D48088074E0454884
:1099D0000068002802D106984249086041480168A1
:1099E0000A31059100680A38049006980599884262
:1099F00008DD3C4900200860394908600CA93F484F
:109A0000088059E006980499884208DA3549002010
:109A10000860334908600CA9384808804CE02B499D
:109A2000E42008587022895E884208DA2D49002017
:109A300008602B4908600CA92F4808803CE02848A2
:109A40000168491C016000682749884208D31F4902
:109A5000E420085870228A5A801A2322D2008852A1
:109A60001A482321C900405E012822DB174825211E
:109A7000C90040581D4901F01BFE039003981C4982
:109A80000968884215D00398194908601948016887
:109A90008A09891A01600D492322D2008B5E02686F
:109AA000D218026000688009029002988D2252004C
:109AB00088520CA90020088000210CA8405E0DB03F
:109AC00000BDC04651B89E3FB81E85EBA0000020E7
:109AD0007B14AE47E17AF03F0AD7A3703D0AEF3F0F
:109AE00000100020F80F0020312A000080510100F2
:109AF000FC0F002004100020FDFF0000FEFF00000E
:049B0000FFFF000063
:109B040000B583B00290029917484843C117090C65
:109B140040180014019001981449401801900199CB
:109B240064204843019001980A2101F097FD1049EF
:109B3400C831C8800620085E0822895E884204DD98
:109B44000B49C831C88808810BE00949C83106208F
:109B5400085E0A22895E884203DA0549C831C8884A
:109B6400488103B000BDC046E40C0000A8FDFFFF1F
:049B7400A00000202D
:109B780000B585B004900498C1170A4AC832029209
:109B880052880023019301F04FFD019B062201F04A
:109B98004BFD0A4602991204000C8018C86005B0F3
:089BA80000BDC046A000002032
:109BB00000B581B010480090104901604121890032
:109BC00041600021816007221302C360016101230B
:109BD00043619B0483611023C3610162416281621E
:109BE000C26201634163F9F72BF8002801D003F04A
:109BF000ADFD01B000BDC046A00D00200030014009
:109C000000B591B0109000200F900E900D900C9028
:109C10000B90109800681E49884236D11D48026892
:109C2000012109030A430260006808400A900A986B
:109C30001948026801210A4302600068084009903F
:109C40000998E0200B9002200C90002001900D90CC
:109C50000E900F900520000702900BA9F7F764FE05
:109C600001990298089107910691059104910122AA
:109C70000392D30304930592069104A9F7F754FEC7
:109C80000298039A202104F09AF811B000BDC04652
:0C9C90000030014040100240341002403F
:109C9C0082B00A48026801210A4302600068084049
:109CAC000190019806480268012109070A430260E5
:109CBC00006808400090009802B0704740100240C5
:049CCC003C10024006
:109CD00002480068002800D1FAE7704714100020FD
:109CE00000B581B0F6F7CCFA0D480168491C016057
:109CF0000C4900910068C0087D280FD3F6F7CCFA14
:109D0000094988420AD30949C831C86D401CC86551
:109D1000886D401C886502490020086001B000BDC4
:109D2000F00F0020204E0000214E0000A000002077
:109D300080B50248F7F78CFA80BDC046680E002057
:109D400080B50248FBF774FA80BDC046140B0020B2
:109D500080B50248F9F7ACFD80BDC046C40E0020B6
:109D600030B518490122500208800B46C833002044
:109D7000D86598654524A500134C4C53C5435D64D4
:109D80009D644725AD004C538F256D004C53232512
:109D9000ED004C538D256D004C5302240C814A81FB
:109DA00005248C81D4071C62084C5C62D2031A81A2
:109DB000074A5A81074C5C619A61C122520088525D
:109DC00030BDC046A0000020FFFF0000FFFFFF7F66
:089DD000FF7F00000080FFFF8F
:109DD80000B587B054480068382108400090202812
:109DE80000D982E00098810001A040588746C0460B
:109DF800F39E0008F39E0008F39E0008F39E0008F7
:109E0800F39E0008F39E0008F39E0008F39E0008E6
:109E18007D9E0008F39E0008F39E0008F39E00084C
:109E2800F39E0008F39E0008F39E0008F39E0008C6
:109E3800999E0008F39E0008F39E0008F39E000810
:109E4800F39E0008F39E0008F39E0008F39E0008A6
:109E5800859E0008F39E0008F39E0008F39E000804
:109E6800F39E0008F39E0008F39E0008F39E000886
:109E78008F9E000830492F48086045E02E497D2014
:109E88000002086040E02C490120C00308603BE064
:109E98002648016803221140039100687021084098
:109EA8000009401C02900398032805D10299214813
:109EB80001F0FAFB059004E002991D4801F0F4FB5B
:109EC8000590059A194801687F231B021940090A61
:109ED800514305910068400F401C0490059804996F
:109EE80001F0E2FB144908600EE0144800680721FD
:109EF800C9020840C10A01208840019001990C4814
:109F080001F0D2FB0C490860074800680F210902DC
:109F1800084081090A4840580690069A0649086888
:109F2800D040086007B000BD081002400C10024085
:109F38000024F40000127A0098000020001002406B
:049F4800FCC700084A
:109F4C0010B58EB00D9000200C900B900A900990DB
:109F5C0008900D9800681F49884238D11E48026845
:109F6C00012189030A4302600068084007900798A2
:109F7C001A48026802210A430260006808400690F1
:109F8C0006984020089002200190099001200A9028
:109F9C00002004900B900C901148029008A903919A
:109FAC00F7F7BCFC019B02980399049A802408944F
:109FBC0009930A920B920C92F7F7B0FC049A1B20AF
:109FCC000590114603F073FE059802F029FE0EB0C1
:109FDC0010BDC04600380140401002403410024011
:049FEC00000400501D
:109FF0000649086E4042E12213014343D817292243
:10A00000D2008B50891848607047C046A0000020DD
:10A01000F0B595B07E48416800680843002809D132
:10A020007C484D21890041587B48484378490022AB
:10A030004A6008607948416800680843002809D1EF
:10A0400074482721C9004158734848437349002286
:10A050004A6008606F48E4214058002815D46D48D4
:10A0600009907221415A1491E421415814984843AF
:10A07000642101F0F5FA09995F229200885070205E
:10A080000B5E8858C01A885005E06249F0200858D5
:10A090005F22920088505F4D08955F20800029580C
:10A0A000C81712911390D8202958C81710911190F1
:10A0B00012981399109A119B01F0BAFA7D22D200DE
:10A0C0000023079301F018FB079B0F910E90286E59
:10A0D0000D930C900C980D99E122120101F0A8FA51
:10A0E0000B910A900F9C0E9E17200201A918486838
:10A0F000AB589B196041AB5048600F9F0E982923C5
:10A10000DE00AC196368AD592D1808987B41855164
:10A110006360496883580B980A9AD21A884107DA13
:10A120000B980A9B3B49172212018B5089184860F3
:10A1300038492920C200881840688A580021521ED8
:10A14000884106DB33492920C20000208850891845
:10A150004860304906912920C2008858891849680A
:10A16000E122120104920023059301F0C5FA049A3A
:10A17000059B06995B24A400085117200401085987
:10A180000919496801F0B8FA014606982F22D20051
:10A1900081502121C9004058002823D51D48039033
:10A1A000C8300290006C4442E317194948680A68B5
:10A1B000121958410A60486008684968164A002325
:10A1C00001F0B2FA039902460298C266426E7D20FF
:10A1D000C0005043C96D01F06BFA03994F22920001
:10A1E000885213E00B48C8300190046CE3170B4908
:10A1F00048680A68121958410A6048600868496846
:10A20000054A002301F090FA0199086715B0F0BDE6
:10A2100018060020A000002080EE36002006002056
:10A2200000B581B00D485B2189004058002805D455
:10A230000A485B2189004058009005E007485B21EF
:10A2400089004058404200900098044911221201B0
:10A25000885000F005F801B000BDC046A000002005
:10A2600000B587B0002005907D20C00004901D48F7
:10A27000432189004058002805D51A49452082000D
:10A28000194888522BE01749432080000858039052
:10A290000398C96D884206D31249452082007D206B
:10A2A000C00088521BE00F48C06D002805D10D4941
:10A2B000452082000C48885211E003987D21CA0095
:10A2C00000230193194601F0B3F9019B054A02925C
:10A2D000D26D01F029FA029945229200885207B006
:0CA2E00000BDC046A0000020FFFF0000F1
:10A2EC0000B589B01848006E0023009307930690C0
:10A2FC0006980799E122120101F094F902460098A0
:10A30C0001920A46019905920491039002900599D5
:10A31C0004980843002810D00B49172002018858D4
:10A32C0089184968094A002301F07CF9049A059BB5
:10A33C0001F0DCF90391029002E0002003900290FE
:10A34C00029809B000BDC046A0000020A086010004
:10A35C0000B58DB000200B9031480A9031485B213C
:10A36C0089004058002806D52E485B2189004058AA
:10A37C004042059001E0002005900599C81708910E
:10A38C000990002007900690264811210901405899
:10A39C00002815DC08980999214A0492002303939C
:10A3AC0001F040F9039B1F4A126E01F09FF903461E
:10A3BC0003980A460499C91A90410691079016E031
:10A3CC0008980999164A02920023019301F02AF980
:10A3DC00144A11231B01D258D31701F087F90346F5
:10A3EC0001980A460299C91A90410691079007985C
:10A3FC00069A00210C4BD21A884104DB00200790EE
:10A40C000748069008E00799069A002052428841B6
:10A41C0002DB00200790069006980DB000BDC046E8
:0CA42C00A0860100A0000020A186010015
:10A4380000B58FB000200D9039490C910B90394828
:10A44800112109014058002809DC3649C86D2D2220
:10A45800D200895840180021099108900AE0314932
:10A468004320800008582D22D20089584118C81767
:10A47800089109902B490846C830029000690322C8
:10A48800D201895A4018C10F41184810C9170791BD
:10A49800069008980999069A079B01F0C5F87D224D
:10A4A800D200002301F024F90246029803920A46DA
:10A4B800039905920491806C01280EDB0498059994
:10A4C800174A002301F0B0F8164A11231B01D2588D
:10A4D800D31701F00DF90B900CE004980599104A78
:10A4E8000023019301F0A0F8019B0E4A126E01F0BF
:10A4F800FFF80B900B9AD01700210B4BD21A88410A
:10A5080002DB07480B9007E00B9AD1170020524254
:10A51800884101DB00200B900B980FB000BDC046AE
:0CA52800A0860100A0000020A186010018
:10A5340010B586B013480190006E00230093059374
:10A54400049004980599E122120101F06FF8024683
:10A5540000980B46019903930292039A029C1723D5
:10A564001B01CC50CB185A602922D20088508A187B
:10A5740050605B229200885009225201885006B034
:08A5840010BDC046A00000203C
:10A58C00C20F490089184000034A40428A4101D356
:0CA59C0000207047012070470000E0FF25
:10A5A8000122D2079143034A4A401043414248419D
:08A5B8007047C0460000F07F6F
:10A5C000074A0A40531E9A41C00F4900081805491E
:10A5D000884201D3002000E0012010407047C046AF
:08A5E0000000F07F0000E0FF25
:10A5E80030B50E4B5D1C0C0D2C4010D0AC420ED07B
:10A5F800A2189A4205DD0120C00701400948091840
:10A6080009E0002A04DD064B19401205114330BD4C
:10A618000120C0070140002030BDC046FE070000F1
:08A62800FFFF0F800000F07F2E
:10A6300010B54B005B0D084CA34201D0002B02D19A
:10A640000023136010BD054C1B191360044A114010
:10A65000044A891810BDC046FF07000002FCFFFF36
:08A66000FFFF0F800000E03F46
:10A66800F0B587B00E4604460021C843574F069000
:10A67800401C0590384601914841590004914D0D00
:10A68800534900D18CE0E50F7100029149190391FB
:10A69800650006994D1B03998F4100D282E0D10FC6
:10A6A800049D69185500059F7D1B88417AD30121B7
:10A6B800C807304004904748354605400340101B02
:10A6C8001846A84171D2039109050298470D0591D2
:10A6D80003D0481E06400E430DE08D420AD203986F
:10A6E800C004E10F6E00761864007F1E854235466F
:10A6F800F7D300E02E461D0D3748054004D00599D4
:10A70800481E03400B430FE0059883420CD2039880
:10A71800C00406901946D30F4800C31852006D1E96
:10A72800069881421946F6D3AF4212DDA01A314687
:10A73800994104D454405E40264302D113E0204698
:10A748003146C40F49000E1944007F1EAF42EDDCAC
:10A758002F462046841A35469D41059906D4504017
:10A768005E40064304D1019C049916E00446354630
:10A778000D420AD10398C004E10F6A005118640021
:10A788007F1E05420D46F7D000E02946002F15DD53
:10A79800781E049A891800050918204607B0F0BDEC
:10A7A800019CFAE7019C0A49F7E762405D401543BE
:10A7B80000D00496002DD7D10024D5E70398C21BFA
:10A7C800204600F011FF04460020E2E7FFFFDFFF0C
:0CA7D8000000F87FFFFFFF7FFF0700007C
:10A7E400F0B583B00D46044628494A1C280D104094
:10A7F400421E8A4240D22749884205D20024002DB5
:10A80400264635DA264E33E03331884201D92E46C6
:10A814002EE01F49461820462946324600F0D6FE4F
:10A824001D4A114001434A424A410020002D01DAE9
:10A83400014600E00121114302911849019032467A
:10A8440000F0E4FE074632460E462E402740019BA8
:10A85400D843401C1049594100F0C8FE029A3818E8
:10A864007141002A00D10E46002A00D107463C4619
:10A874002046314603B0F0BD002802D10121C907AA
:10A884000D402E460028F3D10024F1E7FE07000016
:10A8940001FCFFFFFF030000FFFF0F000000F0FFBB
:04A8A4000000F0BF01
:10A8A800F0B587B00A0D521E484B9A4214D206AA38
:10A8B800FFF7BAFE06460F464948301A4748814115
:10A8C800069C3046394618DA0022474B00F0E4FA75
:10A8D80006460F46641E14E0C30F4A00D31844000E
:10A8E80064423B4C9C416AD3520D6CD000290A4605
:10A8F80000DA394A002963DA66E00022394B00F0B1
:10A90800CBFA059403900D460024E24304943046A4
:10A918003946FFF765FE354B002200F0BDFA0246C6
:10A928000B460398294600F049FC03900F4602465F
:10A938000B4602F028FF04460D462D4E02213046F4
:10A9480022462B4603F093FC2A4A2B4B00F0A4FA2C
:10A958000290019110360321304622462B4603F01F
:10A96800AEFC02460B460298019900F027FC2246ED
:10A978002B4602F008FF039C22463B4602F003FFE9
:10A9880022463B4600F088FA06460F46059800F036
:10A99800B5FD04460D46194A194B02F0F4FE32463D
:10A9A8003B4600F079FA06460F46164B20462946E4
:10A9B800049A02F0E8FE32463B4600F06DFA0A4679
:10A9C800114607B0F0BD034A0020F9E7FE07000072
:10A9D8000000E0FF0000F0FF0000F87F9EA0E63FC7
:10A9E800CE3B7F660000F0BF0000E0BF0000E03F04
:10A9F800C00000089AB5B312FF0750C0A80C615CEC
:08AA080010D02BBF0030E63F27
:10AA1000F0B585B00C4607465948411C220D0A4046
:10AA2000511E814200D38EE05948C01B5748A041B7
:10AA300000DAA2E000205849C91B5649A14101464D
:10AA40007FD30120C007214681435648381A544815
:10AA5000814174D3544A554B3846214602F097FE43
:10AA60000122D2072240524BD31800252A460495D2
:10AA700000F016FA00F0A4FC039000F043FD0290F1
:10AA80000E464C4B002202F082FE3A46234600F06E
:10AA900007FA04460F46484A484B0298314602F0EE
:10AAA00076FE22463B4600F0FBF906460D4602467E
:10AAB0000B4602F06CFE0F46414A424B04460290A0
:10AAC00002F065FE404A414B00F0EAF922463B465F
:10AAD00002F05DFE3E4B049C224600F0E1F9324656
:10AAE0002B4602F054FE05460E46204630492A46C3
:10AAF000334600F0B9FA01900091364A364B029C79
:10AB00002046394602F043FE344A354B00F0C8F97E
:10AB100022463B4602F03BFE019A009B00F0C0F942
:10AB200002460B462846314600F04CFB049A204B67
:10AB300000F0B6F9039A521CFFF756FD01E01749E1
:10AB4000002005B0F0BDF80F6100081879004942F7
:10AB50000C49814121460ED30120C00781430A4898
:10AB60004840384300D075E7002C214600DA002128
:10AB7000002C00DA00273846E3E70349E0E7C04647
:10AB8000FE0700000000E0FF0000F07F422E86403C
:10AB9000EF39FAFE2B2386C0D2BC7ADD0000F03FED
:10ABA000A19CC73B2342920C3CF92F9E2C15F73FEA
:10ABB0000000E03F0030E6BFA80C615C10D02B3FE6
:10ABC0001CDC586FA452F13EE0F6B36FE4707C3F9A
:10ABD0000000D03F0938DE6F993F403FB3514271CA
:04ABE0008E71AC3F87
:10ABE400F0B585B016460024E7438B4D7A1C2A46FF
:10ABF40062414A4002436FD001955A00550D00D17D
:10AC040008E100940290874C601C039104930D0D9D
:10AC140005406D1EA54273D21D461C0D0440824B97
:10AC2400E4185B1C9C426BD337463046294600F03F
:10AC3400C5FB064600F064FC2A46029D784051405C
:10AC44000143039C30D101200290C00786422BD0DF
:10AC5400002E0096714B41D0F0174640361A00275B
:10AC640001970393012E019A00D02A460497012EDE
:10AC74006A4B00D023462F462846214602F085FD24
:10AC8400224605460C46304602990840634B00D0E4
:10AC9400134642423A400498039902F076FD07466F
:10ACA4000B467608DDD11AE00022284621461346D9
:10ACB40000F064FB002802D0604900241DE001205C
:10ACC400C007844328462146FFF7ECFD3A46049B1F
:10ACD40002F05BFDFFF79AFE04460EE00027002019
:10ACE4004E493A461D4600F06BFA04460098002887
:10ACF40000D42946002800D43C46204605B0F0BDC7
:10AD04000298C30F4C00E3184400641E484C5C4195
:10AD1400E2D20125F30FD21873005B1B434B9A4117
:10AD240010D23F4A114210D0424B0C465C400443BF
:10AD340026D00C4654400443049827D100283CDA1A
:10AD44002146DAE734460499D7E737463046049C6F
:10AD5400214600F033FB064600F0D2FB4C403B4654
:10AD64004340234327D1049900291C46194600DA9D
:10AD74002B49F007C1D0E807039E06407118BCE7D1
:10AD84000094049800281ADA009819E05840064301
:10AD940002982CD1284A4A400243009C1F49ACD057
:10ADA400EA07039B93430022391A019898411446F9
:10ADB4002ED31B4A2CE0049A3FE711469DE7104628
:10ADC40003903046049F394600F0F8FA044600F038
:10ADD40097FB794070400843039802D1E807039930
:10ADE4000818E10700D00390009C039985E7EB075E
:10ADF4000C469C430023391A0198A0411C4619466D
:10AE040000D37AE70C48039E46400298304301D0B1
:10AE1400114672E7014970E7FFFFEF3F0000F03F82
:10AE24000000F07FFE07000001F8FFFF0000E0FFD4
:10AE3400FFFF1F000000F0FF0000F0BF0000F87FDC
:10AE4400F0B581B000280090124D13D00146C01710
:10AE540041400F1A0026104CF80707D00CCC30469E
:10AE64002946083C02F091FC06460D4608347F084A
:10AE7400F2D100E000260020064932462B4600F0BD
:10AE84009FF9009A002A00D43046002A00D42946AB
:0CAE940001B0F0BD0000F03FE800000835
:10AEA000F0B40125ED070F005F405AD48B4200D16A
:10AEB000824205D950404240504059404B40594091
:10AEC0004E18760DDF187F0D3BD0741C640529D019
:10AED000F41B352C26D80E0DDB022B43DB0AC902EE
:10AEE0002943C9121700202C1ED2E741E2405740E7
:10AEF000E3415A40A340E3405A400024801859419E
:10AF00000AD3B21C520521D0C207012F624117009B
:10AF10004008CB0718434908013636054208AF41BF
:10AF200060417141F0BC7047203C06D01F00E741F2
:10AF3000E3405F400024012A6741C0186141EBD320
:10AF4000DFE7002EEED129400020EBE70136310586
:10AF50000020E7E7E742E5D10020C143090DC9041D
:10AF6000E0E76B400E00871A9E4104D26E40C01B82
:10AF7000B141D21973414E18DF18AC0AE642E9D24A
:10AF8000760D7F0D31D0F41B362CCBD8B4460E0D88
:10AF9000DB022B43DB0AC9022943C90A012C32D840
:10AFA00004D1D4075208DF073A435B08EF0A644232
:10AFB000904199411ED0002239424DD1241940417F
:10AFC00049410124394204D1013400184941394230
:10AFD000FAD06246A24204D9361B013E36058919D1
:10AFE000A0E7F10AC90700209CE736429AD1002069
:10AFF000002197E70200224394D0B842DED201003C
:10B0000020002024E3D1202C13DD203CE241170056
:10B01000A240E2405740E3415A40A340E3405A4037
:10B02000012FBF410137174300227C4298419141D3
:10B030000CE01700E741E2405740E3415A40A3408B
:10B04000E3405A407C429041994100220F0303D2D1
:10B05000013E241940414941013E36054708AC41B3
:08B0600050417141F0BC704742
:10B06800F0B40125ED076B40004C2047A7AE00085F
:10B0780030B405004D400124E407254042004B0050
:10B08800120E32D01B0E3CD0FF2A33D0FF2B3FD0FC
:10B09800D21800022043000A09022143090AC4B257
:10B0A8004C43000AC3B24B43000A4843210A5B18C9
:10B0B800190A091801D44900013A080A7F3A2ADB1B
:10B0C800FE2A0FD2D2051C43240601D001242143B5
:10B0D800C9B280295041802901D140084000284345
:10B0E80030BC7047FF20C005F9E71B0EFF2B0AD0C4
:10B0F8002800F5E7400206D1FF2BF3D1490202D11F
:10B10800F0E7FF2AF4D17F2000010C300005E7E7C3
:10B118004902F8D1E6E743020132E9D15B12023372
:08B12800E6D9D805E4E7C046B2
:10B1300030B405004D400124E407254042004B0097
:10B14000120E26D01B0E34D0FF2A2DD0FF2B35D067
:10B15000D21A000220430902214343084908A00DE6
:10B160005B1A02D2013A5B005B185B008B4200D392
:10B170005B1A4041F9D37F3222DDFF2A06D2D20585
:10B18000C91A8B425041284330BC7047FF20C0058C
:10B19000F9E71B0E03D0FF2B12D1490210D07F20FC
:10B1A00000010C300005EFE74002F8D1FF2BEDD194
:10B1B000F5E7FF2AEAD14002F1D1E7E74902EED1F3
:04B1C0002800E1E79B
:10B1C400F0B40125ED070C005C402C40A446AE0A07
:10B1D4004C18DF18F4423DD2F74245D2640D4CD0EE
:10B1E4007F0D3CD0E41BC9022943CF0ADB022B4369
:10B1F400DB0A0600B61A9F4104D2013CB6197F410E
:10B20400B6185F416812800D241838DD0018844296
:10B2140025D8E80C0021B6197F41B61A9F4103D303
:10B2240040414941F7D304E0B6185F410018494151
:10B23400F1D32405B6197F41B61A9F4105D337438C
:10B24400C20717430022012F504161416246114356
:10B25400F0BC70470CD100280AD1F74208D2002074
:10B26400C143490D0905F1E7002A01D1F74206D08F
:10B274000020C143090DC904EAE77F0DF8D000207E
:04B284006146E5E753
:10B2880030B401256D054C00E54215D85C00E54257
:10B2980012D80C001C436400044314430FD005D299
:10B2A80082428B418041013030BC704790429941C5
:10B2B8008041013030BC7047002030BC704701200D
:04B2C80030BC7047DF
:10B2CC0070B4012676054C005D00E6420CD8EE42C7
:10B2DC000AD825430543154303D0994204D1904223
:10B2EC0002D1012070BC7047002070BC7047C04672
:10B2FC0030B401256D054C00E54215D85C00E542E3
:10B30C0012D80C001C436400044314430FD005D224
:10B31C00904299418041013030BC704782428B4150
:10B32C008041013030BC7047002030BC7047012098
:04B33C0030BC70476A
:10B3400030B401256D054C00E54215D85C00E5429E
:10B3500012D80C001C436400044314430CD005D2E3
:10B3600082428B418041404230BC704790429941BB
:10B370008041404230BC7047002030BC7047C0461E
:10B3800030B401256D054C00E54215D85C00E5425E
:10B3900012D80C001C436400044314430CD005D2A3
:10B3A000904299418041404230BC704782428B417B
:10B3B0008041404230BC7047002030BC7047C046DE
:10B3C000F4464A1805D200F063F801D5C0174008CA
:10B3D000604701235B05D34206D200F059F801D53E
:10B3E0000120C0074042604701D10042F5D0D0178C
:04B3F000400870475A
:10B3F4004A00520D01239B02D21A01321DD452423B
:10B404003F321DDD8C46C902430D1943C00201239E
:10B41400DB071943202A02D308000021203AD14136
:10B42400D04048409140D140484063461B4203D538
:10B43400002340428B4119007047002000217047CF
:10B44400002801D0012211434B0001225205D342AE
:10B4540000D959080020C90FC90701D4C0434108C5
:04B464007047C04627
:10B4680041000DD2090E7F390AD449421F3105D453
:10B4780000020122D2071043C8407047C81770471E
:04B4880000207047E9
:10B48C004A0010D2520D03231B02FF33D21A0AD4E6
:10B49C0052421F3209D4400DC90208430123DB0775
:10B4AC001843D040704700207047D0177047C046F3
:10B4BC004B001BD25A0D01239B02D21A013215D418
:10B4CC0052423F3215DBC902430D1943C00201231E
:10B4DC00DB071943202A02D308000021203AD1416E
:10B4EC00D04048409140D140484070470020002156
:08B4FC007047D01701007047F2
:10B50400054B004206D5404200B5984708BC0122CD
:0CB51400D2071143184700009DB5000845
:10B520000B00034329D0CA0FD200043212023D326D
:10B53000094203D5002349424042994102D101000A
:10B540000020203A0B0C04D1103A0904030C1943D3
:10B550000004094203D4013A00184941FBD584464E
:10B56000C00A4B051843C90A120563465B055B41D7
:0CB5700002D3012B0023584151417047C9
:10B57C009D2201000AD002D4013A4900FCD5D20523
:10B58C00080A0906494100D3012950417047C046B9
:10B59C0042221201033A010007D002D4013A0018EA
:0CB5AC00FCD51205C30A40059918704731
:10B5B8000B00034305D0042212023D320942014B1D
:08B5C800184770473DB500086B
:10B5D000202A07D203009040914052422032D340AB
:10B5E00019437047203A0100914000207047C0463F
:10B5F000202A07D2D0400B00D14052422032934043
:10B6000018437047203A0800D04000217047C046D8
:10B61000202A07D2D0400B001141524220329340E1
:10B6200018437047203A08001041C9177047C046B8
:10B6300030B5514343435C18010C130C0D005D43BE
:10B64000641992B2514380B242430D0C090452185E
:10B6500065415843010C00048018694130BDC04663
:10B66000CA1751408B1A17D0C1174A409446484018
:10B67000411A48081A0000E052008242FCD900201A
:10B6800000E05208914200D3891A40419A42F8D111
:10B6900062465040801A704710B500F095F810BD12
:10B6A00007B5FFF7DDFF0EBC4243891A00BDC04657
:10B6B0000A0015D00300400800E052008242FCD985
:10B6C000002000E052089B1A06D340418A42F9D17B
:10B6D000704752089B18F8D200188A42F9D1704777
:08B6E00010B500F071F810BD77
:10B6E80038B504004D42FFF7DFFF4543611938BD07
:10B6F80070B5CC1760406140001BA141DD176A405E
:10B708006B40521BAB4100F00BF862406340121BC8
:10B71800A3416C4060406140001BA14170BDC04620
:10B72800002B09D1002907D110B51100FFF7D8FF68
:10B738000A000021002310BD70B400240125ED0784
:10B74800002B07D1002905D0834203D21300002221
:10B758002C0000250026A419994200D1904212D944
:10B7680092185B4103D2EE076D086408F3E7DE0721
:10B778005B08520892190126F6079B1903E0DE07B9
:10B788005B0852089219801A994103D364416D41AC
:10B79800F5D30FE024196D410AD2DE075B08520881
:10B7A800921980185941F5D364416D41E7D301E0FE
:10B7B8008018594102000B002000290070BC704716
:08B7C800002000217047C0467B
:10B7D000F0B503AF93B06E46F51D2135F41D393435
:10B7E00074613362F261F160306102F0AEFDB0600D
:10B7F000C21D07218A436946B1616946881A706093
:10B800008546F41D1D3400212422204600F0CAFF85
:10B810000B487169F2680A6048600A48286030691C
:10B820002862B06868617068E8602046F169326A31
:10B8300000F01EF8B1698D46FE1F053EB546F0BD0D
:08B840003BE30008FFFFFF7F5E
:10B8480083B010B581B0044603A80EC0054800684F
:10B8580003AA0092214602F09CF801B010BC02BC79
:08B8680003B008478C0000202A
:10B87000F0B59FB012920B460446002020600121D3
:10B880000A020F924A020B928A020192CA020092A5
:10B8900003220D92920205920D034A0307928A0336
:10B8A00003920491C90317910A90C0430290169421
:10B8B00009951978252909D0002901D100F03CFE0D
:10B8C0005C1C169802F00CF82346F2E7DB1C0A9F7A
:10B8D0000B9C981E00780246203A102A2CD8802112
:10B8E00092003E461F4602A39A583B46374697466B
:10B8F00035B9000855B9000855B900084FB9000816
:10B9000055B9000855B9000855B9000849B90008EB
:10B9100055B9000855B9000879B900084DB90008B3
:10B9200055B9000841B9000855B9000855B90008D3
:10B9300045B9000840210AE05E28294607D009E001
:10B94000102104E0214602E0179900E020210F4376
:10B950005B1CBEE75B1E014630390024092916D85E
:10B960000A2161434418303C591C18780246303A89
:10B970000A2A0B46F4D30AE0129901C91291C10FA9
:10B9800009010F43C1174840441A581E0078002689
:10B990002E281CD118782A2805D158789B1C12997A
:10B9A00040C912910FE05B1C0146303909290CD8BF
:10B9B0000A2171434618303E591C18780246303A25
:10B9C0000A2A0B46F4D3002E01D40F990F43E11736
:10B9D0006B2808DC4C2803D068283CD06A280AD1A0
:10B9E0000220074305E06C2830D07A2801D0742863
:10B9F00001D118785B1C8C43462811931BDD01464E
:10BA00006339152937D8C0467944097949008F44EC
:10BA1000710B4D1BD70A0B0A0A0A0A8194610A0AA4
:10BA20008F0A560A0A3A44E70C94039C27430021E4
:10BA3000089139468EE0442815DD452834D0462843
:10BA400000D036E7079807430098BAE018786C28CA
:10BA50002ED1022003E0187868282CD10820074353
:10BA600058789B1CC7E7252800D08EE22521169820
:10BA700001F036FF7AE2472800D19FE0582800D035
:10BA800017E707990F430C94D34A782800D1203246
:10BA9000039C0F990F42394601D0D04B19403B0609
:10BAA000DB171340089355E007980743019888E097
:10BAB0005B1C049A01E05B1C042217439BE70C9477
:10BAC0000F990F4201D0C5490F403946039C00220F
:10BAD00008923FE00C9438060F990F430E97C01759
:10BAE000232101400891129820C8129000240820B8
:10BAF0000690D3E1129E3578621E169C2046394688
:10BB0000159201F03FFF2046294601F0E9FE361D5F
:10BB10001296C2E01298006839071699096800D594
:10BB200037E2BA07016000D434E20021416031E21B
:10BB30001596129901C912918EE00C940F990F423B
:10BB4000394601D0A54A11403A06D2173023134096
:10BB50000893039C02220A40214205D1002A129A2E
:10BB600008D1131D00240BE0002A129B13D104CB33
:10BB7000D41715E0D21D07239A435468134608339F
:10BB8000129315684A0713D408220A4000D0EDB278
:10BB9000002A0ED102E1DB1D0722934314CB0033B0
:10BBA00012934B0707D40B0700D5E3E01546E4E0FA
:10BBB000ADB20024F2E015B21204DDE007980743AD
:10BBC000059807430F98074201D0304600E0062051
:10BBD0000C943946059A1140891A4A424A41002874
:10BBE00000D002461592129CE41D0720844326686B
:10BBF000656830462946FEF7D7FC083412940028C1
:10BC0000304629460ED000221346FFF7B9FB3A46CC
:10BC100007990A4000280C9C0FD0002A704819D0C0
:10BC2000704817E0FEF7B2FC00280C9C37D007984C
:10BC300007426D480ED06D480CE0002A6C4900D0D8
:10BC40006C49002A01D06B4800E06948401CBA06E4
:10BC500000D5084668490F400028684E00D00646C7
:10BC60000F980742304602D100F016FD02E0159908
:10BC700000F04AFD054659480740621B16983946B0
:10BC8000159201F07FFE002D07D0169C31782046DA
:10BC900001F026FE761C6D1EF8D1F8065DE13046F7
:10BCA0002946FEF78DFC002800D10646002800D169
:10BCB000002513963046294602F0DBFA044601209F
:10BCC000002C089001D0C00745401EAA30461095B0
:10BCD0002946FEF7ADFC1E980D9948430A21FFF74F
:10BCE000BFFC06461E90002C01D0602007430022B6
:10BCF000139C2046294614921346FFF7E7FA0028C2
:10BD000018D1701CFFF79EF822462B46FFF738FB30
:10BD100000281E9806D0411C1E91801CF2E71E9838
:10BD2000401E1E90FFF78EF822462B46FFF708FBB9
:10BD30000028F4D13D4605980540089883021E98D6
:10BD40009D42159E00D113E105998D4207D186428F
:10BD500000DC0DE10421C943884200DC08E10199BF
:10BD60000F42109D0E9300D180E20E2800DCD0E13E
:10BD7000149E7BE255B21206D417002C05D48A0615
:10BD80000AD44A060AD5202207E000226D42A241C9
:10BD90002D230893144601E02B2208920F9A11429A
:10BDA00001D00E4A11400A460F990E920A42049998
:10BDB00000D03146069100276E2838DD6F380928FB
:10BDC00000D98AE078440079400087441967868664
:10BDD000868636868667C04658300000FFFDFFFF26
:10BDE00074E900086FE90008D3EB0008CFEB000806
:10BDF0007EE9000879E90008FFFEFFFF05E500087D
:10BE00002846204369D0E80861074018014607200A
:10BE10002840303018AAD055C808E40862078018B6
:10BE20000A4622437F1C002A0D46EFD155E05828D0
:10BE300034D0642801D069284FD1284620434CD003
:10BE400011461798014010912A461098002808D0F2
:10BE500038460D990840032803D118A82C21C15554
:10BE60007F1C002510462146159414460A222B46B5
:10BE7000FFF75AFC149013910A222B46FFF7D8FBC8
:10BE8000201A3021014318A8C1557F1C0920001B2E
:10BE900015988541149D139CD6D31EE02846204357
:10BEA0001AD007980E990142C04800D0C04829090D
:10BEB0002207891800270A460F212940415C18AB48
:10BEC000D955110924092307C918134623437F1C98
:10BED000002B1546EFD100E00027089DFF2D01D86B
:10BEE000029801E0B348FF300B9C0C9B0699CE1BD7
:10BEF000F1178E43B9195A1A002D00D012180E9955
:10BF0000214203D1169801F03DFD00221592290A25
:10BF1000169C03D0204601F0E3FC01E0002D03D085
:10BF20002046294601F0DCFC20460E99159A01F0C6
:10BF300029FD30212046324602F0F1F9012F0ADBBB
:10BF40007D1C18A84019801E0178204601F0C8FC0D
:10BF50006D1E012DF5D80E98C006099D119B00D4C9
:10BF6000A7E420211698159A02F0D9F9119BA0E4B4
:10BF70000F9934318842109C06950FD113982146B1
:10BF80008D4A8E4BFFF71EF90FE0002800D090E499
:10BF9000E2E201701298001D12908AE44042FEF71E
:10BFA00051FF139A234601F0F2FB04460E4600228D
:10BFB0001346FFF78BF9002839D120463146FEF7AA
:10BFC000F3FA00282046314600D01CE60E970022E6
:10BFD0007B4BFFF793F900281E9F0FD000222046CD
:10BFE0003146774BFFF7EEF804460E460022744BBD
:10BFF000FFF784F97F1C0028F0D11E97002220460D
:10C000003146704BFFF7BCF9002811D000222046C2
:10C0100031466B4B01F0BBFB04460E460022694BD8
:10C02000FFF7AEF97F1E0028F0D11E9700E00E97B3
:10C03000059806998142159801D0014600E0411EFD
:10C04000029D0028149100D1002113914842FEF76F
:10C05000F9FE2A46FEF7C8FA22463346FEF720FFCD
:10C0600006460D4600220692554C2346FFF746F938
:10C0700000280AD01E98401C1E90002230462946F7
:10C080002346FFF79FF806460D4610961595139820
:10C09000002866D000990B4680330E9A13408B42DD
:10C0A00061D1102800DB10200546FEF7CBFE32469A
:10C0B000159B01F06CFBFFF701FA0C46014621438A
:10C0C000069914914FD0214606463F4A3F4BFFF751
:10C0D000AFFA4A08C3079A184008C90708183C492C
:10C0E000081A3C48904114953DD330460A2200235B
:10C0F0002146FFF719FB0C4607460A220023FFF7EB
:10C1000013FB1498401E14902DD01A433846EDD0DE
:10C1100029E0C143711810290E4600DB10263A06AB
:10C1200000D5A3E0002900D1A0E03046FEF78AFE4A
:10C13000139A2B4601F02BFB00242246264BFEF7D8
:10C14000AFFEFEF74FFB22461D4BFEF78DFA22464F
:10C150002346FFF7BBF8002800D184E0761EE4D127
:10C1600082E00698149080210E9806460140149AA9
:10C1700011430C98801A002901D1401F00E0801F54
:10C18000139009981E9C064201D1089D46E00321A8
:10C190002046FFF785FA881C0125C04678440079BF
:10C1A000400087441B2A381B2A00C046BFEB00080A
:10C1B000AFEB0008FFFEFFFFA0C8EB85F3CCE17FEB
:10C1C000000024400000F03FCDCCCCCCCCCCCCCC7B
:10C1D00099999999999999190000E03F641E1E94C4
:10C1E000002210981599DF4B01F0D1FA10901591AB
:10C1F0001398401E139002250DE0A41E1E940022E9
:10C2000010981599D84B01F0C2FA10901591139817
:10C21000801E13900325149AD01782437006800F56
:10C22000149202D01398401E1390204602F073F827
:10C23000632802DD1398401E13900898C002374609
:10C24000874310981599FFF739F906460C46FFF712
:10C25000B3F902460B4610981599FEF705FF1090AA
:10C260001591139A76E034461E9826461038149697
:10C270007142884200DC0846FEF7E4FD029AFEF7B0
:10C28000B3F9139A2B46FEF70BFE05460C461E9893
:10C29000401CFEF7D7FD2A462346FEF7F5FF00288F
:10C2A0001E9800D0401C002814D4112818D3014631
:10C2B00010391E911021081AFEF7C4FD2A462346A4
:10C2C00001F065FAFFF7FAF806460C4600201590D3
:10C2D000109018E01095159400261E96344612E032
:10C2E00000201E9028462146FFF7E8F806461594E0
:10C2F0000C46FFF761F902460B4628461599FEF7F2
:10C30000B3FE1090159138460E998843974908312D
:10C3100000250A4608326D1C0B684968F31A23464B
:10C320008B411146F6D280213940149A11434B1E9D
:10C330000A469A41002901D00021C9437B069B0F80
:10C3400000D0D1431E9A891A0C9A149BD21A511804
:10C350004A1B0746D017114681430B9810300E97A1
:10C3600007420AD1012A08DB0F462021169801F066
:10C37000B7FA7F1EF9D10E9A01E03A460F464020E7
:10C380001040910603D4002809D0202104E00028A1
:10C3900001D02D2100E02B21169801F0A1FA0E9872
:10C3A000C00607D4002F05D03021169801F098FA66
:10C3B0007F1EF9D16D1EE8006C4A111849681258A9
:10C3C000B01A2046884101D2302007E03020B61A4A
:10C3D0008C41401CB31A23468B41F8D2C1B2169847
:10C3E00001F07EFA002DE5D113970E9E3446009899
:10C3F0000440169F0BD01E98012808DB401E1E909B
:10C400003021384601F06CFA1E980028F6DC8020B6
:10C4100030401499084344D02E21384601F060FA88
:10C42000149D102D00DB1025E8178543002C01D149
:10C43000284601E01E98281A159CFEF703FD149A61
:10C44000012A22DB109A234601F0A1F9FFF736F802
:10C4500004460E462F467F1EF800444A11184968CC
:10C460001258A01A3046884101D2302007E030200F
:10C47000A41A8E41401CA31A33468B41F8D2C1B294
:10C48000169801F02DFA002FE5D11499481B169F3C
:10C490000E9E06D06C1A3021384601F021FA641C39
:10C4A000F9D301980642099D139F38D00798064298
:10C4B00001D0452100E06521169E304601F010FABA
:10C4C0001E980028304604D42B2101F009FA1E984A
:10C4D00005E02D2101F004FA1E9840421E906428C8
:10C4E0000DDB6421FFF7E4F801463031304601F0FE
:10C4F000F7F91E986421FFF7D3F808461E910A2128
:10C50000FFF7AEF801463031304601F0E9F91E98E8
:10C510000A21FFF7C5F83031304601F0E1F9002F6C
:10C52000119B01D1FFF7C5F9169C2021204601F08F
:10C53000D7F97F1EF9D119E5169CE068002805D0CF
:10C5400006CC083C914201D20A9A4254204601F09E
:10C550000CFA20681FB0F0BD169801F006FA029898
:10C56000F8E7C046000024400000594030010008B0
:10C5700009490968091A4A1E9141084A1268121AA3
:10C58000531E9A410A4006490968081A411E88410B
:10C59000104040427047C0468C00002090000020B0
:04C5A00094000020E3
:10C5A4000F480321016141610E4A82610E49C16154
:10C5B400012189020162002181624162C162026635
:10C5C4000A4A4266102282660167C1664167084AC8
:10C5D4000F234B40D35C4354491C1029F8D17047B6
:10C5E4006C0A002094E9000842100020C2140020C4
:04C5F40083E90008CF
:10C5F800F0B581B00D461821414316484618F06A37
:10C60800183602281ED0144601280ED0002700280C
:10C618001DD1304601F0CFF9A04218D33046294643
:10C62800224601F0D3F9274611E0304601F0C3F95C
:10C638000746A04200D32746304629463A4601F02D
:10C64800C5F904E03046294601F0DDF907463846C9
:08C6580001B0F0BD6C0A0020E6
:10C66000F0B581B014460D4606460A480078002809
:10C6700001D1FFF797FFEFF31087012181F31088B5
:10C68000304629462246FFF7B7FF87F3108801B0EE
:08C69000F0BDC0466C0A002059
:10C69800F0B581B00178002925D003220146009227
:10C6A80091430D680023DC438607F60EB440E4434B
:10C6B8002C43114D6719A743104A174206D14C68FD
:10C6C80067191646A643091D3E42F8D022060FD028
:10C6D8002204120E09D02202120E08D0220E009B4C
:10C6E80006D0042304E0002004E0012300E0022334
:10C6F800C918081A01B0F0BDFFFEFEFE80808080D8
:10C70800F0B581B00022002934D00378002B31D055
:10C7180003270246BA430024E5438607F60EB540D0
:10C72800EE431568354306463E40711804290CD37C
:10C738000097134EAF19114BAB433B4204D1091F6D
:10C748005568121D0329F5D8009F2B060DD02B0420
:10C758001B0E07D02B021B0E06D02B0E00D0042771
:10C768003C4602E0012400E002248C4200D30C463F
:10C77800101A0219104601B0F0BDC04680808080B2
:04C78800FFFEFEFEB4
:10C78C00002A03D0013A8B5C8354FBD17047C0461E
:10C79C0000220B0011001A00002A02D0013A815429
:04C7AC00FCD1704705
:10C7B00002480068002800D101487047D00F0020CF
:04C7C00074000020E1
:10C7C4007F2805D8034A125C0348405C1040704738
:0CC7D40000207047D7EB0008FEE90008C9
:10C7E0007F2805D8034A125C0348405C104070471C
:0CC7F00000207047D7EB0008FEE90008AD
:10C7FC00000000000000000000000000000000002D
:10C80C00000000000000000000000000000000001C
:10C81C000100000002000000030000000400000002
:10C82C0006000000070000000800000009000000DE
:10C83C0000000000000000000000000000000000EC
:10C84C0001000000020000000300000004000000D2
:0CC85C0005E8000888C8000868C800084B
:10C86800C5C700085FE300089BDA0008E1C70008B5
:10C878006BE30008A9DA00084FE300086DDA000846
:10C8880007E80008FDE90008FDE90008FDE90008DF
:10C89800FDE90008FDE90008FDE90008FDE90008D8
:10C8A800FDE90008FDE90008FFFFFFFFFFFFFFFFAC
:10C8B800FFFFFFFFFFFF0000CBE70008AFE900081C
:10C8C8000CE50008CCE9000863E500089DE90008CC
:08C8D800A6E900086AE500086A
:10C8E000034C206804348047FBE7FCF7CDF8FEE7F3
:04C8F00058EC0008F8
:10C8F4000448054988438546044880470448054957
:10C904000160EBE7008000200700000055D7000815
:08C9140008ED00E0000000083E
:10C91C00FEE7FEE7FEE7FEE7FEE7FEE7FEE7FEE7E3
:10C92C00FEE7FEE7FEE7FEE7FEE7FEE7FEE7FEE7D3
:10C93C00FEE7FEE7FEE7FEE7FEE7FEE7FEE7FEE7C3
:10C94C00FEE7FEE7FEE7FEE7FEE7FEE7FEE7FEE7B3
:0CC95C00FEE7FEE7FEE7FEE7FEE7FEE771
:04C96800D99D00084D
:10C96C0087B006900591049203A9002008701F203F
:10C97C0002900299481E029000200029019009D0D3
:10C98C00059802991F221140C840012108404142DC
:10C99C00484101900198C007002800D0E9E70498AD
:10C9AC00009018284CD80098810001A04058874668
:10C9BC004BCA00084DCA00084DCA00084DCA0008F1
:10C9CC004DCA00084DCA00084DCA00084DCA0008DF
:10C9DC003DCA00084DCA00084DCA00084DCA0008DF
:10C9EC004DCA00084DCA00084DCA00084DCA0008BF
:10C9FC002FCA00084DCA00084DCA00084DCA0008CD
:10CA0C004DCA00084DCA00084DCA00084DCA00089E
:10CA1C0021CA00080298072802D303A90120087034
:10CA2C0011E00298082802D303A9012008700AE03B
:10CA3C000298102802D303A90120087003E002E039
:10CA4C0003A90120087003A8007800280DD10598CF
:10CA5C00069909684861069800688068182188431F
:10CA6C000499084306990968886003A8007807B000
:02CA7C00704701
:10CA7E0081B000900098806804210840800801B0C1
:02CA8E007047EF
:10CA900084B00390029100200190029800900C282D
:10CAA00032D80098810001A040588746E1CA0008AA
:10CAB00009CB000809CB000809CB0008EBCA000825
:10CAC00009CB000809CB000809CB0008F5CA00080B
:10CAD00009CB000809CB000809CB0008FFCA0008F1
:10CAE00003980068406B01900EE003980068806B2B
:10CAF000019009E003980068C06B019004E003987E
:0ECB00000068006C0190FFE7019804B07047D8
:10CB0E0083B002900191009202984069019A04212B
:10CB1E000A400721914088430099914008430299A9
:06CB2E00486103B07047EE
:10CB340081B000900098806802210840400801B04C
:02CB4400704738
:10CB460081B000900098006807218905084001B06F
:02CB5600704726
:10CB580081B000900098C0680321890208404142D2
:06CB6800484101B07047D6
:10CB6E0000B583B002900298806A0190019801F09E
:06CB7E006BF803B000BDDE
:10CB840000B583B002900298806A01900199886D83
:10CB94004022104388650199C86D04221043C8657A
:0ACBA400019801F052F803B000BD43
:10CBAE0083B00290019100920298806A019A1F212F
:10CBBE000A400F2319469140884300999B0619405D
:0ECBCE00890E914008430299886203B07047B7
:10CBDC0081B00090009880680121C9070843172193
:0ACBEC0088430099886001B070478B
:10CBF60081B000900098B42140587F21084001B0D0
:02CC0600704775
:10CC080081B000900098006903218907084001B0AD
:02CC1800704763
:10CC1A0081B00090009800680F218904084001B093
:02CC2A00704751
:10CC2C0000B581B001466846017000214056F4F70A
:06CC3C0063F901B000BD28
:10CC420000B581B001466846017000214056F4F7F4
:06CC52006CF901B000BD09
:10CC580085B00490039102920020019001980299F6
:10CC6800490888420ED2039801998A008118805A8F
:10CC78000004498840180499096808600198401C14
:10CC88000190EBE702A80078C007002808D00498B4
:10CC980000680090039801998900405A009908801B
:0ACCA80004980068006805B07047AA
:10CCB20000B587B006900591049200200290069973
:10CCC200022048770698016888680122104388602C
:10CCD2000698006A019001281BD0019802281FD0F3
:10CCE2000198032823D100200390039804998842D5
:10CCF2000AD2059803998900405806990968086084
:10CD02000398401C0390F0E70698006800680290C0
:10CD12000DE006980599049A00F0E8FF029006E0FB
:10CD220006980599049AFFF796FF0290FFE7069985
:0ACD320001204877029807B000BD09
:10CD3C0000B587B0059004910392029301A90020DD
:10CD4C00087005982421405C012803D106A9022013
:10CD5C0008705EE00599242201208854059825214D
:10CD6C00405C012848D10599252202208854059958
:10CD7C000020C86305980168086801229043086088
:10CD8C0005980499039A029BF4F724FA0598006B12
:10CD9C00002806D00598016808680E221043086028
:10CDAC000BE0059801680868042290430860059818
:10CDBC00016808680A22104308600598406C0068F6
:10CDCC00C003002806D50598416C086801221202A0
:10CDDC00104308600598006D002806D00598016D79
:10CDEC00086801221202104308600598016808685F
:10CDFC0001221043086009E005998020C863059959
:10CE0C0024220020885401A901200870019806A949
:0ACE1C00087006A8007807B000BDFA
:10CE260084B0009101460098039102A908800398F6
:10CE360000690988084203D001A90120087002E0B0
:0ECE460001A90020087001A8007804B0704710
:0ACE540081B06946088001B0704704
:10CE5E0000B585B00390029101920398029B01994F
:10CE6E0000910321C9020022F5F785FF002808D0A2
:10CE7E000399086E20221043086604A90320087047
:10CE8E0029E00398029B0199009180210022F6F778
:10CE9E0006F8002808D00399086E20221043086671
:10CEAE0004A90320087016E00398029B01990091D3
:10CEBE00032149020022F5F75EFF002808D00399EE
:10CECE00086E20221043086604A90320087002E0B1
:0ECEDE0004A90020087004A8007805B000BD6B
:10CEEC0084B0039002910192029A1F210A40012002
:10CEFC0090400090009B039A106A98431062019A2C
:10CF0C000298084082400399086A1043086204B0F2
:02CF1C0070475C
:10CF1E0000B583B001900198002803D102A9012029
:10CF2E0008703EE001983D21405C002806D1019931
:10CF3E003C2200208854019800F084FF01993D2284
:10CF4E0002208854019901C9F6F7CDF901994822BA
:10CF5E000120885401993E220120885401993F22D4
:10CF6E00885401994022885401994122885401998C
:10CF7E004222885401994322885401994422012067
:10CF8E008854019945228854019946228854019962
:10CF9E004722885401993D220120885402A900207D
:0ACFAE00087002A8007803B000BD6F
:10CFB80000B585B00390029101926946002008707F
:10CFC80003983C21405C012803D104A90220087081
:10CFD80075E003993C22012088540198002815D156
:10CFE80003980068029B19685A68DB68F6F760FDC9
:10CFF8000398016888690C229043886102988268C6
:10D008000398016888691043886151E001980428F1
:10D0180017D103980068029B19685A68DB6800F00A
:10D0280052F8039801688869032292029043886144
:10D038000298806802020398016888691043886131
:10D0480036E00198082815D103980068029B1968F2
:10D058005A68DB6800F009FF03980168C8690C2268
:10D068009043C8610298826803980168C8691043B0
:10D07800C8611DE001980C2817D103980068029B2D
:10D0880019685A68DB6800F055F803980168C869A0
:10D09800032292029043C8610298806802020398B2
:10D0A8000168C8691043C86102E069460120087038
:10D0B80003993C2200208854009804A9087004A809
:06D0C800007805B000BD78
:10D0CE0086B005900491039202930598006A009031
:10D0DE000599086A102290430862059880690190AC
:10D0EE0001980321090288430190039801020198D7
:10D0FE000843019001980F2109038843019002987B
:10D10E00000381B20198084301900099A020814349
:10D11E00009104990901014000980843009001987C
:0ED12E000599886100980599086206B070475F
:10D13C0086B005900491039202930598006A0090C2
:10D14C000599086A01221203904308620598C06988
:10D15C000190019803210902884301900398010270
:10D16C0001980843019001980F210903884301900D
:10D17C000298000381B201980843019000990520A0
:10D18C00400381430091049909030140009808432E
:10D19C00009001980599C86100980599086206B03D
:02D1AC007047CA
:10D1AE0081B0009000982821405CC00700280AD06A
:10D1BE000098006840680121490488430099CA6AB2
:10D1CE0010430968486000982821405C80070028B9
:10D1DE000AD5009800684068012109048843009927
:10D1EE000A6B10430968486000982821405C40078C
:10D1FE0000280AD5009800684068012189048843F8
:10D20E0000994A6B10430968486000982821405CD9
:10D21E00000700280AD50098006840680121C9035C
:10D22E00884300998A6B104309684860009828214A
:10D23E00405CC00600280AD500980068806801216D
:10D24E00090388430099CA6B1043096888600098E7
:10D25E002821405C800600280AD500980068806866
:10D26E0001214903884300990A6C104309688860BC
:10D27E0000982821405C4006002819D500980068C7
:10D28E004068012109058843009A536C18431268BF
:10D29E0050600098406C88420AD10098006840683F
:10D2AE0003214905884300998A6C10430968486038
:10D2BE0000982821405C000600280AD500980068D6
:10D2CE0040680121C90488430099CA6C104309685B
:06D2DE00486001B070473A
:10D2E40082B00190019880214058212835D10198BD
:10D2F4006A21405A694608806846008800282CD074
:10D3040001985621405A00280DD101980168886877
:10D314000122D20590438860019801680868402280
:10D324001043086019E001980068C06900060028ED
:10D334000ED50199086D0078096888620199086D15
:10D34400401C086501995622885A401E8852FFE7FE
:0ED354000098401E69460880CEE702B0704780
:10D3620081B0009000988021405821281FD1009858
:10D372005621405A00280CD1009801680868802282
:10D3820090430860009801680868402210430860D2
:10D392000DE00099086D0078096888620099086DAF
:10D3A200401C086500995622885A401E885201B0D6
:02D3B2007047C2
:10D3B40000B585B0049004986021405A02A9088001
:10D3C400049884214058222831D104980068406A86
:10D3D40001A908800498806D03900198029908407F
:10D3E400039908800499886D801C8865049A5E21DD
:10D3F400505A401E50520498405A002816D104989E
:10D404000168086809225201904308600498016881
:10D4140088680122904388600499842220208850DF
:10D4240004990020C866049800F0F9FD05E004980A
:0ED434000168886908221043886105B000BDB8
:10D4420000B583B0029002986021405A01A9088079
:10D4520002988421405822282FD102980068406AFD
:10D46200694608800098019908400299896D087000
:10D472000299886D401C8865029A5E21505A401EAE
:10D4820050520298405A002816D102980168086842
:10D4920009225201904308600298016888680122BB
:10D4A20090438860029984222020885002990020AB
:10D4B200C866029800F0B4FD05E002980168886928
:0AD4C20008221043886103B000BD8A
:10D4CC0030B587B00A9C06900591049203A803809E
:10D4DC000088002803D003A80088032802D303A9DE
:10D4EC000120088003A800880930029004980028C5
:10D4FC0002D00498012802D10298401C0290069890
:10D50C000A99059A049B03AC2488029D019500940A
:10D51C00F7F770FD069900204877069988840699DC
:10D52C000884069926228854069908770699C88398
:0AD53C0006992222885407B030BD82
:10D5460000B581B0009000980168086840229043B9
:10D5560008600099802220208850009900200867E2
:0AD56600009800F05FFD01B000BD69
:10D5700000B581B00090009926220C208854009AB2
:10D580001068FF21283151188B239B00D25AF7F7DE
:06D5900071F801B000BDBE
:10D5960081B0009000998B2082000020885001B055
:02D5A6007047CC
:10D5A80081B0009000994520C20000208850009961
:06D5B800087501B0704788
:10D5BE0000B585B0049000200390049827300290A7
:10D5CE000498FFF7E1FF02980078049AFF212831B2
:10D5DE00019150540398401C0390049840180299EE
:10D5EE00039A0B7800F0D8FD019903900498401827
:10D5FE00039900F0A7FD0390039804998B229200E3
:10D60E0088500498FFF7ADFF0498FFF7C6FF05B0EA
:02D61E0000BD4D
:10D6200084B003900291019200930298803002909E
:10D6300002980399009A88540098401C0090019821
:10D640000399009A88540098401C0090009804B0F8
:02D65000704721
:10D6520030B593B014460546169A11A8058010AD50
:10D6620029800FA90C800EAC23800DAB1A800022FA
:10D67200805E895E884204DC002111A8405E04902D
:10D6820003E000210FA8405E049004980C90002251
:10D6920010A8805E0EA9895E884204DC002110A8D1
:10D6A200405E039003E000210EA8405E03900398C1
:10D6B2000B9000220FA8805E11A9895E884204DDCA
:10D6C20000210FA8405E029003E0002111A8405EF5
:10D6D200029002980A9000220EA8805E10A9895E2C
:10D6E200884204DD00210EA8405E019003E0002183
:10D6F20010A8405E01900198099000210DA8405E9B
:10D7020008900A980C99401A07900798002803D1AC
:10D7120012A90020088013E009980B9A811A089830
:10D722000C9BC01A48430A99C91A514340180690E3
:10D7320006980799FDF793FF0590059812A90880AE
:0AD74200002112A8405E13B030BDB4
:02D74C00704724
:02D74E00704722
:02D75000704720
:02D7520070471E
:02D7540070471C
:10D7560008D1002806D1F54204D801D3002A01D108
:10D766006D0D09D10020C143090DC904F0BDF9D1E1
:10D776001242F7D1640DF5D00020C143490549088E
:10D78600A6E000206146F0BDF0B50127FF070E00B8
:10D796005E403E40B446BE0A4C18DD18F442D7D26D
:10D7A600F542E4D2640DECD06D0DEAD06419C902DD
:10D7B6003943460DC0023143DB023B43DB0A10B45A
:10D7C6008E4685B297B26F43140C6C433E0CA41977
:10D7D600260C2404BFB227439CB26C43A419190C2F
:10D7E6006943250CA4B249190D04090C6419000CEF
:10D7F60095B245433E0C76193743BFB2360C150C2D
:10D806004543AD19A6B2240CAD192E0437432E0C90
:10D8160036199DB24543AD19ACB22E0C89191D0CB3
:10D8260045436D182E04290C3443704680B295B2D8
:10D8360045433E0C76193743BFB2360C150C4543AB
:10D84600AD19A6B2AD19240C2E0437432E0C361989
:10D856009DB24543AD19ACB22E0C89191D0C45433A
:10D866006D182E043443290C75462D0C90B268436E
:10D876003E0C80190604BFB23E43070CA0B23F1807
:10D88600120C6A43D019020C80B2240CA4189AB266
:10D896006A43121914042043120C89181B0C6B439B
:10D8A600C91810BC01273D05294203D1B6194041CC
:10D8B6004941013CFF077D0D013D641B0BDB6D00FB
:10D8C600AC4209DA240500254208BE41684161419F
:0AD8D60066463143F0BD54E74EE70B
:10D8E00030B581B0044668460170206900280FD029
:10D8F0000CCC083C9A4233D26269531C6361815458
:10D90000A069616981422BD1204600F02EF827E002
:10D91000E068002809D00CCC083C9A4220D2551C63
:10D920009D4200D1002181541AE0A068002808D04F
:10D930000CCC083C9A4213D2551C9D420DD0C9B262
:10D940000CE0236A002B0BD003CC083C884207D2A2
:10D95000694601222046984702E00021920081504A
:0AD960002068401C206001B030BDBB
:10D96A0010B54269002A07D00446036A002B01D089
:0AD97A00216998470020606110BD8C
:10D9840080B5CB0606D4890501D5302100E02021DD
:06D9940000F0C3FC80BDA1
:10D99A0070B514460D460646FEF705FF01463046A9
:0AD9AA002A462346FDF70FFF70BD6B
:0AD9B40080B50068FEF752FE80BD4A
:10D9BE00C2680169914201D9D04302E0D24389186D
:06D9CE0080680818704794
:10D9D400F0B581B0154604464068A268E66880192F
:10D9E400971BBD4204D22A46FEF7CEFE751909E004
:10D9F4000E463A46FEF7C8FEF119ED1B60682A464A
:0ADA0400FEF7C2FEE56001B0F0BDC0
:10DA0E00F0B583B016460D46C7680021019002910D
:10DA1E000269F943BA4202D95418816802E05218D9
:10DA2E00816854184268C91B8C4200D30C46B4421C
:10DA3E0000D33446D01929462246FEF7A0FEE71938
:10DA4E00019881688F4200D100270299C760361B6A
:0EDA5E002D196118002EDAD1084603B0F0BD74
:10DA6C0010B50446002000290DD0002A0BD00978EF
:10DA7C0048B2002808D4002C00D021600021196085
:0EDA8C005960411E884110BD0120C04310BDED
:0EDA9A00014641391A2901D220210843704764
:0EDAA800014641391A2901D220210843704756
:10DAB60081B0009000988068012109070840000F96
:04DAC60001B07047F4
:10DACA0081B00090009880680121084001B0704739
:10DADA0082B0019000910198406900990422114096
:0CDAEA0007228A401040C84002B070477C
:10DAF60000B585B0039003980068FFF718F8019009
:10DB060003980068FFF7DEFF002842D0019800283E
:10DB16003FD103980068806805210840012808D194
:10DB260003980068F2F771FD039801680320086006
:10DB36000CE00399886D102210438865039AD16D15
:10DB460001200143D16504A9087025E0F2F7A1FB85
:10DB56000290039800688068C007002819D0F2F781
:10DB660098FB0299401A032812D30398006880682C
:10DB7600C00700280CD00399886D102210438865D1
:10DB8600039AD16D01200143D16504A9087003E011
:10DB9600DFE704A90020087004A8007805B000BDDE
:10DBA60000B583B002900298806A01900198806D5A
:10DBB6005021084238D10199886D01225202104342
:10DBC600886501980068FEF7C4FF002828D00198F0
:10DBD600807E002824D1019800680068000700288C
:10DBE6001ED501980068FEF747FF00280ED1019860
:10DBF600016848680C22904348600198806D0121B5
:10DC06000843090288430199886509E00199886DEE
:10DC16002022104388650199C86D01221043C8650A
:10DC26000198FBF798FB0DE00198806DC00600286F
:10DC360003D5019800F008F804E00198006D416BE7
:08DC46000298884703B000BDFD
:08DC4E0081B0009001B07047A5
:08DC560081B0009001B070479D
:10DC5E0082B00190009101980068072189058843E0
:0CDC6E00009908430199086002B070475B
:10DC7A0081B00090009880680121084001B0704787
:10DC8A0081B0009000988068C00F401E4142484110
:04DC9A0001B070471E
:10DC9E0082B0019000910198B42280587F21884370
:0CDCAE00009908430199885002B07047AB
:10DCBA0000B583B0034602A80370019100920021C7
:0CDCCA0040560199F3F7D9F803B000BDF3
:10DCD60000B581B000900098F3F73DF901B000BDA2
:08DCE60081B0009001B070470D
:10DCEE0086B0059004910392002002900298039949
:10DCFE008908884214D2049802998A008118805C9F
:10DD0E0000064A78120480188A7812028018C978A0
:10DD1E0040180599096808600298401C0290E5E7D2
:10DD2E0003A80078800700283DD0039803210840FF
:10DD3E00012806D1049802998900405C059909686A
:10DD4E00087003980321084002280FD10498029905
:10DD5E008A008118805C00024978401801A9088069
:10DD6E000598006800900198009908800398032197
:10DD7E000840032817D1049802998A008118805C04
:10DD8E0000024978401801A90880059800680090A3
:10DD9E0001980099088004990298800040188078B4
:10DDAE0005990968087005980068006806B0704704
:10DDBE0083B0029001A801806846027000780028A6
:10DDCE0004D001A800880299886103E001A80088A8
:08DDDE000299886203B070474E
:10DDE60083B0029001A80180029949690091009AC6
:10DDF6000188104608400004914340180299886142
:04DE060003B07047AE
:10DE0A0083B002A908700020019002986946087040
:10DE1A00684600780A2807D30198401C01900098A8
:10DE2A000A3869460870F3E701980007000E694648
:08DE3A000978084303B07047AA
:08DE420081B0009001B07047AF
:08DE4A0081B0009001B07047A7
:08DE520081B0009001B070479F
:08DE5A0081B0009001B0704797
:08DE620081B0009001B070478F
:08DE6A0081B0009001B0704787
:10DE720086B005900491039202930598006A00907F
:10DE82000599086A01221202904308620598C06946
:10DE92000190019803218843019003990198084356
:10DEA20001900198F0218843019002980001C1B2CB
:10DEB2000198084301900099052040028143009196
:10DEC20004990902014000980843009001980599BD
:0CDED200C86100980599086206B070470E
:08DEDE0081B0009001B0704713
:10DEE60086B004900391029201A90020087004985C
:10DEF6003C21405C012803D105A9022008703BE0C3
:10DF060004993C220120885402980090002806D0EB
:10DF1600009804280ED00098082817D022E004980C
:10DF26000068806E0F2188430399084304990968A5
:10DF360088661AE004980068806E0F2109028843FB
:10DF4600039908430499096888660EE004980068F6
:10DF5600806E0F21090488430399084304990968D0
:10DF6600886602E001A90120087004993C2200207D
:10DF76008854019805A9087005A8007806B070476E
:08DF860081B0009001B070476A
:08DF8E0081B0009001B0704762
:10DF960010B586B0089C0490039102A80270019304
:10DFA60004980068C06903990840401A41424841F4
:10DFB60002A9097888422AD10898401C002825D051
:10DFC600F2F767F90199401A0899884202D8089829
:10DFD60000281BD10498016808680D22520190435D
:10DFE6000860049801688868012290438860049953
:10DFF60080222020885004998422885004997C220B
:10E006000020885405A90320087003E0C8E705A985
:0CE016000020087005A8007806B010BDBE
:08E0220081B0009001B07047CD
:08E02A0081B0009001B07047C5
:10E0320083B0019001987C21405C012803D102A9A0
:10E042000220087026E001997C220120885401995F
:10E05200802224208850019800680068009001986E
:10E0620003681868012188431860009849078843AB
:10E07200009001990020486600980199096808609B
:10E0820001992020885001997C220020885402A9FD
:0CE092000020087002A8007803B070475E
:10E09E0081B00090009880214058212820D100980E
:10E0AE005621405A00280CD1009801680868802239
:10E0BE009043086000980168086840221043086089
:10E0CE000DE00099086D0078096888620099086D66
:10E0DE00401C086500995622885A401E88520BE053
:10E0EE0000980168086880229043086000980168D3
:0CE0FE00086840221043086001B0704721
:10E10A0000B585B00490039104980399891EF7F726
:10E11A00CAF9014601A80180049A03998A18511E76
:10E12A0009780902921E12788A1869460A800088BC
:10E13A000988884202D10398029002E00020C04375
:08E14A000290029805B000BD2F
:10E1520000B585B00490039104980399F7F7A7F9E5
:10E16200014602A80180029901AA1170407869460D
:10E17200087001980499039A88540398401C0390EC
:10E1820000980499039A88540398401C03900398BA
:04E1920005B000BD17
:10E1960081B000900098007D0121084001B07047D1
:10E1A60010B588B007900691059204A803700698EA
:10E1B6004078039003980190032806D0019806281A
:10E1C6000CD00198102812D01AE007980699059AE3
:10E1D60004AB1B78F7F7DFF9029018E00798069969
:10E1E600059A04AB1B78F7F74EFA02900FE00798F2
:10E1F6000699059A04AB1B78F7F7A7FA029006E092
:10E2060007980399059B0122FFF707FA02900298E7
:04E2160008B010BD7F
:10E21A0080B50520000701221103FFF7CBFD80BD61
:08E22A0080B5F8F736FA80BD5B
:0CE2320080B501204002F3F7C6FC80BD5F
:10E23E00F0B581B01E4615460C4607461846FEF749
:10E24E0090F90146002000290AD46543A54207D360
:10E25E00304639462A46FFF7A6FB2146FDF721FA3E
:04E26E0001B0F0BD4E
:04E27200C80F70471A
:10E27600F0B581B01C4615460091CA0017183E46F7
:10E28600103EB068F1682A46FFF77EFA0CCEFCF71E
:10E2960004FE009A032A0DDB183F561E2A46234623
:10E2A600FFF772FA0CCF083FFCF7F7FD761E083F22
:10E2B600012EF3D82A462346FFF766FA01B0F0BDD1
:10E2C600F0B581B01D4616460346C800022916DB86
:10E2D60000931F18083F4C1C304629460CCF083FB8
:10E2E600FCF7DBFD32462B46FFF74EFA641E083F6D
:10E2F600022CF3D8009B083306460D4600E01B1897
:10E30600083B0CCB30462946FCF7C7FD01B0F0BDF3
:08E31600C1174840401A70478E
:10E31E0070B5012A09DB0C460546561C28462146D7
:0CE32E00FFF7D7FA761E012EF8D870BD5C
:10E33A0010B50C46436A01212046FFF77BFF10BD4A
:04E34A0040207047B8
:10E34E00024601207F2901D9C043704711707047E2
:0CE35E00014661391A2900D220387047AE
:0CE36A00014661391A2900D220387047A2
:10E376004552524F52205452494D4D494E47205610
:07E38600414C5545530A000C
:0FE38D0049205265666572656E7A3D25660A0005
:0BE39C00547368756E743D25660A001E
:10E3A7002D2D2D204761696E2044726966742043C4
:07E3B700414C202D2D2D002B
:0FE3BE0041637475616C20543D256620430A004D
:10E3CD0041637574616C20493D256620412877694C
:10E3DD0074686F7574206761696E2074656D702047
:10E3ED00647269667420636F7272656374696F6EAF
:03E3FD00290A00EA
:10E400004B6F7272656B74757266616B746F723D7F
:10E410002566205B2031202F2043656C736975735E
:03E420005D0A0092
:10E423004552524F52204144535F313236305F4997
:0FE433006E7075744D757853656C6563740A006F
:10E4420046697273742073746172742064657465B2
:07E4520063746564210A00F8
:0FE459004953454E534F523A20496E69740A0099
:10E46800466C617368206F6220756E6C6F636B20F9
:07E478006572726F720A0069
:0FE47F00466C61736820206C6F636B65640A00E4
:10E48E002E2E2E466C61736820756E6C6F636B65F5
:03E49E00640A000D
:10E4A1004F5554505554535F4C56505F5348554E39
:10E4B100545F4F56455254454D5045524154555263
:03E4C100450A0009
:0FE4C4004F5554505554204C5650204F4B0A0082
:10E4D3004F5554505554535F4F56505F5348554E04
:10E4E300545F4F56455254454D5045524154555231
:03E4F300450A00D7
:0FE4F6004F5554505554204F5650204F4B0A004D
:07E50500286E756C6C290003
:10E50C004A616E75617279004665627275617279E5
:10E51C00004D6172636800417072696C004D6179E5
:10E52C00004A756E65004A756C79004175677573A4
:10E53C00740053657074656D626572004F63746F1F
:10E54C00626572004E6F76656D626572004465633C
:07E55C00656D6265720000AD
:07E56300414D00504D000086
:0FE56A0025612025622025652025542025590094
:0EE5790075617274206572726F72200A0D0057
:10E587002D2D2D204761696E202043414C202D2DD4
:02E597002D0055
:10E599004144535F313236305F4261747465727938
:10E5A90043757272656E744761696E43616C696225
:10E5B900726174696F6E53746172743A2045525274
:10E5C9004F5220494E2043414C4942524154494FF0
:10E5D9004E2C204E4F205245464552454E4345202C
:0AE5E90043555252454E54210A00DA
:0AE5F30054736869703D25660A0044
:10E5FD002D2D2D204761696E202043414C20454E25
:06E60D0044452D2D2D00F7
:0EE6130064656C746120543D256620430A0046
:0AE6210052656620493D25660A0097
:10E62B004552524F52204144535F313236305F5383
:10E63B006574436F6E76657273696F6E4D6F64654B
:02E64B000A00C3
:10E64D004E6F726D616C2073746172742077697492
:10E65D00686F757420454550524F4D206368616E4B
:0EE66D006765732064657465637465640A00F4
:10E67B00454550524F4D2046554C4C205245535416
:06E68B004F5245210A0078
:10E69100454550524F4D2053544F524520434F4E04
:06E6A100464947210A0072
:0EE6A7004144533132363020496E69740A0006
:10E6B5002E2E2E456E61626C65206C6F636B206536
:06E6C50072726F720A0080
:10E6CB002E2E2E466C617368206C6F636B20616C11
:0EE6DB007265616479206163746976650A0076
:10E6E9002E2E2E466C617368206F6220756E6C6FDA
:06E6F900636B65640A007A
:10E6FF00466C617368204F7074696F6E62797465D0
:10E70F002070726F6772616D6D206661696C6564F0
:02E71F000A00EE
:10E721002E2E2E44697361626C65206C6F636B20C1
:10E7310070726F636573732066696E69736865646F
:02E741000A00CC
:10E743004F5554505554535F4C56505F42415454A7
:10E753004552595F554E444552564F4C54414745D7
:02E763000A00AA
:10E765004F5554505554535F4C56505F434849508C
:10E775005F4F56455254454D5045524154555245AB
:02E785000A0088
:10E787004F5554505554535F4F56505F4348495067
:10E797005F4F56455254454D504552415455524589
:02E7A7000A0066
:10E7A9004F5554505554535F4F56505F4348495045
:10E7B9005F554E444554454D504552415455524577
:02E7C9000A0044
:10E7CB0053756E646179004D6F6E64617900547599
:10E7DB006573646179005765646E65736461790074
:10E7EB00546875727364617900467269646179006B
:0AE7FB0053617475726461790000C7
:02E805004300CE
:02E807002E00E1
:10E8090056616C7565206E6F742076616C69640A57
:01E8190000FE
:10E81A004672657175656E6379204D6561737572AF
:09E82A006564203D2025640A000C
:10E83300492028776974686F757420636F6D7065FC
:0DE843006E736174696F6E293D25660A00D1
:10E850004552524F52204144535F313236305F535C
:10E860006574496E7465726E616C52656665726539
:05E870006E63650A0063
:0DE8750057726974696E6720534E210A00C6
:10E88200554E4B4E4F574E20434F4D4D414E440A2D
:01E892000085
:10E89300537461727420656E61626C652072656188
:10E8A300646F75742070726F74656374696F6E0A38
:01E8B3000064
:10E8B4002E2E2E466C61736820756E6C6F636B0A26
:01E8C4000053
:10E8C500466C617368204F7074696F6E6279746508
:09E8D500206C6F636B65640A009E
:10E8DE002E2E2E456E61626C65206C6F636B207000
:10E8EE00726F636573732066696E69736865640A17
:01E8FE000019
:10E8FF00466C617368204F7074696F6E62797465CE
:0DE90F002070726F6772616D6D65640A00A3
:10E91C004F5554505554535F4C56505F4F564552BB
:09E92C0043555252454E540A00B5
:10E935004F5554505554535F4F56505F42415454B0
:10E945004552595F4F564552564F4C544147450A1B
:01E9550000C1
:10E956004F5554505554535F4F56505F4F5645527E
:09E9660043555252454E540A007B
:05E96F002D494E460099
:05E974002D696E660034
:05E979002B494E460091
:05E97E002B696E66002C
:10E9830000000000000054545220524547474553AD
:01E993000083
:09E994005465726D696E616C003E
:09E99D00256D2F25642F2579005A
:09E9A60025483A254D3A2553009D
:10E9AF0053756E004D6F6E005475650057656400AA
:0DE9BF0054687500467269005361740000D1
:10E9CC004A616E00466562004D61720041707200D2
:10E9DC004D6179004A756E004A756C00417567008F
:10E9EC00536570004F6374004E6F7600446563008E
:01E9FC00001A
:01E9FD000019
:0DE9FE000007032004170201085710408095
:10EA0B004552524F52204144535F313236305F539F
:0CEA1B00657444617461526174650A0006
:10EA27004B6F7272656B74757266616B746F723D52
:04EA370025660A0046
:10EA3B002D2D2D204761696E204472696674204329
:0CEA4B00414C20454E4445202D2D2D004F
:10EA57004552524F52204144535F313236305F5353
:0CEA6700657443686F704D6F64650A00B1
:10EA7300454550524F4D20776173206368616E673F
:10EA8300656421205765206E65656420746F20706E
:10EA9300726573657276652063616C696272617415
:10EAA300696F6E20616E642073657474696E677339
:08EAB3002064617461210A0076
:10EABB00454550524F4D20464143544F52592052D9
:10EACB004553544F52452F555044415445210A004C
:10EADB007265616420636F6E6669672E2E2E0A0065
:10EAEB00666163746F727920726573746F72652ED1
:04EAFB002E2E0A00B1
:10EAFF00466C61736820756E6C6F636B2065727204
:04EB0F006F720A0017
:10EB130050524F54454354494F4E3A204F425F524F
:0CEB230044505F4C4556454C5F300A00E2
:10EB2F0050524F54454354494F4E3A204F425F5233
:0CEB3F0044505F4C4556454C5F310A00C5
:10EB4B0050524F54454354494F4E3A204F425F5217
:0CEB5B0044505F4C4556454C5F320A00A8
:10EB67004F5554505554535F4C56505F5348554E6C
:10EB7700545F554E44455254454D504552415455A6
:04EB870052450A00E9
:10EB8B004F5554505554535F4F56505F5348554E45
:10EB9B00545F554E44455254454D50455241545582
:04EBAB0052450A00C5
:10EBAF0030313233343536373839414243444546B4
:10EBBF0030313233343536373839616263646566E4
:04EBCF004E414E0065
:04EBD3006E616E0001
:10EBD70020202020202020202068282828282020C6
:10EBE700202020202020202020202020202020201E
:10EBF70048101010101010101010101010101010D6
:10EC07008484848484848484848410101010101075
:10EC170010818181818181010101010101010101CE
:10EC27000101010101010101010101101010101082
:10EC3700108282828282820202020202020202029F
:10EC47000202020202020202020202101010102047
:10EC580019ED00089D000020361400002BED000877
:10EC68000000002078EC00089D000000EBC80008B8
:10EC780088B00590049103A90020087005980290B7
:10EC8800049801901549086801229204104308600D
:10EC9800EFF3108006900698009072B603A80078EB
:10ECA8003F280ED801980068029908600198001D55
:10ECB80001900298001D02900398401C03A9087057
:10ECC800ECE707480068C003002800D5F9E700987A
:10ECD8000790079880F3108808B070471420024006
:10ECE800102002405CC800085CC800085CC8000826
:10ECF8005CC800085CC8000804000000C40F0020BD
:10ED0800C80F0020CC0F00200024F40001000000F0
:10ED1800206861680834002200E042540139FCD5BB
:02ED2800704732
:10ED2A0020686168A2680C3401E08B5C8354013A64
:04ED3A00FBD570474E
:020000040801F1
:04C7FC00AB1898A03E
:040000050800C8F532
:00000001FF
